:100000000C947F160C94B0160C94B0160C94B01689
:100010000C94B0160C94B0160C94B0160C94B01648
:100020000C94B0160C94B0160C94B0160C94B01638
:100030000C94B0160C94E6580C94B0160C94B016B0
:100040000C94B0160C94BEB20C94B0160C94B0166E
:100050000C94B0160C94B0160C94D47C0C949C5850
:100060000C94B0160C947B4B0C94B0160C94B016F8
:100070000C94B0160C94B0160C94B0160C94B016E8
:100080000C94B0160C94B0160C94B0160C94B016D8
:100090000C94B0160C94B0160C94B0160C94B016C8
:1000A0000C94B0160C94B0160C94B0160C94B016B8
:1000B0000C94B0160C94B0160C94B0160C94B016A8
:1000C0000C94B0160C94B0160C94B0160C94B01698
:1000D0000C94B0160C94B0160C942B580C94EC574E
:1000E0000C94B01655317231A331C031D531FE3187
:1000F0006B32D1327A33B437C237BB37E237E637A7
:1001000000385B3C153861388838AF38D8382E391C
:100110003F3950396139723983395B3C663B5B3C0E
:10012000713BE13BE73B073C81C084C073C077C0B3
:100130007DC0BBC088C08CC092C096C09AC0A0C011
:10014000A4C0A8C0BBC0AEC0B2C0B6C01EC623C645
:1001500028C632C63CC6B5C646C64EC656C660C6DA
:100160006AC674C683C68DC6B5C697C6A1C6ABC6D9
:10017000084AD73B3BCE016E84BCBFFDC12F3D6C0E
:1001800074319ABD56833DDA3D00C77F11BED9E474
:10019000BB4C3E916BAAAABE000000803F05A84C54
:1001A000CDB2D44EB93836A9020C50B99186880820
:1001B0003CA6AAAA2ABE000000803F004E414E493C
:1001C0004E495459494E46CDCCCC3D0AD7233C1715
:1001D000B7D13877CC2B329595E6241FB14F0A0062
:1001E0000020410000C84200401C4620BCBE4CCA52
:1001F0001B0E5AAEC59D74434F4D4D554E4943415C
:1002000054494F4E0044525952554E004552524F98
:10021000525300494E464F004543484F0047322F46
:1002200047332062616420706172616D657465722C
:10023000730A00206F6620004D424C20473239205F
:10024000706F696E74200059206F7574206F66207E
:1002500072616E67652028312D35292E0A005820DD
:100260006F7574206F662072616E67652028312D6E
:1002700035292E0A004D6573682070726F62696EB1
:100280006720646F6E652E0A005374617274206D6E
:100290006573682070726F62696E67207769746831
:1002A0002022473239205331222066697273742E1E
:1002B0000A004732380A47323920533200537461FA
:1002C00074653A20004D65736820626564206C6532
:1002D00076656C696E6720686173206E6F2064615B
:1002E00074612E0A0053206F7574206F662072614E
:1002F0006E67652028302D35292E0A004D657368FC
:1003000020706F696E742063616E6E6F7420626519
:10031000207265736F6C7665640A00456E642066B2
:10032000696C65206C6973740A00426567696E20A8
:1003300066696C65206C6973740A00286E6F2066AC
:10034000696C6529005344207072696E74696E6728
:10035000206279746520004E6F74205344207072BF
:10036000696E74696E670A0043757272656E7420F7
:1003700066696C653A20005072696E742074696D0C
:10038000653A20006F6E2E0A006F66662E0A0047DF
:1003900032362044656275672000180213020C0291
:1003A0000502F7016F66660044454255473A004B27
:1003B000494C4C45442E20004D3131332053006FC1
:1003C0006B002C20002C2000544845524D414C5FBE
:1003D00050524F54454354494F4E004155544F528B
:1003E00045504F52545F53445F535441545553004A
:1003F000454D455247454E43595F50415253455232
:1004000000434153455F4C494748545F4252494776
:1004100048544E45535300544F47474C455F4C4951
:100420004748545300534F4654574152455F504F2D
:10043000574552004255494C445F50455243454E42
:1004400054004C4556454C494E475F444154410089
:100450005A5F50524F4245004155544F4C45564506
:100460004C005052494E545F4A4F420050524F4741
:1004700052455353004155544F5245504F52545FCB
:1004800054454D5000564F4C554D4554524943002C
:10049000454550524F4D0053455249414C5F584FCE
:1004A0004E5F584F4646004649524D574152455FB0
:1004B0004E414D453A4D61726C696E20312E312EA0
:1004C0003920284769746875622920534F55524373
:1004D000455F434F44455F55524C3A68747470739E
:1004E0003A2F2F6769746875622E636F6D2F4D61A7
:1004F000726C696E4669726D776172652F4D6172BB
:100500006C696E2050524F544F434F4C5F564552CA
:1005100053494F4E3A312E30204D414348494E45C4
:100520005F545950453A3344205072696E74657275
:100530002045585452554445525F434F554E543A06
:100540003120555549443A63656465326132662D00
:10055000343161322D343734382D396231322D63E4
:1005600035356336326633363766660A002F2F20FC
:1005700000205400205200416363656C6572617411
:10058000696F6E3A2050005741524E494E47212024
:100590004C6F77205A204A65726B206D6179206C10
:1005A00065616420746F20756E77616E7465642078
:1005B0007061757365732E0A00546F6F20666172E7
:1005C0002066726F6D207265666572656E63652068
:1005D000706F696E740A0020466C6F773A200000D5
:1005E00001363726032BFFFFFF3C3D382AFFFFFF74
:1005F000FF2E303E12FFFFFFFFFFFFFF0809FF2C19
:10060000071A1C18FFFFFF08440A2C4324221E204F
:10061000643A0020693A0020703A00496E76616CB5
:1006200069642065787472756465720A0043290AEA
:100630000061626C656420286D696E2074656D7060
:100640002000436F6C642065787472756465732054
:10065000617265200020643A0020693A0020703AF7
:10066000004E6F2063617365206C696768740A00CF
:10067000454550524F4D204F4B0A00205A004475BB
:10068000616C20456E6473746F702041646A757389
:10069000746D656E7420286D6D293A20003F4B20E3
:1006A00076616C7565206F7574206F662072616E5F
:1006B00067652028302D3130292E0A00416476618B
:1006C0006E6365204B3D0041637469766520457813
:1006D0007472756465723A2000496E76616C696463
:1006E0002065787472756465720A0043616E6E6F7E
:1006F0007420656E746572207375626469723A2045
:10070000004739310A4731205A2D302E310A4739F6
:1007100030005370656369616C204D656E753A20D9
:100720005A20446F776E20302E310A004739310A43
:100730004731205A2D302E30320A4739300053705D
:10074000656369616C204D656E753A205A20446F6F
:10075000776E20302E30320A004739310A47312077
:100760005A2B302E30320A47393000537065636996
:10077000616C204D656E753A205A20557020302EE0
:1007800030320A004739310A4731205A2B302E3196
:100790000A473930005370656369616C204D656E9E
:1007A000753A205A20557020302E310A00473239D0
:1007B000205332005370656369616C204D656E751E
:1007C0003A204E657874204D65736820506F696ECD
:1007D000740A0047323920533100537065636961F0
:1007E0006C204D656E753A205374617274204D65AE
:1007F0007368204C6576656C696E670A004D31340C
:100800003020533630005370656369616C204D654C
:100810006E753A2050726568656174204265640A9D
:10082000004D353032005370656369616C204D6551
:100830006E753A204C6F61642046572044656661AE
:10084000756C74730A004D35303000537065636900
:10085000616C204D656E753A205361766520454583
:1008600050524F4D0A004D33303320452D31205327
:100870003630204336205531005370656369616C12
:10088000204D656E753A204175746F2054756E6504
:1008900020486F74626564205069640A004D3130ED
:1008A0003620533230340A4D333033204530205314
:1008B0003231302043362055310053706563696111
:1008C0006C204D656E753A204175746F2054756EBD
:1008D0006520486F74656E64205049440A003C539B
:1008E00070656369616C5F4D656E753E003C537069
:1008F000656369616C5F4D656E753E002F002F006A
:100900002F002F2E2E0A002F2E2E002F2E2E003CD1
:100910005370656369616C5F4D656E753E0A003C9E
:100920005370656369616C204D656E753E003C5384
:1009300070656369616C204D656E753E003C4C6F5F
:1009400061642046572044656661756C74733E008F
:100950003C4C6F61642046572044656661756C7439
:10096000733E003C4175746F2054756E6520486F6E
:1009700074626564205049443E003C4175746F20A8
:1009800054756E6520486F74626564205049443E1A
:10099000003C4175746F2054756E6520486F746516
:1009A0006E64205049443E003C4175746F2054757C
:1009B0006E6520486F74656E64205049443E003C6B
:1009C000457869743E003C457869743E003C53614B
:1009D000766520454550524F4D3E003C536176654B
:1009E00020454550524F4D3E003C4E657874204D99
:1009F00065736820506F696E743E003C4E65787474
:100A0000204D65736820506F696E743E003C5374CE
:100A1000617274204D657368204C6576656C696EF3
:100A2000673E003C5374617274204D657368204CBE
:100A30006576656C696E673E003C507265686561FD
:100A400074206265643E003C507265686561742084
:100A50006265643E003C5A20446F776E20302E3130
:100A60003E003C5A20446F776E20302E313E003CD1
:100A70005A20446F776E20302E30323E003C5A2090
:100A8000446F776E20302E30323E003C5A20557035
:100A900020302E30323E003C5A20557020302E300F
:100AA000323E003C5A20557020302E313E003C5AD8
:100AB00020557020302E313E0056313136004A33F9
:100AC0003320004D3530300A4D3432302053310A56
:100AD0004731205A313020463234300A47312058CD
:100AE00030205930204636303030004A3232004A09
:100AF0003232004731205A3520463234300A4731ED
:100B00002058313930205932302046363030300AC2
:100B10004731205A302046323430004731205A3590
:100B200020463234300A473120583139302059318B
:100B300039302046363030300A4731205A3020468E
:100B4000323430004731205A3520463234300A479B
:100B5000312058313930205932302046363030304B
:100B60000A4731205A302046323430004739310AA2
:100B70004731205A313020463234300A4739300A62
:100B80004732380A4732390A473120583230205923
:100B900032302046363030300A4731205A30204635
:100BA000323430004A3032004A3132004731205A64
:100BB0003130004F4B004731205A31300047393037
:100BC0000047312045256946353030004731204502
:100BD0002D302E314625690047312045302E3146D3
:100BE0002569004731205A2569462569004731208B
:100BF0005A2D302E31462569004731205A302E318A
:100C00004625690047312059256946256900473145
:100C100020592D302E314625690047312059302E7C
:100C20003146256900473120582569462569004726
:100C30003120582D302E314625690047312058305B
:100C40002E31462569004739310047323800473296
:100C500038205A004732382059004732382058008F
:100C60004132305620004731205A3130004A30346A
:100C7000004A3231004A3230004B494C4C45442E38
:100C800020004A303400454E4400464E20004A3091
:100C900032003939393A393939004D004800413785
:100CA000562000413656202D2D2D004A303200416D
:100CB000365620005A3A2000593A2000583A20006F
:100CC0004135560041345620004133562000413210
:100CD000562000413156200041305620004D383416
:100CE000004A3136004A3138004739310A4731204D
:100CF0005A313020463234300A473930004A3134D4
:100D0000004A3030004A3031004A31300024F4D4F7
:100D10003050C38E20C2A24017828B7011127A917C
:100D20000D816CD90AA861E108C758660761514373
:100D3000061E4B5D05C145A7041A411104093D98E3
:100D400003713931034036DB0265339102D43054EC
:100D500002802E1D02632CEE01752AC501B028A069
:100D600001102781018F2564012B244B01E02234DF
:100D700001AC211F018D200D01801FFC00841EEDA0
:100D800000971DDF00B81CD200E61BC600201BBC6C
:100D900000641AB200B219A8000A19A0006A1899D2
:100DA00000D117910040178B00B516840031167ED4
:100DB00000B31579003A157300C7146F0058146A10
:100DC00000EE1366008813630025135E00C7125BF4
:100DD000006C12570015125400C111510070114FD0
:100DE0000021114B00D61049008D104700461044D9
:100DF0000002104200C00F4000800F3E00420F3C36
:100E000000060F3B00CB0E3800930E37005C0E350A
:100E100000270E3400F30D3200C10D3100900D306B
:100E200000600D2E00320D2D00050D2C00D90C2B6D
:100E300000AE0C2900850C29005C0C2700350C271E
:100E4000000E0C2600E80B2400C40B2400A00B238A
:100E5000007D0B23005A0B2100390B2100180B20B9
:100E600000F80A1F00D90A1E00BB0A1E009D0A1DB9
:100E700000800A1D00630A1C00470A1B002C0A1B85
:100E800000110A1A00F7091A00DD091900C409192E
:100E900000AB091900920917007B091800630917B4
:100EA000004C09160036091600200916000A09151B
:100EB00000F5081500E0081400CC081400B8081468
:100EC00000A4081400900813007D0812006B08139A
:100ED00000580812004608120034081100230811B7
:100EE000001208110001081100F0071000E00710BF
:100EF00000D0071000C0071000B0070F00A10710B6
:100F00000091070E0083070F0074070F0065070E9E
:100F10000057070E0049070E003B070D002E070E75
:100F20000020070D0013070D0006070D00F9060C41
:100F300000ED060D00E0060C00D4060C00C8060CFF
:100F400000BC060C00B0060C00A4060B0099060CB1
:100F5000008D060B0082060B0077060B006C060B5B
:100F60000061060A0057060B004C060A0042060AFA
:100F70000038060A002E060A0024060A001A060A8D
:100F8000001006090007060A00FD050900F405091E
:100F900000EB050900E2050900D9050900D00509A3
:100FA00000C7050900BE050900B5050800AD050824
:100FB00000A50509009C050800940508008C05089B
:100FC00000840508007C050800740508006C05070E
:100FD00000650508005D050700560508004E050779
:100FE00000470507004005080038050700310507E0
:100FF000002A050700230507001C05060016050743
:10100000000F0507000805060002050700FB04069F
:1010100000F5040700EE040600E8040600E20407F9
:1010200000DB040600D5040600CF040600C9040650
:1010300000C3040600BD040600B7040600B10405A1
:1010400000AC040600A6040600A00405009B0406EC
:101050000095040500900406008A04050085040537
:1010600000800406007A040500750405007004057C
:10107000006B04050066040500610405005C0405BE
:101080000057040500520405004D040500480405FE
:1010900000430405003E0404003A0405003504053D
:1010A00000300404002C0405002704040023040578
:1010B000001E0404001A04040016040500110404B0
:1010C000000D0404000904050004040400000404E5
:1010D00000FC030400F8030400F4030400F003041C
:1010E00000EC030400E8030400E4030400E003044C
:1010F00000DC030400D8030400D4030400D003047C
:1011000000CC030400C8030300C503030024F40457
:10111000D9201BC40C5C0E9804C4095F02650771DA
:1011200001F405F900FB04B30048048700C103691A
:10113000005803550003034500BE023A0084023103
:101140000053022A002902250004022000E4011CA9
:1011500000C8011900AF01170098011400840113A1
:1011600000710110006101100051010E0043010DDA
:101170000036010B002B010B0020010B00150109AB
:10118000000C01090003010800FB000800F300083F
:1011900000EB000700E4000600DE000600D80006B1
:1011A00000D2000600CC000500C7000500C2000503
:1011B00000BD000400B9000400B5000400B1000443
:1011C00000AD000400A9000400A5000300A2000374
:1011D000009F0004009B000300980003009500029C
:1011E0000093000300900003008D0002008B0003B9
:1011F00000880002008600020084000300810002D3
:10120000007F0002007D0002007B000200790002E6
:1012100000770001007600020074000200720001F5
:1012200000710002006F0002006D0001006C0002FE
:10123000006A000100690002006700010066000109
:10124000006500010064000200620001006100010D
:1012500000600001005F0002005D0001005C000111
:10126000005B0001005A0001005900010058000114
:101270000057000100560001005500010054000114
:101280000053000000530001005200010051000112
:1012900000500001004F0001004E0000004E000110
:1012A000004D0001004C0001004B0000004B00010C
:1012B000004A000100490001004800000048000108
:1012C0000047000100460000004600010045000004
:1012D00000450001004400010043000000430001FC
:1012E00000420000004200010041000000410001F6
:1012F00000400001003F0000003F0001003E0000F0
:10130000003E0001003D0000003D0001003C0000E7
:10131000003C0000003C0001003B0000003B0001DD
:10132000003A0000003A00010039000000390001D5
:1013300000380000003800000038000100370000CD
:1013400000370001003600000036000000360001C2
:1013500000350000003500000035000100340000B9
:1013600000340000003400010033000000330000AE
:1013700000330001003200000032000000320001A2
:101380000031000000310000003100010030000099
:101390000030000000300001002F0000002F00008E
:1013A000002F0000002F0001002E0000002E000082
:1013B000002E0001002D0000002D0000002D000077
:1013C000002D0001002C0000002C0000002C00006B
:1013D000002C0001002B0000002B0000002B00005F
:1013E000002B0001002A0000002A0000002A000053
:1013F000002A000100290000002900000029000047
:101400000029000000290001002800000028000039
:10141000002800000028000000280001002700002C
:10142000002700000027000000270000002700011F
:101430000026000000260000002600000026000014
:101440000026000100250000002500000025000006
:1014500000250000002500000025000100240000F8
:1014600000240000002400000024000000240001EB
:1014700000230000002300000023000000230000E0
:1014800000230000002300000023000100220000D0
:1014900000220000002200000022000000220000C4
:1014A00000220001002100000021000000210000B6
:1014B00000210000002100000021000000210001A7
:1014C000002000000020000000200000002000009C
:1014D000002000000020000000200000002000018B
:1014E000001F0000001F0000001F0000001F000080
:1014F000001F0000001F0000001F0001001E000070
:10150000001E0000001E0000001E000000232C0032
:1015100000B8220000561800003A0F0000B808007A
:1015200000B1040000710200003E010000696E205D
:101530006D6F76655F746F282920666565645F76D8
:10154000616C756520666F722058593A002C2065D1
:10155000793D0029202D3E202865783D002C207300
:10156000793D0020436F6E6E656374696E67207706
:1015700069746820766572746963616C206C696E49
:1015800065202873783D002C2065793D0029202DA9
:101590003E202865783D002C2073793D0020436F64
:1015A0006E6E656374696E67207769746820686F12
:1015B00072697A6F6E74616C206C696E6520287335
:1015C000783D003F53706563696669656420582CF7
:1015D0005920636F6F7264696E617465206F7574F2
:1015E000206F6620626F756E64732E0A003F28526A
:1015F0002965706561742076616C7565206E6F7405
:1016000020706C61757369626C653B206D757374D5
:10161000206265206174206C6561737420312E0A2C
:10162000003F2852296570656174206D75737420C0
:1016300062652073706563696669656420776865B3
:101640006E206E6F74207573696E6720616E204C1A
:1016500043442E0A003F53706563696669656420E0
:101660006E6F7A7A6C652074656D706572617475E1
:101670007265206E6F7420706C61757369626C6541
:101680002E0A003F53706563696669656420666968
:101690006C616D656E742073697A65206E6F74205D
:1016A000706C61757369626C652E0A003F537065DA
:1016B000636966696564207072696D65206C656E2A
:1016C000677468206E6F7420706C61757369626CEA
:1016D000652E0A003F5072696D65206C656E6774F7
:1016E00068206D7573742062652073706563696628
:1016F000696564207768656E206E6F742075736904
:101700006E6720616E204C43442E0A003F53706583
:10171000636966696564206E6F7A7A6C65207369A7
:101720007A65206E6F7420706C61757369626C6588
:101730002E0A003F537065636966696564205265CF
:101740007472616374696F6E204D756C7469706C2E
:10175000696572206E6F7420706C61757369626C5C
:10176000652E0A003F52657472616374696F6E2062
:101770004D756C7469706C696572206D7573742039
:101780006265207370656369666965642E0A003F4F
:10179000537065636966696564206C617965722060
:1017A000686569676874206E6F7420706C6175730A
:1017B00069626C652E0A003F5370656369666965EE
:1017C00064206265642074656D7065726174757201
:1017D00065206E6F7420706C61757369626C652032
:1017E0002834302D31343043292E0A004732362038
:1017F000636F6D6D616E6420737461727465642EC5
:101800002057616974696E6720666F722068656130
:101810007465722873292E0A00024A3135004A3154
:1018200032004A3137002020506C616E6E65724282
:10183000756666657242797465733A200020467257
:101840006565204D656D6F72793A2000436F6D704C
:10185000696C65643A204A616E2020342032303150
:10186000390A00207C20417574686F723A20286420
:101870006176696472616D69726F2C20666F722087
:10188000416E796375626963206933204D656761D4
:10189000290A00323031392D30312D303200204CC0
:1018A00061737420557064617465643A2000312E50
:1018B000312E390A004D61726C696E0020536F66DB
:1018C00074776172652052657365740A00205761F0
:1018D000746368646F672052657365740A00204200
:1018E000726F776E206F75742052657365740A008D
:1018F0002045787465726E616C2052657365740A58
:1019000000506F77657255700A0073746172740AC3
:10191000004D3234004D3233202573006175746FF1
:1019200025692E67006572726F722077726974691B
:101930006E6720746F2066696C650A00205A3A0051
:1019400020593A0020583A00656E6473746F7073C2
:10195000206869743A2000446F6E6520736176696F
:101960006E672066696C652E0A004D32390020745E
:101970006F6F206C6F6E6720657874727573696F16
:101980006E2070726576656E7465640A0020636F00
:101990006C6420657874727573696F6E20707265FF
:1019A00076656E7465640A006F70656E20666169A5
:1019B0006C65642C2046696C653A200043616E6E4C
:1019C0006F74206F70656E20737562646972200099
:1019D0004A3035004A3233004739310A4731205AFC
:1019E0002D313020463234300A47393000534420FC
:1019F00063617264206F6B0A006F70656E526F6F67
:101A000074206661696C65640A00766F6C756D653B
:101A10002E696E6974206661696C65640A0045729E
:101A2000726F723A00534420696E6974206661696E
:101A30006C0A006563686F3A00454550524F4D206F
:101A40006461746173697A65206572726F722E0ABF
:101A500000290A002062797465733B206372632059
:101A60000053657474696E67732053746F72656494
:101A7000202800290A002062797465733B20637274
:101A80006320002073746F726564207365747469D9
:101A90006E677320726574726965766564202800CC
:101AA000202863616C63756C6174656429210A0088
:101AB00020213D2000454550524F4D2043524320A8
:101AC0006D69736D61746368202D202873746F7263
:101AD00065642920002053697A653A2000496E64C4
:101AE00065783A2000204D61726C696E3D5635353F
:101AF000290A0028454550524F4D3D00454550525A
:101B00004F4D2076657273696F6E206D69736D61DC
:101B100074636820001000C90210012C01400122EA
:101B20000170011801B0010E01F00104015002FA28
:101B300000B002F0003003E600D003DC009004D2D5
:101B4000007005C800A006BE000008B400B009AAD5
:101B500000D00BA000600E960060118C0000158272
:101B60000020197800C01D6E00A0226400B0275A22
:101B700000902C500000314600E0343C0010383218
:101B800000903A2800603C1E00A03D1400803E0AF0
:101B900000203F00002CFFFFFFFFFF0001010101BB
:101BA000016265640A002C2073797374656D20737B
:101BB000746F7070656421204865617465725F4957
:101BC000443A20004265642068656174696E67204C
:101BD0006661696C65640048656174696E6720665A
:101BE00061696C65640045312048656174696E67A0
:101BF000206661696C65640048656174696E672080
:101C00006661696C65640070012C0190012701B068
:101C1000012201C0011D01F0011801100213013061
:101C2000020E016002090190020401C002FF0000DF
:101C300003FA004003F5008003F000D003EB00201E
:101C400004E6007004E100E004DC004005D700C0B9
:101C500005D2004006CD00D006C8008007C3003082
:101C600008BE00F008B900C009B400B00AAF00B067
:101C70000BAA00D00CA500000EA000500F9B00C0C6
:101C80001096005012910000148C00C0158700B00F
:101C9000178200B0197D00D01B7800001E73004031
:101CA000206E0090226900F024640040275F0090BD
:101CB000295A00E02B5500102E500020304B001008
:101CC000324600E033410090353C00103737007059
:101CD000383200A0392D00B03A2800A03B23006024
:101CE0003C1E00103D1900903D1400103E0F007086
:101CF0003E0A00C03E0500003F0000403FFBFF8061
:101D00003FF6FFC03FF1FF453120544845524D4159
:101D10004C2052554E4157415900424544205448A9
:101D200045524D414C2052554E415741590054683F
:101D300065726D616C2052756E6177617900453115
:101D4000204572723A204D415854454D500045721D
:101D5000723A204D415854454D5020424544004D63
:101D6000415854454D5020747269676765726564C7
:101D7000004531204572723A204D494E54454D5030
:101D8000004572723A204D494E54454D502042450F
:101D900044004D494E54454D502074726967676543
:101DA000726564004D383420582059205A2045006F
:101DB000202F002042403A0020403A00256973005D
:101DC00025696D20256973002569682025696D20C6
:101DD00025697300256964202569682025696D20BF
:101DE00025697300256979202569642025696820A3
:101DF00025696D2025697300656E71756575656966
:101E00006E672022004B494C4C45442E20005072F6
:101E1000696E7465722073746F7070656420647588
:101E20006520746F206572726F72732E2046697818
:101E300020746865206572726F7220616E6420750F
:101E40007365204D39393920746F20726573746160
:101E500072742E202854656D706572617475726598
:101E60002069732072657365742E20536574206930
:101E7000742061667465722072657374617274692E
:101E80006E67290A004E6F20436865636B73756D3A
:101E90002077697468206C696E65206E756D626567
:101EA000722C204C617374204C696E653A20004E90
:101EB0006F20436865636B73756D20776974682064
:101EC0006C696E65206E756D6265722C204C617355
:101ED00074204C696E653A2000636865636B7375A6
:101EE0006D206D69736D617463682C204C6173742F
:101EF000204C696E653A20004C696E65204E756D08
:101F0000626572206973206E6F74204C6173742057
:101F10004C696E65204E756D6265722B312C204CBC
:101F2000617374204C696E653A20004D3131300088
:101F30004D33310053442072656164206572726FC5
:101F4000720A00446F6E65207072696E74696E6704
:101F50002066696C650A0020496E76616C696420B0
:101F600065787472756465722000000040C00000DE
:101F7000000000000000000057430000574300002D
:101F80004D43486F6D696E67206661696C656400DA
:101F9000206E6F7420656E74657265642E0A00464B
:101FA000696C652064656C657465643A0044656CB1
:101FB0006574696F6E206661696C65642C20466982
:101FC0006C653A200050726F7465637465642050CC
:101FD000696E0A0046696C616D656E742075736583
:101FE000643A200053746174733A20002C204C6FC3
:101FF0006E67657374206A6F623A2000546F746173
:102000006C2074696D653A200053746174733A20D2
:10201000002C204661696C65643A20002C204669DA
:102020006E69736865643A20005072696E74733A21
:10203000200053746174733A20004A3036004A30ED
:1020400034004A30370020573A004A3038004A30CE
:10205000390020573A00205A3A0020593A002043CC
:102060006F756E7420583A0020453A00205A3A00A5
:1020700020593A00583A003A004361703A00205A19
:1020800000205900580020204D61783A2000205A45
:1020900000205900580020204D696E3A20004F6EF4
:1020A00020004F666600536F667420656E6473741B
:1020B0006F70733A20004B64200023646566696E7C
:1020C000652044454641554C545F004B6920002330
:1020D000646566696E652044454641554C545F0011
:1020E0004B70200023646566696E65204445464157
:1020F000554C545F00504944204175746F74756E9F
:10210000652066696E697368656421205075742066
:10211000746865206C617374204B702C204B6920AF
:10212000616E64204B6420636F6E7374616E7473B0
:102130002066726F6D2062656C6F7720696E746FB8
:1021400020436F6E66696775726174696F6E2E6881
:102150000A00504944204175746F74756E6520669D
:1021600061696C6564212074696D656F75740A001E
:10217000453120544845524D414C2052554E41570F
:1021800041590042454420544845524D414C20524B
:10219000554E4157415900546865726D616C20522B
:1021A000756E617761790045312048656174696EAB
:1021B00067206661696C65640042656420686561DA
:1021C00074696E67206661696C6564004865617456
:1021D000696E67206661696C6564005049442041FE
:1021E00075746F74756E65206661696C6564212015
:1021F00054656D706572617475726520746F6F20BF
:10220000686967680A00204B643A2000204B693AED
:102210002000204B703A20000A20436C61737369E0
:102220006320504944200A002054753A2000204B76
:10223000753A2000206D61783A2000206D696E3A71
:10224000200020643A200020626961733A20005027
:102250004944204175746F74756E65206661696CC0
:1022600065642120426164206578747275646572CA
:10227000206E756D6265720A005049442041757484
:102280006F74756E652073746172740A004F6666B0
:102290000A004661646520486569676874200042E9
:1022A0006564204C6576656C696E672000466169DF
:1022B0006C656420746F20656E61626C6520426598
:1022C00064204C6576656C696E670A004D657368BD
:1022D00020426564204C6576656C20646174613AC7
:1022E0000A004D65736820706F696E742063616EBB
:1022F0006E6F74206265207265736F6C7665640A18
:10230000004D34323120696E636F727265637420E0
:10231000706172616D657465722075736167650ABD
:10232000007C3C3E5E2B3D3F2F5B5D3B2C2A225CBC
:1023300000627573793A2070617573656420666F09
:102340007220696E7075740A00627573793A207034
:10235000617573656420666F7220757365720A001B
:10236000627573793A2070726F63657373696E6713
:102370000A004A3135004B494C4C45442E20004B55
:10238000494C4C20636175736564206279204B4928
:102390004C4C20627574746F6E2F70696E0A004B1E
:1023A000494C4C45442E20004B494C4C20636175F0
:1023B00073656420627920746F6F206D7563682087
:1023C000696E6163746976652074696D65202D207E
:1023D00063757272656E7420636F6D6D616E643AC1
:1023E00020004A3131005072696E74657220686154
:1023F0006C7465642E206B696C6C28292063616C99
:102400006C6564210A00000040C00000000000006C
:1024100000005761726E696E673A20486F6D696E91
:10242000672042756D702044697669736F72203C35
:1024300020310A000202040000A0400000A0400079
:1024400000004000005A430000574300004D43FF86
:10245000FFFFFFFDFCFAF8F6F4F2F0EEECEAE9E734
:10246000E5E3E1E0DEDCDAD9D7D5D4D2D0CFCDCBED
:10247000CAC8C7C5C3C2C0BFBDBCBAB9B7B6B4B37A
:10248000B2B0AFADACAAA9A8A6A5A4A2A1A09E9DDA
:102490009C9A99989795949392908F8E8D8B8A8918
:1024A00088878684838281807F7E7D7B7A79787736
:1024B000767574737271706F6E6D6C6B6A69686734
:1024C000666564636261605F5E5D5C5B5A59585823
:1024D0005756555453525150504F4E4D4C4B4A4AFB
:1024E0004948474646454443424241403F3E3E3DBF
:1024F0003C3B3B3A39383837363535343332323174
:1025000030302F2E2E2D2C2B2B2A29292827272619
:10251000252524232322212120201F1E1E1D1C1CB3
:102520001B1B1A1919181817161615151413131240
:10253000121111100F0F0E0E0D0D0C0C0B0A0A09C3
:10254000090808070706060505040403030202013B
:102550000000545249474745524544006F70656E2C
:10256000003A20007A325F6D696E007A5F6D696EA5
:1025700000795F6D696E00785F6D696E00526570FD
:102580006F7274696E6720656E6473746F70207308
:1025900074617475730A000A4D65617375726564C0
:1025A00020706F696E74733A0A005A206F66667302
:1025B00065743A20004E756D20582C593A20352C00
:1025C000350A0000000001000000010000800055F5
:1025D0005555000000400033333300AAAA2A0049B1
:1025E00092240000002000C7711C0099991900D1A5
:1025F000451700555515003BB11300244912001131
:10260000111100000010000F0F0F00E3380E0043FF
:10261000790D00CCCC0C00C3300C00E8A20B006498
:10262000210B00AAAA0A00703D0A009DD8090042A9
:102630007B090092240900DCD30800888808001078
:1026400042080000000800F0C107008787070075F6
:10265000500700711C07003EEB0600A1BC06006994
:1026600090060066660600703E06006118060017B8
:10267000F4050074D105005BB00500B2900500625E
:102680007205005555050078390500B81E0500058E
:102690000505004EEC040087D40400A1BD040090A1
:1026A000A7040049920400C17D0400EE690400C73C
:1026B000560400444404005C320400082104004134
:1026C000100400000004003FF00300F8E0030026BF
:1026D000D20300C3C30300CCB503003AA803000A29
:1026E0009B0300388E0300C08103009F750300D058
:1026F000690300505E03001D53030034480300913A
:102700003D03003333030016290300381F030097ED
:10271000150300300C0300030303000BFA02004909
:10272000F10200BAE802005CE002002DD802002DA0
:10273000D0020059C80200B0C0020031B90200DA6C
:10274000B10200AAAA0200A0A30200BC9C0200FAE7
:102750009502005C8F0200DF880200828202004541
:102760007C02002776020027700200436A02007C88
:10277000640200D05E02003F590200C8530200000C
:10278000002100240027002A002D00300033000122
:10279000010000040107010A0100002200250028B1
:1027A000002B002E0031003400020100000501085A
:1027B000010B01000020002300260029002C002F1F
:1027C00000320000010000030106010901050505B2
:1027D00005070508080808020202020A0A08080498
:1027E00004040401010101010101010303030303C6
:1027F000030303040707070C0C0C0C0C0C0C0C0255
:1028000002020206060606060606060B0B0B0B0B5B
:102810000B0B0B0102102020080810204010204054
:102820008002010201080402010102040810204094
:1028300080804020100804020180040201804020B2
:1028400010080402010804020101020408102040DB
:1028500080010204081020408000000A0B02090CCD
:102860000D0E080703040100000000000000000036
:102870000000000000000000000000000000000058
:102880000000000000121110000000000000000015
:1028900000000000000000000000000000000055E3
:1028A0006E6B6E6F776E20636F6D6D616E643A2034
:1028B00022002066697273740A005A005900580099
:1028C000486F6D652000000048420000484200004B
:1028D00080400000000048617264636F646564209A
:1028E00044656661756C742053657474696E6773B2
:1028F000204C6F616465640A00B80B0000D00700CB
:10290000003C000000102700000000FA430000FA1D
:10291000430000C040000070420000A0420000A040
:10292000420000C8433333B94220286D6D2900208E
:10293000204D393030204B004C696E65617220416A
:102940006476616E63653A0A0020440020490020E5
:10295000204D3330342050002044002049002020F6
:102960004D333031205000504944207365747469F0
:102970006E67733A0A00205A0020204D3636360022
:10298000456E6473746F702061646A7573746D65ED
:102990006E743A0A00205A0020590020204732392C
:1029A000205333205800205A0020204D343230204C
:1029B00053004D65736820426564204C6576656CF4
:1029C000696E673A0A00205A0020590020204D32D3
:1029D0003036205800486F6D65206F6666736574E9
:1029E0003A0A00204500205A0020590020580020B3
:1029F000540020530020204D323035205100204516
:102A00003C6D61785F655F6A65726B3E0020583C83
:102A10006D61785F785F6A65726B3E20593C6D61CD
:102A2000785F795F6A65726B3E205A3C6D61785FB2
:102A30007A5F6A65726B3E00416476616E636564BD
:102A40003A20513C6D696E5F7365676D656E745FAA
:102A500074696D655F75733E20533C6D696E5F668A
:102A6000656564726174653E20543C6D696E5F7487
:102A7000726176656C5F66656564726174653E005F
:102A800020540020520020204D323034205000418C
:102A90006363656C65726174696F6E2028756E6919
:102AA00074732F7332293A20503C7072696E745FD0
:102AB000616363656C3E20523C726574726163743D
:102AC0005F616363656C3E20543C74726176656C33
:102AD0005F616363656C3E0A00204500205A002058
:102AE000590020204D3230312058004D6178696DF9
:102AF000756D20416363656C65726174696F6E20EA
:102B000028756E6974732F7332293A0A00204500C4
:102B1000205A0020590020204D3230332058004DDB
:102B20006178696D756D2066656564726174657341
:102B30002028756E6974732F73293A0A00204500A6
:102B4000205A0020590020204D393220580053745B
:102B50006570732070657220756E69743A0A002082
:102B6000204D3230302044300A0020204D323030A9
:102B70002044002044697361626C65640A00466900
:102B80006C616D656E742073657474696E67733AF9
:102B9000002020473231202020203B005265736501
:102BA0006E643A20006F6B0020746F6F206C6F6E44
:102BB0006720657874727573696F6E2070726576C0
:102BC000656E7465640A0020636F6C6420657874B8
:102BD000727573696F6E2070726576656E74656468
:102BE0000A004572726F722077726974696E67208D
:102BF000746F20454550524F4D210A005772697439
:102C0000696E6720746F2066696C653A20006F708A
:102C1000656E206661696C65642C2046696C653A56
:102C200020006F70656E206661696C65642C2046BB
:102C3000696C653A200046696C652073656C656354
:102C40007465640A002053697A653A200046696C0D
:102C500065206F70656E65643A20002066696C655A
:102C60003A2000646F696E67006672657368004E93
:102C70006F772000454E4420535542524F555449DA
:102C80004E450A002220706F730022207061726529
:102C90006E743A2200535542524F5554494E4520C6
:102CA00043414C4C207461726765743A22004B4971
:102CB0004C4C45442E2000747279696E6720746F05
:102CC0002063616C6C207375622D67636F6465208F
:102CD00066696C6573207769746820746F6F206D06
:102CE000616E79206C6576656C732E204D4158209D
:102CF0006C6576656C2069733A00CBE2ACE4112414
:102D00001FBECFEFD1E2DEBFCDBF00E00CBF14E0AD
:102D1000A0E0B2E0EEE1F3EE01E00BBF02C00790ED
:102D20000D92A831B107D9F728E1A8E1B4E001C0BC
:102D30001D92AE3FB207E1F716E1CEE7D6E100E023
:102D400006C021970109802FFE010E94E7F0CD37D0
:102D5000D10780E00807A9F70E9418DD0C947EF1E6
:102D60000C9400002F923F924F925F926F927F924D
:102D70008F929F92AF92BF92CF92DF92EF92FF928B
:102D80000F931F93CF93DF93CDB7DEB7CA58D10906
:102D90000FB6F894DEBF0FBECDBF21E020935A10CE
:102DA00080914B188D3411F40C94B021843511F4BA
:102DB0000C94702E873411F00C94BC2E809149181D
:102DC00090914A188A31910509F4BEC79CF4843069
:102DD00091053CF482309105B4F597FF2DC00C9419
:102DE000AC218430910509F4D2C1059709F40EC2D3
:102DF0000C94AC218A32910511F40C94A3204CF46C
:102E00008C31910509F4A4C74D9709F4A6C70C9419
:102E1000AC218B35910511F40C942E218C35910544
:102E200011F40C9432218A35910511F00C94AC21E7
:102E300010922B040C94BE2E8091270281110C94C9
:102E4000C32E0C94BE2E20912702222311F40C9441
:102E5000BE2E11E0029709F010E00E94FA9019824C
:102E60001A821B821C821D821E821F82188682E5A6
:102E70000E94554C882309F43AC10E94D54B4B015E
:102E80005C0120E030E0A9010E946EE9882309F48A
:102E900044C1C0903604D0903704E0903804F090DC
:102EA0003904CCAADDAAEEAAFFAAC0903A04D090B9
:102EB0003B04E0903C04F0903D04C8AED9AEEAAECD
:102EC000FBAEC0900D18D0900E18E0900F18F09047
:102ED0001018CCAEDDAEEEAEFFAEC0901118D090A3
:102EE0001218E0901318F09014182496CCAEDDAEB2
:102EF000EEAEFFAE24972CAD3DAD4EAD5FAD6CA9EF
:102F00007DA98EA99FA90E946EE981110BC0A7011E
:102F1000960168AD79AD8AAD9BAD0E946EE98823BC
:102F200009F4FBC020E030E0A901C501B4010E9412
:102F30006EE9881F8827881F181739F0C12CD12CFB
:102F400080E8E82E8FEBF82E06C0C12CD12C00E8CB
:102F5000E02E0FE3F02E2C96CCAEDDAEEEAEFFAE43
:102F60002C972CA93DA94EA95FA96CAD7DAD8EAD66
:102F70009FAD0E94EAED28966CAF7DAF8EAF9FAFFC
:102F8000289728AD39AD4AAD5BAD24966CAD7DADCB
:102F90008EAD9FAD24970E94EAED6B017C012896CF
:102FA0002CAD3DAD4EAD5FAD2897CA01B9010E9471
:102FB000D3E92B013C01A7019601C701B6010E948C
:102FC000D3E99B01AC01C301B2010E94EBED0E9469
:102FD00056F02B013C0120E030E040E05FE30E942E
:102FE000D3E960966CAF7DAF8EAF9FAF6097A501C0
:102FF0009401C501B4010E94D3E94B015C016096C4
:103000002CAD3DAD4EAD5FAD6097CA01B9010E94D8
:10301000D3E99B01AC01C501B4010E94EAED0E9415
:1030200056F02C962CAD3DAD4EAD5FAD2C970E9469
:10303000D3E94B015C01C701B6019058A30192018D
:103040000E94C7EEA50194010E94D3E96B017C01A7
:103050002CAD3DAD4EAD5FAD6CA97DA98EA99FA9EC
:103060000E94EBED20E030E040E05FE30E94D3E916
:103070009B01AC01C701B6010E94EBED2CA93DA953
:103080004EA95FA90E94EAED69837A838B839C83B2
:1030900024962CAD3DAD4EAD5FAD249768AD79ADB6
:1030A0008AAD9BAD0E94EBED20E030E040E05FE3B5
:1030B0000E94D3E96B017C01A301920128966CADBB
:1030C0007DAD8EAD9FAD28970E94C7EEA5019401FE
:1030D0000E94D3E99B01AC01C701B6010E94EBED50
:1030E00028AD39AD4AAD5BAD0E94EAED12C089E46E
:1030F0000E94554C882331F00E94D54B69837A8316
:103100008B839C838AE40E94554C882331F00E9473
:10311000D54B6D837E838F83988720E030E0A901B3
:1031200069817A818B819C810E946EE981110EC038
:1031300020E030E0A9016D817E818F8198850E9419
:103140006EE9811103C0EEE1FAE10DC0412FBE012D
:103150006F5F7F4F8DE098E10E94B0AE0C94BE2E61
:103160000E94188AF80184918F010F5F1F4F81110F
:10317000F7CFEDE1F2E084918F010F5F1F4F8823BD
:1031800011F40C94BE2E0E94188AF801F4CF80E549
:103190000E94554C882379F0809125049091260453
:1031A000009749F04AE050E060E070E00E94EDE7EF
:1031B0006B017C0103C0C12CD12C760183E50E94F8
:1031C000554C882361F00E94D54B20E030E04AE75F
:1031D00054E40E94D3E90E9434EF6B017C010E9409
:1031E000A9690E949058C60ED71EE81EF91E0E94BB
:1031F0009058DC01CB018C199D09AE09BF09B7FDC0
:1032000002C00C94BE2E0E945BAAF1CF80912702CF
:10321000882311F40C94BE2E0E94FA9089E40E9437
:10322000554C882329F00E94D54B2B013C0103C04B
:10323000412C512C32018AE40E94554C882329F0FC
:103240000E94D54B4B015C0103C0812C912C540191
:1032500080E50E94554C882329F00E94D54B6B01D4
:103260007C0103C0C12CD12C760181E50E94554C14
:10327000882339F00E94D54B6CAB7DAB8EAB9FABF6
:1032800004C01CAA1DAA1EAA1FAA20915910C65725
:10329000DF4F2883CA58D040609102027091030228
:1032A000072E000C880B990B0E9474E920914202B2
:1032B0003091430240914402509145020E94D3E96B
:1032C0002AE037ED43E25CE30E94D3E968AB79ABD7
:1032D0008AAB9BAB4091360450913704609138041F
:1032E0007091390448AF59AF6AAF7BAF9A01AB0117
:1032F000C301B2010E94EBEDA1966CAF7DAF8EAF22
:103300009FAFA19740903A0450903B0460903C04DA
:1033100070903D04A3019201C501B4010E94EBED40
:10332000A5966CAF7DAF8EAF9FAFA59720910D187E
:1033300030910E1840910F1850911018C701B60126
:103340000E94EBEDA9966CAF7DAF8EAF9FAFA997B2
:10335000209111183091121840911318509114189F
:103360006CA97DA98EA99FA90E94EBEDAD966CAFCB
:103370007DAF8EAF9FAFAD97C8ACD9ACEAACFBAC1C
:10338000C982DA82EB82FC824D825E826F8278860D
:103390000E9490589B01AC0128533F4F4F4F5F4F05
:1033A000C358DF4F288339834A835B83CD57D0408E
:1033B000BDEC8B2EBCEC9B2EA92CBDE3BB2E259621
:1033C0001FAE259729961FAE29972D961FAE2D97D4
:1033D00061961FAE61970E9437810E9490588B01C1
:1033E0009C01C358DF4FC880D980EA80FB80CD574D
:1033F000D0400C191D092E093F0937FD10C09B0153
:10340000AC0128533F4F4F4F5F4FC358DF4F2883C6
:1034100039834A835B83CD57D0400E945BAAA501C4
:1034200094012596BFAD25972996AFAD29972D9686
:10343000FFAD2D976196EFAD61976B2F7A2F8F2F90
:103440009E2F0E94EBED6CAB78AF8CAF21969FAFB7
:10345000219720E030E040E85FE30E9411F0181669
:1034600044F41CAA18AE30E83CAF4FE321964FAFAE
:10347000219760910D1870910E1880910F189091FE
:103480001018E1966CAF7DAF8EAF9FAFE197809142
:10349000360490913704A0913804B0913904E59630
:1034A0008CAF9DAFAEAFBFAFE59721969FAD219793
:1034B0009F93ACADAF93B8ADBF93ECA9EF93E196FA
:1034C000ACACBDACCEACDFACE197A996ECACFDAC3E
:1034D0000EAD1FADA997A1962CAD3DAD4EAD5FAD24
:1034E000A197E5966CAD7DAD8EAD9FADE5970E9441
:1034F000EAB40F900F900F900F9062966FAF6297A3
:1035000063967FAF639764968FAF649765969FAF1E
:103510006597C0901118D0901218E0901318F09091
:103520001418E996CCAEDDAEEEAEFFAEE997209171
:103530003A0430913B0440913C0450913D04ED9697
:103540002CAF3DAF4EAF5FAFED9721963FAD2197CA
:103550003F934CAD4F9358AD5F936CA96F93E99631
:10356000ACACBDACCEACDFACE997AD96ECACFDAC91
:103570000EAD1FADAD97A5962CAD3DAD4EAD5FAD7B
:10358000A597ED966CAD7DAD8EAD9FADED970E948C
:10359000EAB40F900F900F900F9066966FAF6697FA
:1035A00067967FAF679768968FAF689769969FAF6A
:1035B000699789819A81AB81BC81CF57DF4F88831E
:1035C0009983AA83BB83C158D040CD80DE80EF8031
:1035D000F884CB57DF4FC882D982EA82FB82C55874
:1035E000D0406A961FAE6A9725967FAD259729969B
:1035F0006FAD29972D969FAD2D9761968FAD6197F1
:10360000272F362F492F582FBCA9A8ADFCAD2196E6
:10361000EFAD21976B2F7A2F8F2F9E2F0E94EAED0F
:103620002FE632E143E05BE30E946EE987FD29C1AA
:1036300025967FAD259729966FAD29972D969FAD3D
:103640002D9761968FAD6197272F362F492F582FD1
:10365000BCA9A8ADFCAD2196EFAD21976B2F7A2FB9
:103660008F2F9E2F0E94EBED20E030E040E05FE3E3
:103670000E94D3E9662E972E882E792E9F938F93E2
:103680007F936F93E196ACACBDACCEACDFACE19771
:10369000A996ECACFDAC0EAD1FADA997A1962CADD3
:1036A0003DAD4EAD5FADA197E5966CAD7DAD8EADF8
:1036B0009FADE5970E94EAB40F900F900F900F9086
:1036C0006B966FAF6B976C967FAF6C976D968FAF65
:1036D0006D97C757DF4F9883C958D0407F928F921C
:1036E0009F926F92E996ACACBDACCEACDFACE997E3
:1036F000AD96ECACFDAC0EAD1FADAD97A5962CAD67
:103700003DAD4EAD5FADA597ED966CAD7DAD8EAD8B
:103710009FADED970E94EAB40F900F900F900F901D
:10372000162F072FB82EA92E66962FAD669767968F
:103730003FAD679768964FAD689769965FAD69979B
:10374000CB57DF4F688179818A819B81C558D040F2
:103750000E94EBED20E030E040E05FE30E94D3E91F
:103760001B012C0162962FAD629763963FAD639764
:1037700064964FAD649765965FAD6597CF57DF4F01
:10378000688179818A819B81C158D0400E94EBED8C
:1037900020E030E040E05FE30E94D3E99B01AC0110
:1037A0006B966FAD6B976C967FAD6C976D968FAD8A
:1037B0006D97C757DF4F9881C958D0400E94EAEDF6
:1037C0006B017C0120E030E0A9010E9411F087FF2D
:1037D00004C0F7FAF094F7F8F094A2019101612F78
:1037E000702F8B2D9A2D0E94EAED1B012C0120E0F9
:1037F00030E0A9010E9411F087FF04C057FA5094ED
:1038000057F85094A2019101C701B6010E94EBED57
:103810002DEC3CEC4CEC5DE30E946EE918168CF547
:1038200066961FAF669767960FAF67976896BFAEAD
:1038300068976996AFAE69976B96DFAC6B976296A7
:10384000DFAE62976C96EFAC6C976396EFAE6397C2
:103850006D96FFAC6D976496FFAE6497C757DF4FC8
:103860002881C958D04065962FAF65976CAA98AE4D
:103870008CAE21967FAE219731E06A963FAF6A9772
:10388000B3CE6A964FAD6A97411144C125967FAD7C
:10389000259729966FAD29972D969FAD2D97619607
:1038A0008FAD6197272F362F492F582FBCA9A8AD70
:1038B000FCAD2196EFAD21976B2F7A2F8F2F9E2F86
:1038C0000E94EAED6B017C012DEC3CEC4CEC5DE3DD
:1038D0000E9411F018160CF41DC1A7019601C70132
:1038E000B6010E94EBED2596EFAD25972996BFAD69
:1038F00029972D96AFAD2D976196FFAD61972E2F2D
:103900003B2F4A2F5F2F0E94EBED662E972E882EBD
:10391000792E20E030E040E85FE30E9411F087FF5D
:10392000F9C07F928F929F926F92E196ACACBDAC42
:10393000CEACDFACE197A996ECACFDAC0EAD1FAD03
:10394000A997A1962CAD3DAD4EAD5FADA197E59683
:103950006CAD7DAD8EAD9FADE5970E94EAB40F9042
:103960000F900F900F906A966FAF6A976B967FAF2C
:103970006B976C968FAF6C976D969FAF6D977F929C
:103980008F929F926F92E996ACACBDACCEACDFAC9F
:10399000E997AD96ECACFDAC0EAD1FADAD97A5961D
:1039A0002CAD3DAD4EAD5FADA597ED966CAD7DAD4B
:1039B0008EAD9FADED970E94EAB40F900F900F90DF
:1039C0000F90162F072FB82EA92E262F372F482FEE
:1039D000592FCB57DF4F688179818A819B81C558E8
:1039E000D0400E94EBED20E030E040E05FE30E9439
:1039F000D3E96B017C016A962FAD6A976B963FAD58
:103A00006B976C964FAD6C976D965FAD6D97CF577A
:103A1000DF4F688179818A819B81C158D0400E94A3
:103A2000EBED20E030E040E05FE30E94D3E99B0152
:103A3000AC0162966FAD629763967FAD63976496B3
:103A40008FAD649765969FAD65970E94EAED1B0167
:103A50002C0120E030E0A9010E9411F087FF04C092
:103A600057FA509457F85094A701960166966FAD97
:103A7000669767967FAD679768968FAD68976996EA
:103A80009FAD69970E94EAED6B017C0120E030E078
:103A9000A9010E9411F087FF04C0F7FAF094F7F82B
:103AA000F094A2019101C701B6010E94EBED2DEC4B
:103AB0003CEC4CEC5DE30E9411F018165CF166964C
:103AC0001FAF669767960FAF67976896BFAE689708
:103AD0006996AFAE69976A965FAD6A9762965FAF77
:103AE00062976B966FAD6B9763966FAF63976C96AB
:103AF0007FAD6C9764967FAF64976D968FAD6D9731
:103B000065968FAF65976CAA98AE8CAE21967FAE06
:103B10002197BCCE25967FAD259729966FAD299725
:103B20002D969FAD2D9761968FAD6197272F362FDC
:103B3000492F582FBCA9A8ADFCAD2196EFAD219718
:103B40006B2F7A2F8F2F9E2F0E94EAED4B015C0185
:103B500062968FAD629763969FAD63976496AFADA3
:103B600064976596BFAD659789839A83AB83BC8361
:103B700066968FAD669767969FAD67976896AFAD6F
:103B800068976996BFAD69978D839E83AF83B88729
:103B90007CA968AD9CAD21968FAD2197272F362F3C
:103BA000492F582F60E070E080E89FE30E94EAED23
:103BB0006B017C0120913E0430913F044091400410
:103BC000509141040E94D3E92B013C01209115182A
:103BD000309116184091171850911818BCA9A8AD2B
:103BE000FCAD2196EFAD21976B2F7A2F8F2F9E2F53
:103BF0000E94D3E99B01AC01C301B2010E94EBED2D
:103C000069877A878B879C8720914204309143048F
:103C10004091440450914504C701B6010E94D3E984
:103C20006B017C012091191830911A1840911B18D2
:103C300050911C18BCA9A8ADFCAD2196EFAD219701
:103C40006B2F7A2F8F2F9E2F0E94D3E99B01AC01FF
:103C5000C701B6010E94EBED6D877E878F87988B39
:103C6000CE0101960E94DCCC1CA61DA61EA61FA696
:103C700089819A81AB81BC8188A399A3AAA3BBA3A4
:103C80008D819E81AF81B8858CA39DA3AEA3BFA378
:103C900089859A85AB85BC8588A799A7AAA7BBA764
:103CA000AE01485D5F4FBE016C5D7F4FCE018096D7
:103CB0000E9485BEDE019C966D01C657DF4FE880ED
:103CC000CA58D0408E01005D1F4F9E01235F3F4FB9
:103CD000AE01485D5F4FBE016C5D7F4FCE018096A7
:103CE0000E948559882329F120E030E040E85FE315
:103CF000BCA9A8ADFCAD2196EFAD21976B2F7A2F13
:103D00008F2F9E2F0E946EE987FF13C03CA9259636
:103D10003FAF259748AD29964FAF29975CAD2D96BB
:103D20005FAF2D9721966FAD219761966FAF619729
:103D300052CB80E1EDE0F8E1A6E3B4E001900D9212
:103D40008A95E1F70C94BE2E0E94F24D0C94BE2E83
:103D500080E00E94C6920C94BE2E83E50E94554CD2
:103D6000882321F10E94B54B182F863070F0E5EEC4
:103D7000F2E084918F010F5F1F4F882311F40C94A0
:103D8000BE2E0E94188AF801F4CF833009F44AC18C
:103D900030F4813091F1823009F43FC008C08430A2
:103DA00009F49FC1853009F4ACC101C010E00E9444
:103DB0007992811103C0E5ECF2E013C08091DB172A
:103DC000882319F063E173E002C067E173E08DEBD3
:103DD00092E00E9408B48AE00E94188A0E94BFBE46
:103DE00096C184917F01BFEFEB1AFB0A882309F487
:103DF0008EC10E94188AF701F4CF0E9472BF109200
:103E000001021092000282EB92E090932C078093C3
:103E10002B070E94448A0C94BE2E80910002909140
:103E2000010297FF0EC0E9E8F2E084918F010F5F75
:103E30001F4F882311F40C94BE2E0E94188AF8019B
:103E4000F4CF0097A1F48091520280932C04198240
:103E50001A821B821C8218A219A21AA21BA2BE01DE
:103E60006F5F7F4FCE0180960E94F9C327C08150BB
:103E700065E00E94B3F080FF03C024E0291B922F6D
:103E800025E09202F0011124E80FF11D87FDFA955B
:103E9000EE0FFF1FEE0FFF1FE25AF84E80913E0417
:103EA00090913F04A0914004B0914104808391839C
:103EB000A283B38380912C048093520280910002EC
:103EC00090910102893191050CF067C01092520265
:103ED0009C012F5F3F4F309301022093000265E069
:103EE0000E94B3F080FF03C024E0291B922F409171
:103EF0003E0450913F04609140047091410448A3F6
:103F000059A36AA37BA319821A821B821C8244E0F4
:103F1000840290011124B9016F58764F4B01DB01E7
:103F20002D913D914D915C91B4E09B02C001112413
:103F3000FC01EB57F64F5F016081718182819381B3
:103F4000DE0111966D01E12CF12C00EA10E40E94D3
:103F500029C319821A821B821C82B601CE01809667
:103F60000E94F9C3F50180819181A281B381809380
:103F7000360490933704A0933804B0933904F401C5
:103F800080819181A281B38180933A0490933B0414
:103F9000A0933C04B0933D04BCC080E090E0A0EA54
:103FA000B0E480933E0490933F04A0934004B09308
:103FB00041040E94BA930E94A9698FEF9FEF9093EA
:103FC000010280930002E5E7F2E084918F010F5F28
:103FD0001F4F882321F00E94188AF801F6CF83E949
:103FE00092E09A83898304E610E019A308A3BE0136
:103FF0006F5F7F4FCE0180960E9414C58AEB92E0DE
:104000009A83898319A308A3BE016F5F7F4FCE01F6
:1040100080960E9414C581E00E94C69281E00E94B1
:10402000A69277C088E50E94554C8823A1F00E9493
:10403000A54B1FEF160F1530A8F0EEE5F2E08491C6
:104040008F010F5F1F4F882311F40C94BE2E0E9426
:10405000188AF801F4CF88E50E94188A0E949CE42F
:104060000C94BE2E89E50E94554C8823A1F00E9435
:10407000A54B0FEF060F0530A8F0E7E4F2E08491BE
:104080008F010F5F1F4F882311F40C94BE2E0E94E6
:10409000188AF801F4CF89E50E94188A0E949CE4EE
:1040A0000C94BE2E8AE50E94554C882399F00E94FC
:1040B000D54B25E0129FF0011124E00FF11DEE0F0A
:1040C000FF1FEE0FFF1FE25AF84E60837183828359
:1040D000938335C08AE50E94188A0E949CE40C9460
:1040E000BE2E8AE50E94554C8823A1F30E94D54B31
:1040F00060935A1770935B1780935C1790935D17CA
:104100001EC080E00E94A6920E9472BF18C01230AA
:10411000B1F460910002709101026931710514F0EF
:1041200069E170E088E392E00E94EFB369E170E03A
:1041300083E392E00E94EFB38AE00E94188A0E9413
:10414000A49E0C94BE2E80912702882311F40C9417
:10415000BE2E89E40E94554CE82E882321F00E944F
:10416000A54B062F01C000E08AE40E94554CF82EB2
:10417000882321F00E94A54B162F01C010E0EE20ED
:1041800011F0053020F4FF2081F0153070F0ECEFD5
:10419000F2E084918F010F5F1F4F882311F40C947C
:1041A000BE2E0E94188AF801F4CF0E94614CEE20C6
:1041B00091F034E00302F0011124EB57F64F8081B7
:1041C0009181A281B38180930D1890930E18A093D2
:1041D0000F18B0931018FF2091F044E01402F00182
:1041E0001124EF58F64F80819181A281B381809391
:1041F000111890931218A0931318B093141880E517
:104200000E94554C882319F00E94C64B03C080E5DC
:104210000E940C4C86E40E94554C8823D9F00E94E1
:10422000D54B6B017C0120E030E0A9010E9411F028
:10423000181684F420E030E040E752E4C701B601EC
:104240000E94C7EE6093420270934302809344023F
:10425000909345020E9473CD0C94BE2E20932B04A4
:104260000C94BE2E87E5282E82E0382E98E6E92EA3
:1042700090E1F92E66E374E07DAB6CAB28E1C22ED1
:1042800024E0D22E00E010E0D1018D911D010E94AA
:10429000554C882309F44BC00E94D54B2B013C019F
:1042A000133049F0F60120813181428153810E940F
:1042B000EAED2B013C01ACA9BDA92D913D914D9199
:1042C0005C91C301B2010E94EAED4B015C012DEB50
:1042D00037E346E855EB0E9411F087FD0AC02DEB4D
:1042E00037E346E855E3C501B4010E946EE91816AC
:1042F000F4F4133051F4409242045092430460921B
:1043000044047092450401E012C0A5019401F70134
:1043100060817181828193810E94EBEDD7016D9361
:104320007D938D939C931397812F0E9411941F5F0F
:10433000B4E0EB0EF11CECA9FDA93496FDABECAB9F
:10434000F4E0CF0ED11C143009F09ECF002309F405
:10435000F6CE0E94C5C2F3CE0E9448C50C94BE2E74
:104360008091491890914A188537910511F40C9461
:10437000BE2E0CF0DAC08D34910509F4D3C30CF0D5
:1043800072C08B31910509F452C2ACF586319105AA
:1043900009F401C20CF58231910509F440C584F499
:1043A000419711F00C946D2E5F988A9847988091F0
:1043B0000801817080930601479812980C94BE2ED4
:1043C0008431910509F4A7C1459711F00C946D2E25
:1043D0000E94196B0C94BE2E8831910509F4F7C127
:1043E0000CF4DFC18931910509F4FCC14A9709F445
:1043F00010C20C946D2E8032910509F4BEC2FCF4FB
:104400008D31910511F40C94BE2E0CF4A8C28E319E
:10441000910509F4AEC24F9711F00C946D2E0E94D5
:10442000878468A379A38AA39BA3BE016F5F7F4F94
:10443000CE0180960E943689E3E3FAE1EAC2813335
:10444000910509F431C32CF48A9709F4F8C20C944D
:104450006D2E8B34910509F44CC38C34910509F40D
:104460004CC30C946D2E8A36910509F487C4B4F5BB
:104470008435910509F4D3C4E4F48135910509F438
:10448000A9C44CF48E34910511F00C946D2E0E9449
:10449000FD8F0C94BE2E8235910509F4BDC4833581
:1044A000910511F00C946D2E81E080932A040C94F8
:1044B000BE2E8C35910509F4FAC434F48535910586
:1044C00009F4DCC40C946D2E8836910509F42EC3D2
:1044D0008936910509F4F2C30C946D2E8F3691053F
:1044E00009F460C384F48C36910509F4AEC30CF46E
:1044F00061C48D36910509F423C48E36910509F403
:104500003EC30C946D2E8137910509F4AAC30CF4B7
:10451000A0C38237910509F452C58337910511F084
:104520000C946D2EE7EAF4E087C58E3221E0920705
:1045300011F40C94A92C0CF071C08B3C910509F47A
:1045400095C6CCF58C38910509F4FEC3ACF48737D9
:10455000910509F419C60CF4CAC58837910509F408
:1045600016C68937910511F00C946D2E10924C05EA
:1045700010924B050C94BE2E8E3B910509F4FAC3A4
:1045800034F48B39910509F4B4C30C946D2E883C36
:10459000910509F402C6893C910511F00C946D2E29
:1045A000F7E5EF2EF2E0FF2E02EB10E1A2ECCA2EAF
:1045B000A0E1DA2E42C68C3D910511F40C943C2BFF
:1045C0009CF48D3C910509F4E2C60CF46BC68E3C5C
:1045D000910509F469C7833D910511F00C946D2E86
:1045E0000E948F9D0C94BE2E823E910511F40C9476
:1045F000B72B3CF48D3D910511F40C94492B0C9490
:104600006D2E8C3241E0940711F40C94E02B8D3226
:10461000914011F40C94092C0C946D2E853F61E0AF
:10462000960711F40C94962DDCF58A39A1E09A07CF
:1046300009F413C3BCF48033E1E09E0711F40C9439
:10464000002D14F40C94FD2C833621E0920709F41C
:104650005EC08039914011F00C946D2E0E94A969C2
:104660000C94BE2E853A41E0940711F40C94932DDE
:104670004CF4843A914011F00C946D2E0E946E9F80
:104680000C94BE2E8C3A71E0970709F430C7843F32
:10469000914011F00C946D2E0E943E760C94BE2E2B
:1046A0008A39B2E09B0711F40C94D52DB4F4873FFE
:1046B000F1E09F0711F40C949C2D14F40C94992DA7
:1046C000883F31E0930711F40C94A82D8C30924070
:1046D00011F40C94CC2D0C946D2E8B3853E095076F
:1046E00011F40C94BE2E3CF48438934011F40C94D5
:1046F000022E0C946D2E803AA3E09A0709F47CC137
:10470000873E934011F40C945A2E0C946D2EEEE1DA
:10471000FAE10C94802DEAE2F3E084918F010F5FBF
:104720001F4F882321F00E94188AF801F6CF1092BB
:10473000370C8AEE99E00E9495A38BE1EAEEF9E04E
:10474000DE01159601900D928A95E1F78091E809B6
:104750009091E9099C838B8385E692E09A83898313
:1047600040E050E0BE016F5F7F4F80E090E00E942C
:104770004A6DCE0101960E94F1A9EBE1F3E084912C
:104780008F010F5F1F4F882311F40C94BE2E0E94DF
:10479000188AF801F4CF1092B9091092BA090C9452
:1047A000BE2EE0914718F09148188081882329F0A7
:1047B000803209F410823196F8CF40E061E08091B8
:1047C0004718909148180E94A3D80C94BE2E80914F
:1047D000BA09882319F081E08093B9090E9423B4B3
:1047E0000C94BE2E1092B9098091630F813011F0A4
:1047F0000C94BE2E82E08093630F0E9490586093C9
:104800005F0F7093600F8093610F9093620F0C9411
:10481000BE2E8091BA09882311F40C94BE2E83E534
:104820000E94554C81110C94C82E0C94BE2E83E42A
:104830000E940C4C882309F450C0E8E6F3E0849110
:104840008F010F5F1F4F882321F00E94188AF80103
:10485000F6CF8091850B811103C0EBE3F3E012C02A
:10486000BE016F5F7F4F82E89BE00E945DA28E01D8
:104870000F5F1F4FF80181918F01882349F10E943A
:10488000188AF8CF84918F010F5F1F4F882301F1A1
:104890000E94188AF801F6CF0AE9C02E03E0D02E54
:1048A000E12CF12C20E08091250790E00E2C02C035
:1048B000959587950A94E2F780FDA4C1FFEFEF1A62
:1048C000FF0A32E0C30ED11C45E0E416F10459F7AB
:1048D0008AE00E94188A0C94BE2E8091BA0988231F
:1048E00039F08091B909882319F0E5E4F3E003C0B9
:1048F000E7E5F3E028C084918F010F5F1F4F882305
:1049000021F00E94188AF801F6CF6091330C709163
:10491000340C8091350C9091360C4AE00E943B8D0E
:104920008FE20E94188A60912F0C7091300C809158
:10493000310C9091320C4AE00E943B8D8AE00E943B
:10494000188A0C94BE2E84918F010F5F1F4F88230D
:1049500011F40C94BE2E0E94188AF801F4CF40E0A6
:1049600060E080914718909148180E94A3D80C9459
:10497000BE2E0E948C960C94BE2E8091B909811196
:104980000E94A9698091BA09882311F40C94BE2E63
:1049900080E50E94554C882319F00E94C64B03C045
:1049A00080E50E940C4C182F482F61E08091471839
:1049B000909148180E94A3D883E50E94554C882303
:1049C00081F00E94A54BAB01BC014093330C509386
:1049D000340C6093350C7093360C82E89BE00E9497
:1049E0004EA18091BA09882319F081E08093B9091A
:1049F00011110C94BE2EF2CE809147189091481858
:104A000021E02093B80940E060E00E94A3D80C9414
:104A1000BE2E84918F010F5F1F4F882321F00E94CB
:104A2000188AF801F6CFBE016F5F7F4F87E793E0EA
:104A30000E9408B48AE00E94188A0C94BE2E83E576
:104A40000E94554C882311F40C94BE2E0E94B54B45
:104A5000E82E80E50E94554C882339F00E94B54B22
:104A6000182F87FF03C00C94BE2E1DE089E40E941E
:104A7000554C882351F00E94C64B81110C94412F54
:104A8000EFEDF5E08FE096E00AC089E40E940C4C5F
:104A9000F4CF31968E179F0711F40C94412F249177
:104AA0001213F7CF0C94162FF090240481E0F8260F
:104AB000F0922404EFE8F3E084918F010F5F1F4F21
:104AC000882321F00E94188AF801F6CFFF2019F000
:104AD000E4E8F3E002C0E9E8F3E084918F010F5FBE
:104AE0001F4F882311F40C94BE2E0E94188AF801DF
:104AF000F4CF0E9423B40C94BE2E8091630F8130BA
:104B000011F00C94BE2E82E08093630F0E949058A7
:104B100060935F0F7093600F8093610F9093620FAB
:104B20000C94BE2E0E946AB40C94BE2E88E690E0CF
:104B30000E94519481110C94BE2E8091250783FF11
:104B400002C00C94BE2E83E50E94554C882399F038
:104B50000E94D54B0E942FEFCB010E94B77B0E9491
:104B6000D54B20E030E04AEA52E40E946EE9181684
:104B700014F00E946AB40E94F8B60C94BE2E8EE423
:104B80000E94554C882311F40C94BE2E0E94A54B14
:104B90006093F4187093F5188093F6189093F718B3
:104BA0000C94BE2E83E50E940C4C882359F083E5BB
:104BB0000E94554C882319F00E94B54B01C080E03B
:104BC00080932507E3E3FAE184918F010F5F1F4F84
:104BD000811103C0E8EAF3E004C00E94188AF801DA
:104BE000F3CF84918F010F5F1F4F882321F00E9424
:104BF000188AF801F6CF8091250781114DCEE4EA9D
:104C0000F3E018C0BB24B394B20E222319F08CE257
:104C10000E94188AF60185919491FC0184918F017C
:104C20000F5F1F4F882321F00E94188AF801F6CFEA
:104C30002B2D44CE84918F010F5F1F4F882309F4E1
:104C400047CE0E94188AF801F5CF109220020C94EA
:104C5000BE2E8FEA93E00E9414AA0E941D980C9425
:104C6000BE2E83E50E94554C811103C0E3E3FAE1B7
:104C70000DC00E94B54B8D3320F480932B020C9411
:104C8000BE2E8CE380932B020C94BE2E84918F0158
:104C90000F5F1F4F882321F00E94188AF801F6CF7A
:104CA00040912B0250E060E070E088EB93E00E94BE
:104CB000B5B38AE00E94188A0C94BE2E89E690E073
:104CC0000E945194811111C0EFEBF3E084918F01A8
:104CD0000F5F1F4F882321F00E94188AF801F6CF3A
:104CE0000E94517C8AE00E94188A10925A100C94FB
:104CF000562F83E50E94554C882311F40C94BE2E48
:104D00000E94B54B182F8D3308F01CE310936710E9
:104D10000E9490586B017C01212F30E0A8EEB3E097
:104D20000E94DBEDC60ED71EE81EF91EC09263106E
:104D3000D0926410E0926510F09266100C94BE2E32
:104D40000E9490940C94BE2E8091250783FF02C090
:104D50000C94BE2E83E50E94554C882311F40C94CC
:104D6000BE2E0E94D54B0E942FEFCB010E94E44D36
:104D70000C94BE2E0E94318E0C94BE2E80E50E94B3
:104D8000554C811106C083E50E94554C882359F08B
:104D900005C00E94B54B8111F1C7F5CF0E94A54B0C
:104DA0006F3F710510F06FEF70E0709347046093F0
:104DB0004604E4C780E50E94554C811105C010925D
:104DC000470410924604DAC70E94A54B672B09F0EE
:104DD000D5C7F5CF0E94577D0E9469B9109247044C
:104DE0001092460400E010E062E370E080E090E0A2
:104DF0000E94BEC60E9437810F5F1F4F033111050D
:104E000099F762E370E080E090E00E94BEC60E94E5
:104E100037810E94702FB2C710922A04AFC783E572
:104E20000E94554C882399F00E94D54B20E030E039
:104E30004AE754E40E94D3E90E9434EF60932C02C5
:104E400070932D0280932E0290932F0297C788E5CE
:104E50000E940C4C8111ADC789E50E940C4C811158
:104E6000A8C78AE50E940C4C8111A3C785E40E9463
:104E70000C4C81119EC70E9469B980C783E50E94CE
:104E80000C4C882309F47AC70E94D54B20E030E00F
:104E90004AE754E40E94D3E90E9434EF60935F1024
:104EA00070936010809361109093621067C7B7E5AC
:104EB000CB2EB2E0DB2E11EFE12E17E1F12E10E048
:104EC000D6018D916D010E940C4C882309F46DC0B0
:104ED000133009F063C00E94D54B4B015C0120E008
:104EE00030E040EA51E40E946EE987FF4EC0A50120
:104EF00094016091FD177091FE178091FF179091BA
:104F000000180E94C7EE2B013C019B01AC0160918F
:104F1000F4067091F5068091F6069091F7060E94CE
:104F2000D3E96093F4067093F5068093F6069093A8
:104F3000F706A30192016091140770911507809103
:104F40001607909117070E94D3E960931407709396
:104F5000150780931607909317076091AE10709114
:104F6000AF108091B0109091B1100E9472E9A3012E
:104F700092010E94D3E90E9434EF6093AE107093C7
:104F8000AF108093B0109093B1108092FD17909263
:104F9000FE17A092FF17B092001807C00E94D54BD1
:104FA000F70160837183828393831F5FF4E0EF0EC8
:104FB000F11C143009F084CF0E9499B8DFC60E941A
:104FC000A96983E50E94554C882309F4B8C80E945A
:104FD000A54B6230710509F0B2C80E94C0CC8BE5C8
:104FE0000E94188A6091DA187091DB188091DC18A1
:104FF0009091DD1842E00E94C08D4091DE185091E2
:10500000DF186091E0187091E11885EC93E00E9440
:10501000D2B34091E2185091E3186091E418709176
:10502000E51882EC93E00E94D2B38DE50E94188AC5
:105030008AE00E94188AA2C684918F010F5F1F4FD9
:10504000882321F00E94188AF801F6CF60E087E9F2
:1050500094E00E946D9E61E080E994E00E946D9E64
:1050600061E085E894E00E946D9E61E085E794E050
:105070000E946D9E60E08CE694E00E946D9E61E06F
:1050800082E694E00E946D9E60E088E594E00E94D4
:105090006D9E60E080E594E00E946D9E61E082E498
:1050A00094E00E946D9E60E084E394E00E946D9E17
:1050B00060E085E294E00E946D9E60E087E194E00C
:1050C0000E946D9E60E081E094E00E946D9E60E031
:1050D00080EF93E00E946D9E60E08BED93E00E9474
:1050E0006D9E61E088EC93E00E946D9E47C6009142
:1050F00047181091481883E0D12C40E08150E9F026
:10510000D8019C91292F2B7F2134C1F711962C9126
:105110002133A1F7913421F0953421F441E002C00C
:10512000DD24D39498012E5F3F4F89012F5F3F4FBD
:10513000F80190819032C9F3E1CF442369F0E3E3B1
:10514000FAE184917F012FEFE21AF20A882321F01D
:105150000E94188AF701F5CFDD2069F0EDE6F5E051
:1051600084917F013FEFE31AF30A882321F00E9424
:10517000188AF701F5CFD8018D918D01882309F4A4
:10518000A7CB0E94188AF7CF0E9431C0F7C581E0F3
:1051900080934C0580934B05F1C588EC90E00E940C
:1051A00051948111EBC584E40E940C4C882309F4CE
:1051B00041C00E94D54B6B017C0111E020E030E042
:1051C000A9010E946EE9811101C010E01093C2177D
:1051D00020E030E0A901C701B6010E946EE98823F2
:1051E00049F10E94D54BE091860FB4E0EB9FF001AE
:1051F0001124E953F84E608371838283938320E006
:1052000030E0A9016091C7177091C8178091C91744
:105210009091CA170E946EE981110CC080E090E065
:10522000A0EEBFE38093C7179093C817A093C91748
:10523000B093CA170E94A7B9A1C5F70181917F0158
:105240000E940C4C882351F00E94D54B0E9434EFF1
:10525000D8016D937D938D939C9313970C5F1F4F93
:10526000C016D10651F70E9428B788C5E7E5EE2E93
:10527000E2E0FE2E08E017E0F70181917F010E9435
:105280000C4C882341F00E94D54BD8016D937D933F
:105290008D939C9313970C5F1F4FB7E008311B074A
:1052A00059F76CC583E50E94554C8823A1F00E94F4
:1052B000D54B60930007709301078093020790938A
:1052C00003076093FC067093FD068093FE0690939F
:1052D000FF0610E001C011E080E50E94554C8823D4
:1052E00059F00E94D54B609300077093010780939B
:1052F00002079093030710E082E50E94554C882333
:1053000059F00E94D54B6093040770930507809372
:1053100006079093070710E084E50E94554C882308
:1053200059F00E94D54B6093FC067093FD06809364
:10533000FE069093FF0622C5112309F41FC5409174
:10534000000750910107609102077091030787E7FA
:1053500095E00E94D2B340910407509105076091F7
:1053600006077091070784E795E00E94D2B3409149
:10537000FC065091FD066091FE067091FF0681E7E4
:1053800095E00E94D2B38AE00E94188AF7C481E5B2
:105390000E940C4C8823C1F0809125049091260432
:1053A000009739F04AE050E060E070E00E94EDE7DD
:1053B00003C060E070E0CB01609318077093190799
:1053C00080931A0790931B0783E50E940C4C882357
:1053D00051F00E94D54B6093200770932107809372
:1053E00022079093230784E50E940C4C882351F0F8
:1053F0000E94D54B60931C0770931D0780931E0776
:1054000090931F0788E50E940C4C882351F00E945E
:10541000D54B6093E8067093E9068093EA06909373
:10542000EB0689E50E940C4C882351F00E94D54B75
:105430006093EC067093ED068093EE069093EF0672
:105440008AE50E940C4C8823F1F00E94D54B6093B2
:10545000F0067093F1068093F2069093F3062DEC1C
:105460003CEC4CEC5DE30E946EE9181664F0E7E852
:10547000F5E084918F010F5F1F4F882321F00E9478
:10548000188AF801F6CF85E40E940C4C882309F4B1
:1054900075C40E94D54B6093F4067093F506809313
:1054A000F6069093F7066AC467E5C62E62E0D62E2C
:1054B0007DE4E72E75E0F72E10E0F60181916F0193
:1054C0000E940C4C882359F00E94D54BD7016D9354
:1054D0007D938D939C931397812F0E9411941F5F4E
:1054E000B4E0EB0EF11C133041F70C949F200E94A6
:1054F00017C4811143C406E014E2E6E3F4E0FDAB17
:10550000ECAB9E012F5F3F4F59015FE4852E54E2C3
:10551000952E1901F8016591759185919491ACA929
:10552000BDA9CD90DD90ED90FD90BDABACABA701DA
:1055300096010E94EAED2B013C01F1016083718329
:105540008283938320E030E040EA51EC0E9411F026
:1055500087FD0AC020E030E040EA51E4C301B20117
:105560000E946EE918162CF4F401849118160CF4BC
:1055700052C4D101CD90DD90ED90FD901D0120E051
:1055800030E040EA51ECC701B6010E9411F087FDFE
:105590000AC020E030E040EA51E4C701B6010E94B1
:1055A0006EE918164CF5EEE1FAE184918F010F5F78
:1055B0001F4F811103C0E9EBF5E004C00E94188A77
:1055C000F801F3CF84918F010F5F1F4F882321F0E3
:1055D0000E94188AF801F6CF88E290E099A388A388
:1055E00088EC90E09DA78CA7BE01605E7F4FCE0146
:1055F0008C960E9414C5C2C30C5F1F4FBFEF8B1A5D
:105600009B0AE4E202311E0709F084CF4DE4E42E48
:1056100045E0F42E10E0F50181919191A191B191B5
:105620005F01F70181939193A193B1937F01812F42
:105630000E9411941F5F133071F70E94A49E83E9AA
:1056400092E09DA78CA704E610E019A308A3BE0171
:10565000645D7F4FCE0180960E9414C58AEB92E074
:105660009DA78CA719A308A3BE01645D7F4FCE013F
:1056700080960E9414C582C383E50E94554C8823FE
:1056800009F47CC30E94A54B70930302609302024D
:1056900075C38DED90E00E94519481116FC383E535
:1056A0000E94554C811103C0E3E3FAE13AC0009136
:1056B000860F10E00E94A54B000F111FF801E05C5F
:1056C000FD4F718360838091860F90E07C01EE0C2A
:1056D000FF1CEE0CFF1C87010F5D1D4F880F991FEB
:1056E000FC01E05CFD4F60817181072E000C880B8E
:1056F000990B0E9474E92AE037ED43E25CE30E94D3
:10570000D3E9F701ED53F84E208131814281538175
:105710000E94D3E9D8016D937D938D939C93139749
:105720002DC384918F010F5F1F4F882321F00E94AA
:10573000188AF801F6CF85E40E94188A8091860FB6
:10574000805D0E94188AE091860FF0E0EE0FFF1F47
:10575000E05CFD4F6081718187ED95E00E94EFB3C1
:1057600085E20E94188A8AE00E94188A07C380E5B1
:105770000E940C4C882309F401C30E94A54B6B01C5
:105780007C0183E50E94554C882321F00E94A54BA3
:105790008B0102C00FEF1FEFC8010196039708F0BD
:1057A000EDC2D7FCEBC28C2DEFEDF5E0949189179B
:1057B00009F43CC33196B6E0EF30FB07B9F739C3C3
:1057C00083E50E94554C882319F00E94A54B02C026
:1057D00064E071E079A368A380E50E94554C8823BA
:1057E00039F00E94A54B6938E3E17E0730F402C02E
:1057F00068EE73E07A83698304C088E893E19A8352
:105800008983BE01605E7F4FCE0101960E9414C560
:10581000B5C285E40E94554C811110C080E50E94FC
:105820000C4C882391F00E94D54B6093740F7093B9
:10583000750F8093760F9093770F07C00E94B54B3A
:10584000882361F3EEE1FAE171C089E40E940C4C17
:10585000882381F00E94D54B2CEA35EC47E25EE3C9
:105860000E94D3E96093700F7093710F8093720F51
:105870009093730F84E40E940C4C882381F00E9463
:10588000D54B2CEA35EC47E25EE30E94C7EE60930D
:10589000780F7093790F80937A0F90937B0FE3E3E7
:1058A000FAE184918F010F5F1F4F882321F00E943E
:1058B000188AF801F6CF4091740F5091750F6091DE
:1058C000760F7091770F87E196E00E94D2B32CEAB1
:1058D00035EC47E25EE36091700F7091710F80913B
:1058E000720F9091730F0E94C7EEAB01BC0183E170
:1058F00096E00E94D2B32CEA35EC47E25EE3609179
:10590000780F7091790F80917A0F90917B0F0E94A0
:10591000D3E9AB01BC018FE096E00E94D2B38AE0EC
:105920000E94188A2BC20E94188AF80184918F0164
:105930000F5F1F4F8111F7CFEBE1F6E084918F01EC
:105940000F5F1F4F882309F419C20E94188AF801BB
:10595000F5CF83E50E940C4C182F882371F00E942C
:10596000D54B0E942FEF709326026093250221E011
:10597000672B09F020E02093240780E50E940C4C5F
:10598000882359F02091250230912602232B11F013
:105990000E94C64B80932407F1C11111EFC1E3E3CC
:1059A000FAE184918F010F5F1F4F882321F00E943D
:1059B000188AF801F6CF80912407882319F06BE14B
:1059C00073E002C06EE173E082E496E00E9408B4E6
:1059D000609125027091260281E396E00E94EFB368
:1059E000EDE2F6E084918F010F5F1F4F882309F4E9
:1059F000C5C10E94188AF801F5CF0E945A98BEC10D
:105A000080E50E940C4C882351F00E94D54B609396
:105A10006C0F70936D0F80936E0F90936F0F89E4EE
:105A20000E940C4C882381F00E94D54B2CEA35EC67
:105A300047E25EE30E94D3E96093680F7093690FB9
:105A400080936A0F90936B0F84E40E940C4C882320
:105A500081F00E94D54B2CEA35EC47E25EE30E94D0
:105A6000C7EE6093640F7093650F8093660F9093F9
:105A7000670FE3E3FAE184918F010F5F1F4F8823E3
:105A800021F00E94188AF801F6CF40916C0F5091D6
:105A90006D0F60916E0F70916F0F8DE596E00E9413
:105AA000D2B32CEA35EC47E25EE36091680F709167
:105AB000690F80916A0F90916B0F0E94C7EEAB0146
:105AC000BC0189E596E00E94D2B32CEA35EC47E2AE
:105AD0005EE36091640F7091650F8091660F909105
:105AE000670F0E94D3E9AB01BC0185E596E00E94F7
:105AF000D2B38AE00E94188A41C10E94188AF80134
:105B000084918F010F5F1F4F8111F7CFE1E6F6E01F
:105B100084918F010F5F1F4F882309F42FC10E94CA
:105B2000188AF801F5CF0E94329728C10E94327678
:105B300025C10E948DCB22C183E50E940C4C882395
:105B400021F00E94C64B91E089270E94F8C616C139
:105B500081E08093470F0E942E701092470F882398
:105B600009F40CC1E3E3FAE184918F010F5F1F4F49
:105B7000811103C0E0E7F6E004C00E94188AF80132
:105B8000F3CF84918F010F5F1F4F882309F4F6C074
:105B90000E94188AF801F5CF8091B909882309F489
:105BA000EDC081E08093BC09E9C08AE50E94554CB4
:105BB000811103C0EEE7F6E00BC00E94D54B609365
:105BC0002518709326188093271890932818D6C00C
:105BD00084918F010F5F1F4F882321F00E94188A44
:105BE000F801F6CF4091251850912618609127189A
:105BF000709128188BE796E00E94D2B38AE00E9449
:105C0000188ABCC08BE40E94554C811103C0E3E3A9
:105C1000FAE136C08BE40E94554C8823C1F00E9403
:105C2000D54B6B017C0120E030E0A9010E9411F00E
:105C300087FD0AC020E030E040E251E4C701B60130
:105C40000E946EE9181634F4EDE9F6E00EC0C12C9E
:105C5000D12C76010E94A969C092F806D092F9066B
:105C6000E092FA06F092FB0689C084918F010F5FE3
:105C70001F4F882309F482C00E94188AF801F5CFCB
:105C800084918F010F5F1F4F882321F00E94188A93
:105C9000F801F6CF4091F8065091F9066091FA06A6
:105CA0007091FB068CEB96E00E94D2B38AE00E94D2
:105CB000188A64C081E08093270283E50E94554CD6
:105CC000882339F00E94C64B811158C00E9464D1CC
:105CD00055C083E50E940C4CF7CF0E9448C54EC0CA
:105CE000F09049180E94A9691091DB1780E00E948A
:105CF000A692FF2029F1E3E3FAE184918F010F5F7F
:105D00001F4F882321F00E94188AF801F6CF84E5FE
:105D10000E94188A6F2D70E080E090E04AE00E94B7
:105D20003B8D80E20E94188AE9EDF6E084918F01B4
:105D30000F5F1F4F882311F10E94188AF801F6CFD8
:105D400010925910812F0E94A692E3E3FAE1849108
:105D50008F010F5F1F4F882321F00E94188AF801DE
:105D6000F6CF6091591070E087EC96E00E94EFB397
:105D70008AE00E94188A02C00E9448C510925A10F8
:105D80000E9447D193C00E94FA900E9473CDF6CF33
:105D90000E94A54BAB01BC014093330C5093340CD3
:105DA0006093350C7093360C82E89BE00E944EA104
:105DB000E5CF0E94A96988E50E940C4C882331F048
:105DC0005F9A809135048E7F8093350489E50E9427
:105DD0000C4C882339F08A9A479A809135048D7F3C
:105DE000809335048AE50E940C4C882361F08091F1
:105DF00008018095817080930601479A809135044F
:105E00008B7F8093350485E40E940C4C882309F431
:105E1000B5CF129AB3CFF7FAF094F7F8F094D10116
:105E2000CD92DD92ED92FC921397A3CB0E9481E478
:105E3000A5CF0E94A969BC2C60E08C2D0E94BBC537
:105E40000F3FBFEF1B0759F48C2D0E9465C531E051
:105E500020E0892B09F030E0032F122F05C001301C
:105E6000110561F401E010E08B2D0E9465C58017DB
:105E7000910709F483CF0E945BAAF6CF00E010E0FF
:105E8000F3CF61E0812F0E94BBC56E2D812F0E9450
:105E90008DC5F12CB701812F0E94F7C5193009F08B
:105EA0006DCFF0924704E092460468CFC657DF4FAB
:105EB0000FB6F894DEBF0FBECDBFDF91CF911F911B
:105EC0000F91FF90EF90DF90CF90BF90AF909F9099
:105ED0008F907F906F905F904F903F902F9008959C
:105EE0002F923F924F925F926F927F928F929F92EA
:105EF000AF92BF92CF92DF92EF92FF920F931F93D8
:105F0000CF93DF93CDB7DEB76F970FB6F894DEBFB0
:105F10000FBECDBFC0905004D0905104E090520409
:105F2000F090530420E030E040EA50E4C701B601AD
:105F30000E946EE987FD19C120E030E041E953E499
:105F4000C701B6010E9411F018160CF40EC1109290
:105F5000D60D1092D50D809109014091D40D042EDB
:105F6000000C550B817021E0822790E048175907FB
:105F700009F433C080910901817028272093D40D42
:105F800081111BC00E94196BE1E0FDE084918F013B
:105F9000882351F0082E000C990B0E94146B0F5FA0
:105FA0001F4FF8018491F4CF8DE090E00E94146BB4
:105FB0008AE090E00E94146B10C0E5E0FDE084915F
:105FC0008F01882389F3082E000C990B0E94146B13
:105FD0000F5F1F4FF8018491F4CF8091C70D83307C
:105FE00009F44CC02CF4882351F08130D9F072C0F0
:105FF000843009F43EC0853009F44DC06BC08091F7
:10600000B909882309F466C081E08093C70D0E9416
:1060100090586093CB0D7093CC0D8093CD0D9093E1
:10602000CE0D58C08091B909811154C08091850B63
:10603000882321F082E08093C70D4CC01092C70DD9
:10604000EDEFFCE084918F01882351F0082E000CC5
:10605000990B0E94146B0F5F1F4FF8018491F4CFCE
:106060008DE090E00E94146B8AE090E00E94146B37
:1060700031C08091140E8823E9F22CC08091B909B7
:10608000811128C080913B0990913C09891B8F7038
:1060900009F496C01FC08091B90981111BC080917D
:1060A0003B0990913C09891B8F7009F4ABC012C069
:1060B0008DE090E00E94146B8AE090E00E94146BE7
:1060C0001092C70D8DED9CE090932C0780932B07C9
:1060D0000E94448A8091BC0D9091BD0D03974CF5B0
:1060E00077E0272E79E0372EE0E68E2EEAEE9E2E20
:1060F000A12CB12C82E29FE00E94274B18161906B2
:10610000C4F48091BC0D9091BD0D049794F482E28B
:106110009FE00E94EB4A8093C20DE091C30DF09185
:10612000C40D8A3019F08D3009F07DC0309709F028
:1061300083C08091BC0D9091BD0D009711F40C941B
:10614000E33E01979093BD0D8093BC0D8091BE0DF1
:106150009091BF0D019664E070E00E94D4F090939E
:10616000BF0D8093BE0D0C94E33E8091D50D9091B0
:10617000D60D8136FAEE9F07E8F01092D60D1092F8
:10618000D50DE9E0FDE084918F01882351F0082EC0
:10619000000C990B0E94146B0F5F1F4FF801849144
:1061A000F4CF8DE090E00E94146B8AE090E00E94B2
:1061B000146BD1CE01969093D60D8093D50DCBCE96
:1061C00089EE9CE090932C0780932B070E94448AD1
:1061D0008091140E882311F082E001C084E0809346
:1061E000C70DE5EEFCE084918F01882309F438CFD8
:1061F000082E000C990B0E94146B0F5F1F4FF801C3
:106200008491F3CFE1EEFCE084918F01882309F4BF
:106210004FCF082E000C990B0E94146B0F5F1F4F7D
:10622000F8018491F3CF8A3309F480CFEF35F1057B
:1062300014F40C94773C7ACF8091C00D9091C10DED
:1062400020E6289F7001299FF00C11248701045C2F
:10625000134FE00FF11F108261E470E0C8010E944B
:106260003BF1009711F40C945B3C9093C60D809326
:10627000C50D801B910B8E0D9F1D60E070E0835C4F
:10628000934F0E946FE50E942FEFCB01770FAA0B6F
:10629000BB0B8232910510F00C945B3CFC0188270B
:1062A000EE58FF4F8F4F0C94E7F0E8EDFCE084913F
:1062B0008F01882351F0082E000C990B0E94146B5B
:1062C0000F5F1F4FF8018491F4CF20E030E040E0F1
:1062D0005FE3609150047091510480915204909159
:1062E00053041EC0E3EDFCE084918F01882351F03C
:1062F000082E000C990B0E94146B0F5F1F4FF801C2
:106300008491F4CF60914E0470914F04072E000CDD
:10631000880B990B0E9474E920E030E040E05FE3D5
:106320000E94EBED0E942FEFCB010E94AE4D0E9428
:10633000DFDA8DE090E00E94146B8AE090E00E942A
:10634000146B0C945B3CEEECFCE084918F01882391
:1063500051F0082E000C990B0E94146B0F5F1F4F19
:10636000F8018491F4CF20E030E040E05FE36091F9
:106370004A0470914B0480914C0490914D04D0CF0D
:10638000E9ECFCE084918F01882351F0082E000C89
:10639000990B0E94146B0F5F1F4FF8018491F4CF8B
:1063A0006091480470914904B1CF20914604309126
:1063B000470444E6429FC001439F900D11246FEFB4
:1063C00070E00E94D4F08B016536710510F004E690
:1063D00010E0E4ECFCE084917F01882359F0082E62
:1063E000000C990B0E94146BFFEFEF1AFF0AF701E4
:1063F0008491F3CFB80180E090E028C7E0ECFCE0A6
:1064000084918F01882351F0082E000C990B0E9473
:10641000146B0F5F1F4FF8018491F4CF80E290E07E
:106420000E94146BECEBFCE084918F01882351F007
:10643000082E000C990B0E94146B0F5F1F4FF80180
:106440008491F4CF609136047091370480913804C0
:10645000909139040E94E0DA80E290E00E94146B8F
:10646000E8EBFCE084918F01882351F0082E000CAA
:10647000990B0E94146B0F5F1F4FF8018491F4CFAA
:1064800060913A0470913B0480913C0490913D04EA
:106490000E94E0DA80E290E00E94146BE4EBFCE002
:1064A00084918F01882351F0082E000C990B0E94D3
:1064B000146B0F5F1F4FF8018491F4CF60913E047D
:1064C00070913F0480914004909141040E94E0DA71
:1064D00080E290E092C58091B909882309F450C008
:1064E000EFEAFCE084918F01882351F0082E000C24
:1064F000990B0E94146B0F5F1F4FF8018491F4CF2A
:106500008091BA09882359F18091850B882329F15C
:1065100080912F0C9091300CA091310CB091320CE5
:106520000097A105B105C1F0BC01CD016D597F4FA8
:106530008F4F9F4F24E630E040E050E00E948DED09
:106540006091330C7091340C8091350C9091360C25
:106550000E948DED822F01C080E090E0E6CEEBEA54
:10656000FCE084918F01882309F4E3CE082E000C0F
:10657000990B0E94146B0F5F1F4FF8018491F3CFAA
:10658000E3EAFCE084918F01882309F4D2CE082E3F
:10659000000C990B0E94146B0F5F1F4FF801849140
:1065A000F3CFEEE9FCE084918F01882351F0082EAF
:1065B000000C990B0E94146B0F5F1F4FF801849120
:1065C000F4CF8091CB0D9091CC0DA091CD0DB091D9
:1065D000CE0D892B8A2B8B2B09F477C00E94905803
:1065E000A50194010E948DED69017A016091CB0DA6
:1065F0007091CC0D8091CD0D9091CE0DA50194019F
:106600000E948DED8601021B130BC8016CE370E044
:106610000E94C0F0CB019927EAE0F0E0BF010E94A0
:10662000D4F0282FCB01BF010E94D4F0805D80936D
:106630002D04205D20932E0410922F048DE294E00F
:106640000E94DFDA80E290E00E94146BECE9FCE04B
:1066500084917F01882359F0082E000C990B0E9429
:10666000146BFFEFEF1AFF0AF7018491F3CF80E27A
:1066700090E00E94146BC8016CE370E00E94C0F0CF
:106680006AE070E00E94D4F0605D60932D04805D4C
:1066900080932E0410922F048DE294E00E94DFDAA2
:1066A00080E290E00E94146BEAE9FCE084918F01A3
:1066B000882309F43ECE082E000C990B0E94146B1F
:1066C0000F5F1F4FF8018491F3CF80E290E00E94AA
:1066D000146BE2E9FCE084918F01882309F429CE50
:1066E000082E000C990B0E94146B0F5F1F4FF801CE
:1066F0008491F3CF1092F50D8091090180FF11C0B4
:10670000EEE8FCE084918F01882309F412CE082E74
:10671000000C990B0E94146B0F5F1F4FF8018491BE
:10672000F3CF83E50E9475DA882341F00E9490DA66
:106730000E9434EF7093CA0D6093C90DEAE8FCE043
:1067400084918F01882351F0082E000C990B0E9430
:10675000146B0F5F1F4FF8018491F4CF8DE090E030
:106760000E94146B8AE090E00E94146B8091130EDB
:10677000882309F442C28091C90D9091CA0D8430DA
:10678000910509F4C8C08830910509F47DC1892BB1
:1067900009F0D9C3EEEAFAE084918F01882351F021
:1067A000082E000C990B0E94146B0F5F1F4FF8010D
:1067B0008491F4CF8DE090E00E94146B8AE090E029
:1067C0000E94146BE3EAFAE084918F01882351F070
:1067D000082E000C990B0E94146B0F5F1F4FF801DD
:1067E0008491F4CF8DE090E00E94146B8AE090E0F9
:1067F0000E94146BE7E9FAE084918F01882351F03D
:10680000082E000C990B0E94146B0F5F1F4FF801AC
:106810008491F4CF8DE090E00E94146B8AE090E0C8
:106820000E94146BEBE8FAE084918F01882351F009
:10683000082E000C990B0E94146B0F5F1F4FF8017C
:106840008491F4CF8DE090E00E94146B8AE090E098
:106850000E94146BEDE7FAE084918F01882351F0D8
:10686000082E000C990B0E94146B0F5F1F4FF8014C
:106870008491F4CF8DE090E00E94146B8AE090E068
:106880000E94146BEFE6FAE084918F01882351F0A7
:10689000082E000C990B0E94146B0F5F1F4FF8011C
:1068A0008491F4CF8DE090E00E94146B8AE090E038
:1068B0000E94146BE2E6FAE084918F01882351F084
:1068C000082E000C990B0E94146B0F5F1F4FF801EC
:1068D0008491F4CF8DE090E00E94146B8AE090E008
:1068E0000E94146BE5E5FAE084918F01882351F052
:1068F000082E000C990B0E94146B0F5F1F4FF801BC
:106900008491F4CF8DE090E00E94146B8AE090E0D7
:106910000E94146B18C3E7E4FAE084918F01882386
:1069200051F0082E000C990B0E94146B0F5F1F4F43
:10693000F8018491F4CF8DE090E00E94146B8AE01E
:1069400090E00E94146BE9E3FAE084918F018823C0
:1069500051F0082E000C990B0E94146B0F5F1F4F13
:10696000F8018491F4CF8DE090E00E94146B8AE0EE
:1069700090E00E94146BE3E2FAE084918F01882397
:1069800051F0082E000C990B0E94146B0F5F1F4FE3
:10699000F8018491F4CF8DE090E00E94146B8AE0BE
:1069A00090E00E94146BEDE0FAE084918F0188235F
:1069B00051F0082E000C990B0E94146B0F5F1F4FB3
:1069C000F8018491F4CF8DE090E00E94146B8AE08E
:1069D00090E00E94146BEBEFF9E084918F01882323
:1069E00051F0082E000C990B0E94146B0F5F1F4F83
:1069F000F8018491F4CF8DE090E00E94146B8AE05E
:106A000090E00E94146BE9EEF9E084918F018823F5
:106A100051F0082E000C990B0E94146B0F5F1F4F52
:106A2000F8018491F4CF8DE090E00E94146B8AE02D
:106A300090E00E94146BEBEDF9E084918F018823C4
:106A400051F0082E000C990B0E94146B0F5F1F4F22
:106A5000F8018491F4CF8DE090E00E94146B8AE0FD
:106A600090E00E94146BEDECF9E084918F01882393
:106A700009F448CF082E000C990B0E94146B0F5F8D
:106A80001F4FF8018491F3CFE6ECF9E084918F0178
:106A9000882351F0082E000C990B0E94146B0F5F95
:106AA0001F4FF8018491F4CF8DE090E00E94146BA9
:106AB0008AE090E00E94146BEFEBF9E084918F0183
:106AC000882351F0082E000C990B0E94146B0F5F65
:106AD0001F4FF8018491F4CF8DE090E00E94146B79
:106AE0008AE090E00E94146BE8EAF9E084918F015B
:106AF000882351F0082E000C990B0E94146B0F5F35
:106B00001F4FF8018491F4CF8DE090E00E94146B48
:106B10008AE090E00E94146BE1E9F9E084918F0132
:106B2000882351F0082E000C990B0E94146B0F5F04
:106B30001F4FF8018491F4CF8DE090E00E94146B18
:106B40008AE090E00E94146BEAE7F9E084918F01FB
:106B5000882351F0082E000C990B0E94146B0F5FD4
:106B60001F4FF8018491F4CF8DE090E00E94146BE8
:106B70008AE090E00E94146BE3E6F9E084918F01D3
:106B8000882351F0082E000C990B0E94146B0F5FA4
:106B90001F4FF8018491F4CF8DE090E00E94146BB8
:106BA0008AE090E00E94146BE0E5F9E084918F01A7
:106BB000882351F0082E000C990B0E94146B0F5F74
:106BC0001F4FF8018491F4CF8DE090E00E94146B88
:106BD0008AE090E00E94146BEDE3F9E084918F016C
:106BE000882309F48FCE082E000C990B0E94146B99
:106BF0000F5F1F4FF8018491F3CF8091BA0988236A
:106C000009F478C181E08093370C1092390C10920E
:106C1000380C89E09AE00E9495A38BE1E9E0FAE064
:106C2000DE01159601900D928A95E1F78091070A91
:106C30009091080A9C838B8385E692E09A838983EE
:106C400040E050E0BE016F5F7F4F80E090E00E9427
:106C50004A6DCE0101960E94F1A9C090380CD090E7
:106C6000390C0091C90D1091CA0DC601801B910B02
:106C7000049720F06801F3E0CF0ED11C5EE2452EB0
:106C800059E0552E6FE1662E69E0762EC016D106CA
:106C900008F459C10115110509F09DC06DEB79E0AB
:106CA00089E09AE00E945DA262E273E08DEB99E0D8
:106CB0000E9446F1892B09F048C0F20184914EE20E
:106CC000E42E49E0F42E882359F0082E000C990B8D
:106CD0000E94146BFFEFEF1AFF0AF7018491F3CFC4
:106CE0008DE090E00E94146B8AE090E00E94146BAB
:106CF000F30184913FE1E32E39E0F32E882359F02C
:106D0000082E000C990B0E94146BFFEFEF1AFF0A7C
:106D1000F7018491F3CF8DE090E00E94146B8AE03C
:106D200090E00E94146B80E090E00E94D9DAEFE0DE
:106D3000F9E084917F012FEFE21AF20A882309F427
:106D4000D6C00E94188AF701F4CFEBE0F9E08491F5
:106D50007F01882359F0082E000C990B0E94146BB8
:106D6000FFEFEF1AFF0AF7018491F3CF8DE090E077
:106D70000E94146B8AE090E00E94146BF1018491F0
:106D800027E0E22E29E0F22E882359F0082E000C8D
:106D9000990B0E94146BFFEFEF1AFF0AF701849121
:106DA000F3CF8DE090E00E94146B8AE090E00E94A7
:106DB000146B80E090E00E94D9DAE2E0F9E084917F
:106DC0007F012FEFE21AF20A882309F490C00E9493
:106DD000188AF701F4CF60E070E0C80101970E94C3
:106DE000106F8091BB09882309F45AC0E0E0F9E0F4
:106DF00084917F01882359F0082E000C990B0E9482
:106E0000146BFFEFEF1AFF0AF7018491F3CF8DEBBC
:106E100099E00E94DFDA8DE090E00E94146B8AE036
:106E200090E00E94146BEEEFF8E084917F018823DC
:106E300059F0082E000C990B0E94146BFFEFEF1A0B
:106E4000FF0AF7018491F3CF8AEC99E00E94DFDA20
:106E50008DE090E00E94146B8AE090E00E94146B39
:106E6000C8010E94D9DAECEFF8E084917F012FEF9E
:106E7000E21AF20A882321F00E94188AF701F5CF5E
:106E80009AECE92E99E0F92EF70181917F01882390
:106E900019F00E94188AF8CF8AE00E94188A27C049
:106EA0008DEB99E00E94DFDA8DE090E00E94146B98
:106EB0008AE090E00E94146B8AEC99E00E94DFDA8D
:106EC0008DE090E00E94146B8AE090E00E94146BC9
:106ED000C8010E94D9DA8AECE82E89E0F82EF70181
:106EE00081917F018823C1F20E94188AF8CF0F5F39
:106EF0001F4FCCCEEDEEF8E084918F01882351F046
:106F0000082E000C990B0E94146B0F5F1F4FF801A5
:106F10008491F4CF8DE090E00E94146B8AE090E0C1
:106F20000E94146BEEEDF8E084918F01882309F440
:106F3000E9CC082E000C990B0E94146B0F5F1F4FB9
:106F4000F8018491F3CFE6E8FCE084918F01882377
:106F500009F4EFC9082E000C990B0E94146B0F5F07
:106F60001F4FF8018491F3CF8091B909882339F03C
:106F70000E947C6CA0C48091B9098823E9F00E942A
:106F8000BCC099C48091C70D823019F0833609F0D6
:106F900092C40E945B6CE2E8FCE084918F0188233C
:106FA00009F4C7C9082E000C990B0E94146B0F5FDF
:106FB0001F4FF8018491F3CF8091C70D833609F0FC
:106FC0007AC4DDCF89E79CE00E9414AA80913B0936
:106FD00090913C09891B8F7009F06DC48091C70D99
:106FE000823009F468C4833609F099C464C48DE022
:106FF00090E00E94146B8AE090E00E94146B99C9A3
:1070000080913B0990913C09891B8F7009F053C412
:107010008091C70D823009F44EC4833609F44BC405
:107020008091850B8111CFC446C483E50E9475DA37
:10703000811126C083E40E9475DA882309F43BC4D9
:1070400080913B0990913C09891B8F7009F033C4F2
:1070500020E030E040E251E460913E0470913F0452
:1070600080914004909141040E946EE987FF08C01E
:1070700086E69CE090932C0780932B070E94448A1D
:107080000E9490DA20E030E0A9010E946EE987FDBD
:1070900010C00E9490DA20E030E849E853E40E94F2
:1070A00011F018164CF00E9490DA0E9434EFCB01D8
:1070B00005C080E090E002C083E191E00E94B77BD0
:1070C000FAC383E50E9475DA882309F4F4C30E94A9
:1070D00090DA20E030E0A9010E946EE987FD10C03F
:1070E0000E9490DA20E030E046E153E40E9411F083
:1070F00018164CF00E9490DA0E9434EFCB0105C0C4
:1071000080E090E002C086E990E00E94E44DD3C3A5
:1071100083E50E9475DA8823D9F00E9490DA20E096
:1071200030E04FE753E40E94D3E920E030E048EC40
:1071300052E40E94C7EE0E9434EF6F3F710519F0D0
:1071400010F06FEF70E07093470460934604F1C84D
:107150008FEF90E09093470480934604EAC88091B3
:107160003B0990913C09891B8F7009F0E2C880911E
:10717000B9098111DEC80E941D985F9A809135047B
:107180008E7F809335048A9A479A809135048D7F4B
:107190008093350480910801809581708093060169
:1071A000479A809135048B7F80933504129AC1C829
:1071B00083E50E9475DA882319F10E9490DA20E0B5
:1071C00030E040E252E40E946EE987FD0FC00E9469
:1071D00090DA20E030EC49E754E40E9411F01816F0
:1071E00044F00E9490DA0E942FEF05C068E270E040
:1071F00002C067EE73E070930302609302025BC308
:10720000E0E6FCE084918F01882351F0082E000C09
:10721000990B0E94146B0F5F1F4FF8018491F4CFFC
:10722000C0900202D09003020D2C000CEE08FF0863
:10723000F7FE0EC06DE282E29FE00E949E4A662742
:107240007727CB016C197D098E099F094AE003C09D
:107250004AE0C701B6010E9499DA6BC880913B09E8
:1072600090913C09891B8F7009F025C38091C70D4F
:10727000823009F420C3833609F0EBC21CC380912D
:107280003B0990913C09891B8F7009F052C880918D
:10729000C70D823009F44DC8833609F0B6C349C81A
:1072A00080913B0990913C09891B8F7009F003C3C1
:1072B0008091C70D823009F4FEC2833609F0FBC409
:1072C000FAC280913B0990913C09891B8F7009F0AB
:1072D000F2C28091C70D823009F4EDC2833609F005
:1072E00020C5E9C280913B0990913C09891B8F70B0
:1072F00009F0E1C28091C70D823009F4DCC2833607
:1073000009F045C5D8C28091F50D811103C00E94D6
:10731000196BC4C18E3271F58091F60D8E3209F071
:1073200046C180915A0B882309F4B8C181508093DB
:107330005A0B882361F090E001974FE1489F90013C
:10734000499F300D1124C9018C5D954F02C086EE16
:1073500099E02BE1FC013496A9E0BAE001900D928E
:107360002A95E1F7FC01828193819093080A80932A
:10737000070A94C18C3309F01AC164E273E085EF07
:107380009DE00E9446F1892B21F481E08093130E49
:1073900085C163E373E085EF9DE00E9446F1892B90
:1073A00079F4EAEBF8E084918F010F5F1F4F882397
:1073B00021F00E94188AF801F6CF8DE998E0E4C028
:1073C0006AE473E085EF9DE00E9446F1892B79F431
:1073D000E9E7F8E084918F010F5F1F4F882321F0C8
:1073E0000E94188AF801F6CF86E698E0CDC061E6E3
:1073F00073E085EF9DE00E9446F1892B79F4EBE480
:10740000F8E084918F010F5F1F4F882321F00E94C5
:10741000188AF801F6CF86E498E0B6C06FE673E00C
:1074200085EF9DE00E9446F1892B79F4E6E2F8E0D1
:1074300084918F010F5F1F4F882321F00E94188ACB
:10744000F801F6CF81E298E09FC062E873E085EF33
:107450009DE00E9446F1892B79F4E6E0F8E0849102
:107460008F010F5F1F4F882321F00E94188AF801B7
:10747000F6CF8DEF97E088C060E973E085EF9DE07F
:107480000E9446F1892B71F40AED17E0F80184910E
:10749000882329F00F5F1F4F0E94188AF7CF83EDD2
:1074A00097E072C066EA73E085EF9DE00E9446F1C6
:1074B000892B79F4E4EBF7E084918F010F5F1F4F84
:1074C000882321F00E94188AF801F6CF8DEA97E010
:1074D0005BC068EB73E085EF9DE00E9446F1892B6D
:1074E00079F4E5E9F7E084918F010F5F1F4F88235E
:1074F00021F00E94188AF801F6CF84E897E044C092
:1075000063EC73E085EF9DE00E9446F1892B79F4EE
:10751000EBE6F7E084918F010F5F1F4F882321F086
:107520000E94188AF801F6CF89E597E02DC06FEC2C
:1075300073E085EF9DE00E9446F1892B79F4EEE33C
:10754000F7E084918F010F5F1F4F882321F00E9485
:10755000188AF801F6CF8CE297E016C06DED73E063
:1075600085EF9DE00E9446F1892BA9F4E2E1F7E066
:1075700084918F010F5F1F4F882321F00E94188A8A
:10758000F801F6CF81E097E090932C0780932B07CA
:107590000E94448A83C06AEE73E085EF9DE00E94FA
:1075A00046F1892B09F07AC01092130E77C01D8224
:1075B00018861C821B8285E692E09A8389838091DB
:1075C0000C0A811103C066EE79E002C065E07AE042
:1075D0006115710519F06C5F7F4F02C060E070E0CB
:1075E00021E045EF5DE0CE0105960E94C4A7882307
:1075F00061F18BE1FE013596A9E0BAE001900D92B0
:107600008A95E1F72B813C813093080A2093070A81
:1076100080915A0B8A3008F03DC091E0980F90930A
:107620005A0BFFE18F9FC0011124DC01A85DB54F0B
:107630004BE1E9E0FAE001900D924A95E1F7FC0197
:10764000EC5DF54F3383228325C0E3E3FAE18491B7
:107650008F010F5F1F4F882321F00E94188AF801C5
:10766000F6CFEBEEF6E084918F010F5F1F4F88237A
:1076700021F00E94188AF801F6CF05EF1DE0F8010D
:1076800081918F01882319F00E94188AF8CF8AE02F
:107690000E94188ACE0101960E94F1A91092F50D60
:1076A0008091090180FF07C1E4EAFBE084918F012A
:1076B000882311F40C949931082E000C990B0E9428
:1076C000146B0F5F1F4FF8018491F2CF8FE40E947B
:1076D00075DA81110C94993183E40E9475DA0C9467
:1076E000993183E50E9475DA811159C08FE40E94B7
:1076F00075DA882319F08CE69BE007C084E50E94C8
:1077000075DA882349F084E49BE090932C078093FA
:107710002B070E94448A43C083E40E9475DA8823C1
:1077200019F08BE19BE0F1CF81E50E9475DA8823A7
:1077300019F083EF9AE0E9CF88E40E9475DA882394
:10774000C9F0EFEEFAE084918F01882351F0082E02
:10775000000C990B0E94146B0F5F1F4FF80184916E
:10776000F4CF8DE090E00E94146B8AE090E00E94DC
:10777000146B15C08CE40E9475DA882381F0EBEE5F
:10778000FAE084918F01882361F3082E000C990B95
:107790000E94146B0F5F1F4FF8018491F4CFE3EB4D
:1077A000FBE084918F01882311F40C949931082E09
:1077B000000C990B0E94146B0F5F1F4FF80184910E
:1077C000F2CF80913B0980913C090C94993183E57B
:1077D0000E9475DA882309F46EC083EC9AE09093D6
:1077E0002C0780932B070E94448AE3EBFBE08491F3
:1077F0008F01882311F40C949931082E000C990BF9
:107800000E94146B0F5F1F4FF8018491F2CFEEEBD3
:10781000FAE084918F01882351F0082E000C990B17
:107820000E94146B0F5F1F4FF8018491F4CFE9EBB6
:10783000FAE084918F01882311F40C949931082E79
:10784000000C990B0E94146B0F5F1F4FF80184917D
:10785000F2CF88E50E9475DA811106C089E50E94A1
:1078600075DA882309F4C3C088E50E9475DA882395
:1078700041F08AE59CE090932C0780932B070E94AF
:10788000448A89E50E9475DA882341F084E59CE00A
:1078900090932C0780932B070E94448A8AE50E94CC
:1078A00075DA882341F08EE49CE090932C07809356
:1078B0002B070E94448A8091C00D9091C10D0196C2
:1078C00064E070E00E94D4F09093C10D8093C00DED
:1078D0008091BC0D9091BD0D01969093BD0D80934C
:1078E000BC0D1092C40D1092C30D0C947A304091CF
:1078F000C00D5091C10D9F012F5F3F4F3093C40DBC
:107900002093C30D90E6949F9001959F300D112414
:10791000245C334FE20FF31F80830C947A30009184
:10792000C50D1091C60D780124E0E20EF11C6AE24B
:1079300070E0C7010E943BF1F80124812F3221F44D
:10794000B8016B5F7F4F03C02C3339F4B70185EF6B
:107950009DE00E944FF10C9499311092F50D009723
:1079600019F0FC01319710828091C50D9091C60DE0
:1079700040E061E004960E94A3D88091850B8823A3
:1079800089F0E5E7FCE084918F01882309F42FCB8F
:10799000082E000C990B0E94146B0F5F1F4FF8010B
:1079A0008491F3CFE1E7FCE084918F01882309F40F
:1079B0001ECB082E000C990B0E94146B0F5F1F4FFB
:1079C000F8018491F3CF0E945B6CEDE6FCE08491BA
:1079D0008F01882311F40C949931082E000C990B17
:1079E0000E94146B0F5F1F4FF8018491F2CF8AE55C
:1079F0000E9475DA811138CF83E40E9475DA8823FA
:107A000009F459CF8AE49CE050CF86E40E9475DAED
:107A1000882309F44DC10E9490DA0E9434EF8B0153
:107A200086E49CE090932C0780932B070E94448A65
:107A300088E50E9475DA882309F451C00E9490DA23
:107A40002B013C012DEC3CEC4CE45EE30E946EE922
:107A50009E012F5F3F4F7901181674F020E030E04F
:107A6000A901C301B2010E9411F018162CF41F9352
:107A70000F938BE39CE005C12DEC3CEC4CEC5DEBF3
:107A8000C301B2010E946EE918167CF020E030E0DC
:107A900040E85FEBC301B2010E9411F018162CF40C
:107AA0001F930F938FE29CE0ECC01F930F93C301D1
:107AB000B2010E942FEF7F936F9385E29CE09F932A
:107AC0008F93FF92EF920E9440E90FB6F894DEBFC9
:107AD0000FBECDBFCE0101960E941F8ADFC089E58F
:107AE0000E9475DA882309F441C00E9490DA2B01C4
:107AF0003C012DEC3CEC4CE45EE30E946EE9FE019F
:107B000031967F01181674F020E030E0A901C3011E
:107B1000B2010E9411F018162CF41F930F938AE102
:107B20009CE0AFC02DEC3CEC4CEC5DEBC301B20132
:107B30000E946EE918167CF020E030E040E85FEB30
:107B4000C301B2010E9411F018162CF41F930F9379
:107B50008EE09CE096C01F930F93C301B2010E9478
:107B60002FEF7F936F9384E09CE0A9CF8AE50E947A
:107B700075DA882309F441C00E9490DA2B013C0198
:107B80002DEC3CEC4CE45EE30E946EE9FE01319684
:107B90007F01181674F020E030E0A901C301B201A2
:107BA0000E9411F018162CF41F930F9389EF9BE09D
:107BB00068C02DEC3CEC4CEC5DEBC301B2010E94C3
:107BC0006EE918167CF020E030E040E85FEBC3017E
:107BD000B2010E9411F018162CF41F930F938DEE32
:107BE0009BE04FC01F930F93C301B2010E942FEF80
:107BF0007F936F9383EE9BE062CF85E40E9475DAFA
:107C0000882309F44BC00E9490DA2B013C012DEC33
:107C10003CEC4CE45EE30E946EE9FE0131967F018C
:107C2000181674F020E030E0A901C301B2010E94EF
:107C300011F018162CF41F930F9388ED9BE021C0D0
:107C40002DEC3CEC4CEC5DEBC301B2010E946EE903
:107C500018167CF020E030E040E85FEBC301B20191
:107C60000E9411F018162CF41F930F938CEC9BE0DC
:107C700008C0C301B2010E942FEF7F936F9381EC84
:107C80009BE09F938F93FF92EF920E9440E90F90A9
:107C90000F900F900F900F900F901CCF8DEB9BE0EB
:107CA00090932C0780932B070E94448A0C9499315F
:107CB00000E010E0B5CE20E030E040E251E4609119
:107CC0003E0470913F0480914004909141040E94D1
:107CD0006EE987FF08C086EB9BE090932C078093AA
:107CE0002B070E94448A82E390E09093490480939A
:107CF00048040E940B7D88EC90E00E94B77BE3EB88
:107D0000FBE084918F01882311F40C949931082EA3
:107D1000000C990B0E94146B0F5F1F4FF8018491A8
:107D2000F2CF20E030E040E251E460913E047091F7
:107D30003F0480914004909141040E946EE987FFC6
:107D400008C08CEA9BE090932C0780932B070E943D
:107D5000448A80E590E090934904809348040E940F
:107D60000B7D80EF90E00E94B77BE3EBFBE084911A
:107D70008F01882311F40C949931082E000C990B73
:107D80000E94146B0F5F1F4FF8018491F2CF80E0C7
:107D900090E00E94B77B10924904109248040E9420
:107DA0000B7DE8EAFBE084918F01882311F40C94A9
:107DB0009931082E000C990B0E94146B0F5F1F4F16
:107DC000F8018491F2CF6F960FB6F894DEBF0FBE24
:107DD000CDBFDF91CF911F910F91FF90EF90DF907A
:107DE000CF90BF90AF909F908F907F906F905F905B
:107DF0004F903F902F9008952F923F924F925F9215
:107E00006F927F928F929F92AF92BF92CF92DF92AA
:107E1000EF92FF920F931F93CF93DF93CDB7DEB70F
:107E200062970FB6F894DEBF0FBECDBFF8948FEF08
:107E30009FEF90938900809388002AE02A8B212C61
:107E4000312C78948091A6049091A704A091A80465
:107E5000B091A904892B8A2B8B2B09F016C2809133
:107E60004A0F8823E1F010924A0F8091480F9091B9
:107E7000490F892B09F409C210925E041092490F30
:107E80001092480F90913B0980913C09981709F492
:107E9000FCC180913C098F5F8F7080933C09809179
:107EA000480F9091490F892B09F4EFC14091A2042A
:107EB0005091A3046091A4047091A50480919E0444
:107EC00090919F04A091A004B091A1040091950409
:107ED00010E020E030E0841B950BA60BB70B0817D1
:107EE00019072A073B0710F4D901C801E82F840FAE
:107EF000951FA61FB71F8093A2049093A304A0937D
:107F0000A404B093A5042091840030918500225EE2
:107F10003F4F40917A0450917B0460917C047091B2
:107F20007D0480916A0490916B04A0916C04B091DF
:107F30006D04840F951FA61FB71F80937A0490933A
:107F40007B04A0937C04B0937D04B7FD1CC0889A89
:107F50008091E1179091E217A091E317B091E41797
:107F600040910402042E000C550B660B770B840F16
:107F7000951FA61FB71F8093E1179093E217A09358
:107F8000E317B093E41740917E0450917F04609111
:107F900080047091810480916E0490916F04A0918F
:107FA0007004B0917104840F951FA61FB71F8093B2
:107FB0007E0490937F04A0938004B0938104B7FD66
:107FC0001CC08E9A8091E5179091E617A091E71753
:107FD000B091E81740910502042E000C550B660B7A
:107FE000770B840F951FA61FB71F8093E5179093FB
:107FF000E617A093E717B093E817409182045091D9
:10800000830460918404709185048091720490913E
:108010007304A0917404B0917504840F951FA61F7A
:10802000B71F8093820490938304A0938404B09339
:108030008504B7FD3FC080915804F0910602882363
:10804000C9F08091560482FF02C0F7FD06C08091FE
:108050005504882311F40C94B148809156049091F2
:10806000570493FF02C0F7FD0CC0809154048111A6
:1080700008C006C080910B0180958870809309012B
:10808000419A4091E9175091EA176091EB1770916E
:10809000EC178F2FFF0F990BAA0BBB0B840F951FAB
:1080A000A61FB71F8093E9179093EA17A093EB17C9
:1080B000B093EC1740918604509187046091880436
:1080C000709189048091760490917704A09178044E
:1080D000B0917904840F951FA61FB71F8093860463
:1080E00090938704A0938804B0938904B7FD3AC0A5
:1080F0004091ED175091EE176091EF177091F017C6
:10810000C09007020C2C000CDD08EE08FF084C0D97
:108110005D1D6E1D7F1D4093ED175093EE1760930C
:10812000EF177093F01740916604509167046091C7
:10813000680470916904841B950BA60BB70B8093A0
:10814000860490938704A0938804B0938904909147
:1081500059048091930493FF02C0815001C08F5F46
:1081600080939304809184009091850082179307F7
:10817000C8F380917A0490917B04A0917C04B09123
:108180007D04B7FD15C0409166045091670460916D
:10819000680470916904841B950BA60BB70B809340
:1081A0007A0490937B04A0937C04B0937D04889818
:1081B00080917E0490917F04A0918004B09181040D
:1081C000B7FD15C040916604509167046091680442
:1081D00070916904841B950BA60BB70B80937E04EA
:1081E00090937F04A0938004B09381048E98809133
:1081F000820490918304A0918404B0918504B7FD1A
:108200003AC040916604509167046091680470918F
:108210006904841B950BA60BB70B80938204909383
:108220008304A0938404B093850480915804882328
:10823000E1F08091560482FF04C08091060287FD20
:1082400005C080915504882309F493C78091560492
:108250009091570493FF04C08091060287FD0BC0E4
:1082600080915404811107C005C080910B01887072
:10827000809309014198E15041F0809184009091F0
:10828000850082179307C8F342CE80911102909126
:108290001202A0911302B0911402892B8A2B8B2B0E
:1082A00009F091C080919404882309F453C0809010
:1082B000A2049090A304A090A404B090A504C09040
:1082C0008F04D0909004E0909104F090920440913B
:1082D0009304C814D904EA04FB0480F480915F0479
:1082E0009091600420916304309164042817390749
:1082F00028F4415040939304019714C08C149D04BA
:10830000AE04BF04E0F480915F049091600420917A
:108310006104309162048217930788F44F5F4093A1
:10832000930401969093600480935F0440910D0242
:1083300050910E0260910F02709110020EC08FEFEB
:108340009FEFDC0180930D0290930E02A0930F0229
:10835000B09310024FEF5FEFBA018091930487FD55
:1083600002C0169A01C016988091840090918500F1
:108370004E96209193042223F1F0149A20918400C8
:108380003091850028173907C8F32091930427FFFF
:1083900002C02F5F01C021502093930414982091B4
:1083A0009304222331F32091840030918500281713
:1083B0003907C8F3DDCF4093110250931202609346
:1083C0001302709314028091A6049091A704A091C7
:1083D000A804B091A904892B8A2B8B2B09F046C6DF
:1083E000A091480FB091490F109711F40C945A4A7C
:1083F0008090A2049090A304A090A404B090A5043F
:1084000040919E0450919F046091A0047091A1043A
:1084100084169506A606B706D8F010925E04109250
:10842000490F1092480F90913B0980913C09981791
:1084300011F40C945A4A80913C098F5F8F7080939D
:108440003C0940EDC42E47E0D42EE12CF12C1AC497
:1084500040919A0450919B0460919C0470919D04FA
:10846000481559056A057B0508F4AAC14091960490
:10847000509197046091980470919904D6960D914B
:108480001D912D913C91D9974017510762077307B1
:1084900008F077C1411551056105710549F48090D7
:1084A0005A0490905B04A0905C04B0905D0464C199
:1084B000E12CF980842E952F862F0A811B81FD8166
:1084C000EE813F8128859C80E0915617E89D912C94
:1084D000FF2730915717389D900CF11D10905817B9
:1084E000189CF00DE99F900CF11D399FF00DE89F4D
:1084F000F00D092D1F2F099DE12D332722270F9FF6
:10850000E00D311D2E1D199DE00D311D2E1D1F9FEB
:10851000300D211D032F122F099DF12C3327222707
:108520000F9FF00C311D2E1D199DF00C311D2E1DBD
:108530001F9F300D211D032F122FEE2780905A040C
:1085400090915B0480915C040090B6040E2809F4BD
:1085500083C03091B204309FE1198E089E098E09C4
:108560002091B304209FE01981089E098E09F090A4
:10857000B404F09E801891098E09319FE01981089A
:108580009E098E09219F801891098E09F19E9019EC
:108590008109099DF12C332722270F9FF00C311DF3
:1085A0002E1D199DF00C311D2E1D1F9F300D211DFC
:1085B000032F122F3091AE04309FE10D8E1C9E1DB3
:1085C0008E1D2091AF04209FE00D811C9E1D8E1DED
:1085D000F090B004F09E800C911D8E1D319FE00D37
:1085E000811C9E1D8E1D219F800C911D8E1DF19E54
:1085F000900D811D099DF12C332722270F9FF00C30
:10860000311D2E1D199DF00C311D2E1D1F9F300D8B
:10861000211D032F122F3091AA04309FE1198E08DB
:108620009E098E092091AB04209FE01981089E09C4
:108630008E09F090AC04F09E801891098E09319F4C
:10864000E01981089E098E09219F801891098E09E1
:10865000F19E9019810982C03091B204309FE10DE2
:108660008E1C9E1D8E1D2091B304209FE00D811C49
:108670009E1D8E1DF090B404F09E800C911D8E1DE9
:10868000319FE00D811C9E1D8E1D219F800C911D30
:108690008E1DF19E900D811D099DF12C33272227FF
:1086A0000F9FF00C311D2E1D199DF00C311D2E1D3C
:1086B0001F9F300D211D032F122F3091AE04309FCC
:1086C000E1198E089E098E092091AF04209FE019C0
:1086D00081089E098E09F090B004F09E80189109DF
:1086E0008E09319FE01981089E098E09219F80180B
:1086F00091098E09F19E90198109099DF12C33276A
:1087000022270F9FF00C311D2E1D199DF00C311DDD
:108710002E1D1F9F300D211D032F122F3091AA04F3
:10872000309FE10D8E1C9E1D8E1D2091AB04209F5D
:10873000E00D811C9E1D8E1DF090AC04F09E800CFF
:10874000911D8E1D319FE00D811C9E1D8E1D219F50
:10875000800C911D8E1DF19E900D811D11249C8217
:10876000F9820A831B83FD83EE833F832887912C44
:10877000992AA12CB12CA82A8DE095E121E0298B22
:1087800014C0D2968D909D90AD90BC90D597F4CFAB
:10879000B694A79497948794D988DD0CD98A0496C7
:1087A00025E18932920709F4EAC4FC01059115918B
:1087B00025913491081519052A053B0548F3DFC4B6
:1087C00040908F04509090046090910470909204B7
:1087D000481459046A047B0408F0C3C180918E04D4
:1087E000811121C0FD01EE5BFF4FE080F18002812D
:1087F000138178962081318142815381D2966D9187
:108800007D918D919C91D5970E94FEB2DD24D394E9
:10881000D0928E04E091480FF091490F82A993A95C
:10882000A4A9B5A98EC140918A0450918B0460918E
:108830008C0470918D04DA960D911D912D913C91CF
:10884000DD97401751076207730708F073C14115A0
:1088500051056105710549F480915A0490915B04BA
:10886000A0915C04B0915D046CC1F0E0E985842FB7
:10887000352F262FAA857B856C855D85BE854F8526
:108880009889B0915617B89F612D55274091571779
:10889000489F600D511D10905817189E500DB39FA2
:1088A000600D511D439F500DB29F500DA62F752F87
:1088B000A69FB12D44279927A59FB00D411D9F1F4D
:1088C000769FB00D411D9F1F759F400D911DA42FD8
:1088D000792FA69FE12D44279927A59FE00D411DE3
:1088E0009F1F769FE00D411D9F1F759F400D911D9D
:1088F000A42F792FBB2780915A0430915B042091DB
:108900005C040090B6040F2A09F483C04091B204BD
:108910004A9FB1198F0B3F0B2F0B9091B3049A9F75
:10892000B01981093F0B2F0BE091B404EA9F801925
:1089300031092F0B479FB01981093F0B2F0B979FD0
:10894000801931092F0BE79F30192109A69FE12DCE
:1089500044279927A59FE00D411D9F1F769FE00D9D
:10896000411D9F1F759F400D911DA42F792F409190
:10897000AE044A9FB10D8F1F3F1F2F1F9091AF0470
:108980009A9FB00D811D3F1F2F1FE091B004EA9FF9
:10899000800D311D2F1F479FB00D811D3F1F2F1FC1
:1089A000979F800D311D2F1FE79F300D211DA69F22
:1089B000E12D44279927A59FE00D411D9F1F769F1C
:1089C000E00D411D9F1F759F400D911DA42F792F14
:1089D0004091AA044A9FB1198F0B3F0B2F0B909126
:1089E000AB049A9FB01981093F0B2F0BE091AC04A7
:1089F000EA9F801931092F0B479FB01981093F0B5E
:108A00002F0B979F801931092F0BE79F30192109F0
:108A100082C04091B2044A9FB10D8F1F3F1F2F1F8C
:108A20009091B3049A9FB00D811D3F1F2F1FE091BD
:108A3000B404EA9F800D311D2F1F479FB00D811D8B
:108A40003F1F2F1F979F800D311D2F1FE79F300D58
:108A5000211DA69FE12D44279927A59FE00D411DCB
:108A60009F1F769FE00D411D9F1F759F400D911D1B
:108A7000A42F792F4091AE044A9FB1198F0B3F0B61
:108A80002F0B9091AF049A9FB01981093F0B2F0BC8
:108A9000E091B004EA9F801931092F0B479FB0196C
:108AA00081093F0B2F0B979F801931092F0BE79FEF
:108AB00030192109A69FE12D44279927A59FE00D94
:108AC000411D9F1F769FE00D411D9F1F759F400D0B
:108AD000911DA42F792F4091AA044A9FB10D8F1F99
:108AE0003F1F2F1F9091AB049A9FB00D811D3F1F18
:108AF0002F1FE091AC04EA9F800D311D2F1F479F6F
:108B0000B00D811D3F1F2F1F979F800D311D2F1FFF
:108B1000E79F300D211D1124E987AA877B876C8789
:108B20005D87BE874F87988B90E0932BA0E0B0E0E5
:108B3000A22B07C0A65ABF4F8D919D910D90BC915D
:108B4000A02D2DE035E141E0498BF901459155918A
:108B500065917491481759076A077B0708F499C310
:108B6000A6C3809193048823E1F0FD01E85BFF4FE9
:108B70004081518160E070E000910D0210910E0281
:108B800020910F02309110024017510762077307BE
:108B900041F01092110210921202109213021092E0
:108BA00014024091090250910A0260910B027091E7
:108BB0000C0277FF5FC0AE5ABF4FCD90DD90ED90B5
:108BC000FC908DE095E121E0FC0145915591659186
:108BD00074914C155D056E057F0550F4F694E7948D
:108BE000D794C794220F049675E18932970761F7ED
:108BF0002093950480E2C816D104E104F10428F41E
:108C000070E2C72ED12CE12CF12C90E2C91AD108C8
:108C1000E108F108C114A8E0DA06E104F10408F45F
:108C200002C4B4E0DB9EC0011124835F9E4EFC01B0
:108C3000329625913491EC2D6627E39FA001E29FA7
:108C4000410D561F0694461F561F112460E070E028
:108C5000FC0125913491C901A0E0B0E0841B950B83
:108C6000A60BB70B8093090290930A02A0930B0204
:108C7000B0930C02C0900902D0900A02E0900B025F
:108C8000F0900C028091480F9091490F892B09F0C8
:108C9000E5C10E9480B39093490F8093480F892BC0
:108CA00009F4DCC1E091480FF091490F808183FF06
:108CB0003EC085899689A789B08D8093E1179093EE
:108CC000E217A093E317B093E417818D928DA38DE3
:108CD000B48D8093E5179093E617A093E717B093B0
:108CE000E817858D968DA78DB0A18093E917909395
:108CF000EA17A093EB17B093EC1781A192A1A3A15F
:108D0000B4A18093ED179093EE17A093EF17B09353
:108D1000F01790913B0980913C09981709F4B9CF5D
:108D200080913C098F5F8F7080933C09B2CFC588DA
:108D3000D688E788F08C81E0C114D104E104F10405
:108D400009F480E0018D128D238D348D01151105FC
:108D50002105310509F08260458D568D678D70A122
:108D6000411551056105710509F0846080935E0429
:108D700010928A0410928B0410928C0410928D042D
:108D800010929604109297041092980410929904ED
:108D900085A196A1A7A1B0A580939E0490939F045E
:108DA000A093A004B093A104882499245401881AA4
:108DB000990AAA0ABB0A8092860490928704A0921C
:108DC0008804B09289048092820490928304A092D5
:108DD0008404B092850480927E0490927F04A092D5
:108DE0008004B092810480927A0490927B04A092D5
:108DF0007C04B0927D04CC0CDD1CEE1CFF1CC092E8
:108E00006A04D0926B04E0926C04F0926D04000F3F
:108E1000111F221F331F00936E0410936F042093C1
:108E2000700430937104440F551F661F771F4093E1
:108E3000720450937304609374047093750441A199
:108E400052A163A174A1440F551F661F771F409361
:108E50007604509377046093780470937904880FB4
:108E6000991FAA1FBB1F8093660490936704A09369
:108E70006804B09369041092A2041092A3041092A3
:108E8000A4041092A50482A593A5A4A5B5A58093DA
:108E90009A0490939B04A0939C04B0939D0486A590
:108EA00097A5A0A9B1A980938F0490939004A09353
:108EB0009104B093920481A580936504DF01A95BBE
:108EC000BF4F9C9190939404992339F115962D915D
:108ED0003C911197309364042093630412972D9171
:108EE0003C91119730936204209361041092110217
:108EF00010921202109213021092140212972D91E6
:108F00003C91A90160E070E040930D0250930E0285
:108F100060930F02709310020CC088248A94982CDE
:108F2000540180920D0290920E02A0920F02B09214
:108F30001002EA5BFF4F90812091590492130AC0FE
:108F40002091080230E0482F082E000C550B4217E4
:108F5000530731F090935904809308020E9450B354
:108F60000E9482BF2FEF3FEFA901209309023093A7
:108F70000A0240930B0250930C02E091480FF091CB
:108F8000490FDF01DE96ED90FD900D911C9122A915
:108F900033A944A955A9EA5AFF4F608171818281A2
:108FA00093810E94FEB210928E04E091480FF091DE
:108FB000490FEA5AFF4F80809180A280B3808DE0F4
:108FC00095E121E0FC014591559165917491481519
:108FD00059056A057B0558F4B694A794979487942D
:108FE000220F0496A9E2B5E1A817B90759F7209313
:108FF0009504B0E28B169104A104B10428F4B0E208
:109000008B2E912CA12CB12C30E2831A9108A1084F
:10901000B108811448E09406A104B10408F427C201
:1090200054E0959EC0011124835F9E4EFC01329650
:1090300025913491782D6627739FA001729F410D71
:10904000561F0694461F561F1124FC01C590D4904C
:10905000E12CF12CC41AD50AE108F108C092A6044B
:10906000D092A704E092A804F092A9040091A6046B
:109070001091A7042091A8043091A90440911102F5
:10908000509112026091130270911402F02E198B0C
:10909000F22FE32F401751076207730720F4F42ED5
:1090A000598BF62FE72F8F2D9989AF2FBE2F009761
:1090B000E1E0AE07B10520F08FEF9FEFA0E0B0E058
:1090C000081B190B2A0B3B0B0093A6041093A70453
:1090D0002093A8043093A9044F3FFFEF5F076F0769
:1090E0007F0761F0481B590B6A0B7B0B4093110201
:1090F000509312026093130270931402F89420911B
:10910000840030918500205F3F4F4A8941504A8B4F
:10911000442341F0280E391E2216330610F40C9415
:10912000213F01C019013092890020928800789473
:1091300062960FB6F894DEBF0FBECDBFDF91CF9120
:109140001F910F91FF90EF90DF90CF90BF90AF9065
:109150009F908F907F906F905F904F903F902F9057
:10916000089580910B0180958870809309010C947B
:109170002D4080910B0188708093090167C839895F
:109180003093950480E288169104A104B10428F478
:1091900030E2832E912CA12CB12C30E2831A91085D
:1091A000A108B108811488E09806A104B10420F157
:1091B000E4E09E9EC0011124835F9E4EFC01329626
:1091C00025913491F82DEE27F39F7001F29FE10C69
:1091D000FE1E0694EE1EFE1E1124FC01C590D490C6
:1091E000860120E030E0480159018E189F08A1084F
:1091F000B1087501640122C0950184013695279557
:1092000017950795F801EC7FCF01835F924FFC0122
:10921000C590D490FC01329625913491E82DE770E9
:10922000E29FC001E39F900D112423E0969587955E
:109230002A95E1F7C81AD90AE12CF12C4C0D5D1DD5
:109240006E1D7F1D4093960450939704609398047D
:10925000709399049091940480919304992309F454
:1092600073C0882309F40ECDA85BBF4F8D919C91EC
:10927000A0E0B0E040910D0250910E0260910F020B
:109280007091100284179507A607B70709F05FC011
:10929000F9CCB695A79597958795D988DD0CD98A8D
:1092A0002C5F3F4F45E12932340709F04ECC5989F4
:1092B0005093950480329105A105B10520F480E218
:1092C00090E0A0E0B0E08097A109B109811558E0D5
:1092D0009507A105B10508F443C074E0979F90017C
:1092E0001124235F3E4EF901329645915491EE27A9
:1092F000859FB001849F610D7E1F06946E1F7E1FA7
:109300001124F901C590D490E12CF12CC61AD70A8A
:10931000E108F10880918A0490918B04A0918C045B
:10932000B0918D048C0D9D1DAE1DBF1D80938A04D0
:1093300090938B04A0938C04B0938D04809194043B
:10934000811130C080919304882309F49BCC109242
:10935000110210921202109213021092140292CC77
:10936000AC01BD017695679557954795FA01EC7F5D
:109370009F01235F324FF901C590D490F9013296D5
:10938000459154918770849F9001859F300D1124E1
:10939000F3E036952795FA95E1F7C21AD30AE12C46
:1093A000F12CB8CF8989480E511C611C711C809129
:1093B000480F9091490F481459046A047B04D8F46B
:1093C00020919304222309F45DCCFC01E85BFF4F5C
:1093D00020813181A90160E070E000910D021091BF
:1093E0000E0220910F0230911002401751076207C0
:1093F000730709F447CC10921102109212021092D6
:10940000130210921402FC01E85BFF4F80819181EE
:10941000A0E0B0E080930D0290930E02A0930F02A3
:10942000B09310022FCCD701C601B695A79597959A
:109430008795FC01EC7FCF01835F924FFC01259162
:109440003491FC013296459154916C2D6770649F64
:10945000C001659F900D112463E0969587956A95EC
:10946000E1F7281B390BC901A0E0B0E0FBCBD50127
:10947000C401B695A79597958795FC01EC7FCF0120
:10948000835F924FFC01C590D490FC0132962591E8
:109490003491482D4770429FC001439F900D112485
:1094A000A3E096958795AA95E1F7C81AD90AE12C09
:1094B000F12CD4CD80EDC82E87E0D82EE12CF12CF4
:1094C000E8CBCF92DF92EF92FF92CF93DF936B01C5
:1094D0007C01EA0122E630E140E450EC0E9411F008
:1094E00087FD23C022E430E047E553E4C701B6011D
:1094F0000E946EE91816CCF0C880D980EA80FB8003
:109500002FE632E143E85AEBC701B6010E9411F0A1
:1095100087FD0BC0C1E022E430E047E553E4C7011A
:10952000B6010E946EE918160CF4C0E08C2FDF9192
:10953000CF91FF90EF90DF90CF9008950F931F93FE
:10954000CF93DF93FC01A685B7858D0100581F4F8F
:10955000E8018881998101968F779927AD014E574F
:109560005F4FEA012881398128173907D1F3E801D3
:1095700028813981A20FB31F6C93A685B785A058A7
:10958000BF4F11969C938E93A689B7892C9181E049
:1095900090E0078C02C0880F991F0A94E2F7822B93
:1095A0008C9381E081A30488F589E02D808180641B
:1095B000808381E090E0DF91CF911F910F9108951A
:1095C000FC0181A1882329F0A489B5898C9186FFAB
:1095D000FBCF11A20895FC01A485B585FD01E058DB
:1095E000FF4F208131813296808191812817390780
:1095F00079F080819181A80FB91F8C9120813181F0
:109600002F5F3F4F2F7733273183208390E00895DA
:109610008FEF9FEF0895DC011C96ED91FC911D9753
:10962000DF01A058BF4F2D913C91119712968D915B
:109630009C9111972817390739F08D919C91E80F6B
:10964000F91F808190E008958FEF9FEF0895FC014E
:1096500024853585F901E058FF4F8081918132964C
:109660002081318180589F4F821B930B60E870E00E
:109670000C94D4F00895089580E090E00895CF927E
:10968000DF92EF92FF92C0904202D0904302E090AE
:109690004402F0904502FC0180819181A281B38156
:1096A0008093420290934302A0934402B0934502F8
:1096B0000E9473CDC0924202D0924302E0924402D3
:1096C000F0924502FF90EF90DF90CF900895809147
:1096D000CC189091CD18981759F0E92FF0E0E45B81
:1096E000F74E80819F5F9F779093CD1890E008950B
:1096F0008FEF9FEF08951F920F920FB60F921124D4
:109700000BB60F922F938F939F93EF93FF9320911C
:10971000CD18E091CC1881E08E0F8F779091C60024
:10972000281729F0F0E0E45BF74E9083E82FE093F0
:10973000CC18FF91EF919F918F912F910F900BBEBD
:109740000F900FBE0F901F90189580912504909157
:109750002604009731F04AE050E060E070E00C949D
:10976000C2E660E070E0CB010895EFDF97FD0AC02C
:10977000ECDF6F3F71058105910509F02CF4E5DF01
:10978000862F089580E008958FEF08958091250435
:1097900090912604892B31F0E8DF91E0811103C01C
:1097A00090E001C091E0892F08950F931F93CF930C
:1097B0008091250490912604009711F1FC018F01FE
:1097C000C1912C2F2F7DA9F0C53411F0C536B9F702
:1097D000F801108260E070E08091250490912604E9
:1097E0000E946FE5F801C083562F472F382F292F8D
:1097F0000BC060E070E0CF911F910F910C946FE56A
:1098000050E040E030E020E0652F742F832F922F4E
:10981000CF911F910F91089581548A3108F042C071
:10982000E82FF0E04091431850914418609145189A
:109830007091461804C076956795579547958A9517
:10984000D2F7842F817040FF2FC0E75DF74E9081E3
:10985000992309F1E091D117F091D217E90FF11D89
:10986000908120ED290F2A3098F09E3211F49181D9
:109870000CC09D3211F09B3271F4918120ED290FC3
:109880002A3030F09E3239F4928190539A3018F495
:109890002E2F9F2F02C020E090E02093250490936C
:1098A0002604089580E008950895B6DF882341F0E6
:1098B00081E02091250430912604232B09F480E0D7
:1098C000089580E1E6E3F4E0ADE0B8E101900D92A7
:1098D0008A95E1F708952F923F924F925F926F928F
:1098E0007F928F929F92AF92BF92CF92DF92EF9230
:1098F000FF920F931F93CF93DF9300D01F921F927D
:10990000CDB7DEB77C018B016A0119018090360466
:1099100090903704A0903804B0903904A5019401C8
:10992000FC0160817181828193810E946EE9F1E086
:10993000FD83811112C020913A0430913B04409183
:109940003C0450913D04F8016081718182819381D2
:109950000E946EE9811101C01D82F6014080518094
:109960006280738020911502309116024091170297
:1099700050911802C301B2010E946EE9882309F4D4
:1099800053C04092150250921602609217027092D4
:10999000180220E030E040E450E46091100770913C
:1099A000110780911207909113070E94C7EE6983F7
:1099B0007A838B839C8380920D1890920E18A092CC
:1099C0000F18B092101880913A0490913B04A09126
:1099D0003C04B0913D048093111890931218A09309
:1099E0001318B0931418F60180819181A281B3817C
:1099F0008093151890931618A0931718B093181801
:109A00008091420490914304A0914404B091450494
:109A10008093191890931A18A0931B18B0931C18D0
:109A2000CE0101962CDE4DDFFD81FF2309F1609010
:109A30000C0770900D0780900E0790900F07A09074
:109A40000807B0900907C0900A07D0900B0795014E
:109A5000A601B301C4010E9411F0181614F05301BD
:109A6000640120E030E040E251E4B501C6010CC0E1
:109A700020E030E040EC5FE360911407709115073F
:109A800080911607909117070E94C7EE69837A8329
:109A90008B839C8320912404222349F0AB01BC01D9
:109AA0008DE295E10E94D2B38AE00E94188AF70104
:109AB00080819181A281B38180930D1890930E18BB
:109AC000A0930F18B0931018F80180819181A281A2
:109AD000B3818093111890931218A0931318B09328
:109AE0001418F1012081318142815381609119184C
:109AF00070911A1880911B1890911C180E94EBED20
:109B00006093191870931A1880931B1890931C185F
:109B1000CE010196B4DDD5DE0F900F900F900F901F
:109B20000F90DF91CF911F910F91FF90EF90DF90F9
:109B3000CF90BF90AF909F908F907F906F905F90ED
:109B40004F903F902F90089580E1EDE0F8E1A6E37B
:109B5000B4E001900D928A95E1F708959C0197FD7C
:109B60000EC08436910584F064E670E00E94D4F063
:109B7000CB016AE070E00E94D4F0805D06C03195B0
:109B8000219531098DE201C080E2809331042A30B1
:109B9000310564F0EAE0F0E0C901BF010E94D4F0B1
:109BA000CB01BF010E94D4F0805D01C080E28093B0
:109BB0003204C9016AE070E00E94D4F0805D8093B5
:109BC000330481E394E00895883791051CF028E779
:109BD00080E002C0282F892F2093480480934904F5
:109BE0000C940B7D2F923F924F925F926F927F92D7
:109BF0008F929F92AF92BF92CF92DF92EF92FF929D
:109C00000F931F93CF93DF93CDB7DEB7C455D10920
:109C10000FB6F894DEBF0FBECDBFECEEF7E1849136
:109C20008F010F5F1F4F882321F00E94188AF801CF
:109C3000F6CF0E9417C481110C94D25780E090E0B7
:109C4000A0E8BFE38093051890930618A093071827
:109C5000B093081880E090E0A0ECB0E4809309187D
:109C600090930A18A0930B18B0930C188DEC9CECF1
:109C7000ACE4BEE38093011890930218A0930318FC
:109C8000B093041880E090E0A8ECB1E4809328053C
:109C900090932905A0932A05B0932B058CE390E0BF
:109CA000909327058093260588EC90E090932505F6
:109CB00080932405109223058FE4F7DD882311F0AB
:109CC00074DD04C060E070E080E190E46BAF7CAFD5
:109CD0008DAF9EAF83E4E9DD882311F057DD02C02C
:109CE00083E49ADD61968FAF61978BE4DEDD882394
:109CF00011F04CDD02C08BE48FDD60968FAF609772
:109D000082E4D3DD8823E9F050DD0E942FEF7093C9
:109D10002705609326056115710599F06852710950
:109D20006536710570F0E7EBF7E184918F010F5F05
:109D30001F4F882311F40C94D2570E94188AF801FF
:109D4000F4CF8CE4B2DD882351F12FDD6B017C016F
:109D5000609301187093021880930318909304186D
:109D600020E030E0A9010E9411F087FD0AC020E048
:109D700030E040E050E4C701B6010E946EE91816D9
:109D800074F4EFE8F7E184918F010F5F1F4F882390
:109D900011F40C94D2570E94188AF801F4CF81E58F
:109DA0003BDD882309F440C080912504909126046E
:109DB000892B19F4E4E6F7E12BC0F7DC6B017C0199
:109DC0006093091870930A1880930B1890930C18DD
:109DD0002DEC3CEC4CE45DE30E9411F087FD0AC0E1
:109DE00020E030E040E751E4C701B6010E946EE98F
:109DF0001816D4F4E3E3F7E184918F010F5F1F4F4E
:109E0000882311F40C94D2570E94188AF801F4CFD9
:109E100084918F010F5F1F4F882311F40C94D25748
:109E20000E94188AF801F4CF83E53FDD882319F1F9
:109E3000BCDC4B015C012DEC3CEC4CEC5DE30E9486
:109E400011F087FD0AC020E030E040E85FE3C50183
:109E5000B4010E946EE91816ACF4ECE0F7E18491CD
:109E60008F010F5F1F4F882311F40C94D2570E946B
:109E7000188AF801F4CF5DEC852E5CEC952EA92CA8
:109E80005EE3B52E80E5C8DC882309F443C08091E9
:109E9000250490912604892B71F4E4EDF6E1849178
:109EA0008F010F5F1F4F882311F40C94D2570E942B
:109EB000188AF801F4CF809123058F5F80932305E2
:109EC00074DC6B017C0160932805709329058093F5
:109ED0002A0590932B0520E030E0A9010E9411F0A3
:109EE00087FD0AC020E030E048EC51E4C701B6012C
:109EF0000E946EE9181674F4ECEAF6E184918F0181
:109F00000F5F1F4F882311F40C94D2570E94188AB8
:109F1000F801F4CF86E4C9DC882319F146DC6B0133
:109F20007C0120E030E040E85FE30E9411F087FD13
:109F30000AC020E030E040E850E4C701B6010E94CA
:109F40006EE91816A4F4E3E8F6E184918F010F5F3F
:109F50001F4F882311F40C94D2570E94188AF801DD
:109F6000F4CFC12CD12C40EEE42E4FE3F42EA70108
:109F70009601C701B6010E94D3E99B01AC0160E0E4
:109F800070E084E490E40E94C7EE209105183091BF
:109F9000061840910718509108180E94D3E92B0128
:109FA0003C01A5019401C501B4010E94D3E9A701B8
:109FB00096010E94D3E92CEE31E548EB5DE30E9467
:109FC000C7EE9B01AC01C301B2010E94D3E96093CB
:109FD000051870930618809307189093081888E462
:109FE00064DC8823C9F0E1DB0E942FEF7093250524
:109FF00060932405655A71096437710568F0E5E5D9
:10A00000F6E184918F010F5F1F4F882309F4CAC7BF
:10A010000E94188AF801F5CF85E5FEDB8823E9F078
:10A020000E949058611571058105910511F00E94FB
:10A0300066E58091250490912604892B11F0B5DB0B
:10A0400004C060E070E088E492E460931F057093C0
:10A050002005809321059093220582E5DDDB8111A7
:10A060000DC0E1E2F6E184918F010F5F1F4F88235D
:10A0700009F498C70E94188AF801F5CF8091250449
:10A0800090912604892BA9F060DB2F967FAF6EAFED
:10A090002F97161617069CF0EDEEF5E184918F01CF
:10A0A0000F5F1F4F882309F47DC70E94188AF801AB
:10A0B000F5CF8AE190E02F969FAF8EAF2F9788E57E
:10A0C000F4DB882361F071DB2091180430911904CE
:10A0D00040911A0450911B040E94EAED08C060915F
:10A0E000360470913704809138049091390460935C
:10A0F0001B0570931C0580931D0590931E0589E533
:10A10000D4DB882361F051DB20911C0430911D04C5
:10A1100040911E0450911F040E94EAED08C0609116
:10A120003A0470913B0480913C0490913D0460930B
:10A130001705709318058093190590931A0560917F
:10A140001B0570911C0580911D0590911E0547E12E
:10A1500055E0B7D981110DC0E3ECF5E184918F0191
:10A160000F5F1F4F882309F41DC70E94188AF8014A
:10A17000F5CF84E451DB91E089270E94A69220E08C
:10A1800030E040EA50E460913E0470913F048091D9
:10A190004004909141040E946EE987FF14C0198A1F
:10A1A0001A8A1B8A1C8A80E090E0A0EAB0E48983C6
:10A1B0009A83AB83BC83BE016F5E7F4FCE01019655
:10A1C0000E94F9C3C1DCACD76B017C01A8E8CA0EC0
:10A1D000A3E1DA1EE11CF11C809126059091270570
:10A1E000F3DC6091260570912705072E000C880B83
:10A1F000990B0E9474E99B01AC0160914A04709133
:10A200004B0480914C0490914D040E94EAED4B0167
:10A210005C0120E030E0A9010E9411F087FF04C03A
:10A22000B7FAB094B7F8B09420E030E040E450E4DE
:10A23000C501B4010E9411F01816F4F471D7DC01C5
:10A24000CB018C199D09AE09BF09B7FD0EC068D7B7
:10A250006B017C01B8E8CB0EB3E1DB1EE11CF11C05
:10A260000E94517C8AE00E94188A0E945BAA809119
:10A27000CC188093CD18B5CF8091240590912505F9
:10A280000E94B77B6091240570912505072E000C74
:10A29000880B990B0E9474E99B01AC0160915004FA
:10A2A0007091510480915204909153040E94EAED00
:10A2B0004B015C0120E030E0A9010E9411F087FF12
:10A2C00004C0B7FAB094B7F8B09420E030E040E4AE
:10A2D00050E4C501B4010E9411F01816F4F420D71F
:10A2E000DC01CB018C199D09AE09BF09B7FD0EC079
:10A2F00017D76B017C01E8E8CE0EE3E1DE1EE11C1E
:10A30000F11C0E94517C8AE00E94188A0E945BAA7C
:10A310008091CC188093CD18B5CF10924204109242
:10A32000430410924404109245040E94C5C28091D7
:10A330002305882399F1C5DA209128053091290554
:10A3400040912A0550912B056091191870911A18A7
:10A3500080911B1890911C180E94EBED60931918C6
:10A3600070931A1880931B1890931C1820E030E00B
:10A3700040E751E46091140770911507809116072A
:10A38000909117070E94C7EE69837A838B839C8321
:10A39000CE01019674D995DA0E94D2C080E2E7EF2F
:10A3A000F4E0DF01282F1D922A95E9F7E7EDF4E0AC
:10A3B000DF01282F1D922A95E9F7E7EBF4E0DF0192
:10A3C0001D928A95E9F77DDA809101189091021823
:10A3D000A0910318B0910418809315189093161843
:10A3E000A0931718B093181819821A821B821C8226
:10A3F0009E012F5F3F4F45E158E161E178E18DE03B
:10A4000098E169DA9E01255C3F4F45E158E161E141
:10A4100078E18DE098E15FDA6196BFAD6197BB238B
:10A4200029F06AE374E086E394E004C067E175E034
:10A430008BE195E00E94ABDB298F3A8F4B8F5C8FCD
:10A440006D8F7E8F3FAF2D962FAF2D972D96EFAD51
:10A450002D97E7FD81C4FFADF7FD7EC424E0E20245
:10A46000F0011124EB57F64F4080518062807380D9
:10A470003FAD84E03802F0011124EF58F64FD08050
:10A48000C180328023808D2D9C2DA32DB22D8FABCA
:10A4900098AFA9AFBAAFAE01495C5F4FB201C3013B
:10A4A00010D8882309F45CC420E030E040EA50E48E
:10A4B000B201C3010E94EBEDF62E072F182FE92EF3
:10A4C000862F902FA12FBE2D8BAB9CABADABBEAB1F
:10A4D0008D2D9C2DA32DB22D8FA798ABA9ABBAAB18
:10A4E0002D969FAD2D97911152C0AFADA11105C012
:10A4F0005F2D402F312F2E2D04C0542D452D362D8C
:10A50000272D852F942FA32FB22F8BAB9CABADABF8
:10A51000BEABBFADB43034F4F42C052D162DE72CB2
:10A52000BB2369F020E030E040EA50E46D2D7C2D43
:10A53000832D922D0E94EAED362F272F03C096011E
:10A54000832D922D432F522FBC014FA758AB69ABDF
:10A550007AABEFADE4300CF0A7C020E030E040EA89
:10A5600050E46D2D7C2D832D922D0E94EBED2196D4
:10A570006FAF219723967FAF239725968FAF2597AF
:10A5800027969FAF2797FFADF11185C099C02D96F3
:10A590002FAD2D9724300CF453C03FAD34305CF018
:10A5A00020E030E040EA50E4B201C3010E94EAED4D
:10A5B000362F272F03C0342D252DC301432F522FB3
:10A5C000BC014BAB5CAB6DAB7EAB8FAD8111E1C41D
:10A5D00020E030E040EA50E4B201C3010E94EAED1D
:10A5E000F62E072F182FE92E20E030E040EA50E445
:10A5F0006D2D7C2D832D922D0E94EBED6FA778ABF6
:10A6000089AB9AAB9FAD992309F44EC020E030E0AE
:10A6100040EA50E46D2D7C2D832D922D0E94EAEDB1
:10A6200021966FAF219723967FAF239725968FAF03
:10A63000259727969FAF2797AFADA43064F140C010
:10A64000BFADB1110DC020E030E040EA50E4B201EE
:10A65000C3010E94EAEDF62E072F182FE92E0FC036
:10A66000EFADE430B4F120E030E040EA50E4B20174
:10A67000C3010E94EAED6BAB7CAB8DAB9EAB219628
:10A68000DFAE21972396CFAE239725963FAE259731
:10A6900027962FAE279732ED832E33E5932E3BE797
:10A6A000A32E31E4B32E29C02196DFAE2197239645
:10A6B000CFAE239725963FAE259727962FAE2797A7
:10A6C00022ED822E23E5922E2BEFA22E20E4B22E35
:10A6D00014C02196DFAE21972396CFAE23972596FF
:10A6E0003FAE259727962FAE279792ED892E93E5BB
:10A6F000992E9BEFA92E91E4B92E8BA99CA9ADA907
:10A70000BEA92C968CAF9DAFAEAFBFAF2C979C016E
:10A71000AD01B201C3010E94EAED698B7A8B8B8B8C
:10A720009C8B4FA458A869A87AA8A30192016D2D0B
:10A730007C2D832D922D0E94EAED6D8B7E8B8F8B6D
:10A74000988F2C962CAD3DAD4EAD5FAD2C976091A2
:10A7500036047091370480913804909139040E9436
:10A76000EAED2C966CAF7DAF8EAF9FAF2C97A30117
:10A77000920160913A0470913B0480913C04909165
:10A780003D040E94EAED2B013C018F2D902FA12F5B
:10A79000BE2D89839A83AB83BC8321968FAD21978D
:10A7A00023969FAD23972596AFAD25972796BFADEE
:10A7B00027978D839E83AF83B887809101189091EE
:10A7C0000218A0910318B091041889879A87AB8763
:10A7D000BC872DEC3CEC4CEC5CE3C501B4010E9461
:10A7E000D3E920910518309106184091071850912F
:10A7F00008180E94D3E9209142043091430440910B
:10A800004404509145040E94EBED6D877E878F874D
:10A81000988B2C962CAD3DAD4EAD5FAD2C97CA01FB
:10A82000B9010E94D3E96B017C01A3019201C3012C
:10A83000B2010E94D3E99B01AC01C701B6010E949D
:10A84000EBED20E030E040E050E40E9411F01816FB
:10A850000CF046C00E94D2C01BA21CA21DA21EA2C8
:10A8600020E030E040E05FE360913E0470913F04FF
:10A8700080914004909141040E94EBED6F8F78A38A
:10A8800089A39AA39E012D5D3F4FAE01415E5F4FAC
:10A890006AE374E086E394E01ED81BA21CA21DA20A
:10A8A0001EA220E030E040E05FE36091011870916B
:10A8B000021880910318909104180E94EBED6F8F9D
:10A8C00078A389A39AA39E012D5D3F4FAE01415EFF
:10A8D0005F4FBE01615D7F4FCE01C3960E946B4CFE
:10A8E0001F8E18A219A21AA29E01215E3F4F41E0BD
:10A8F00058E1BE01615D7F4FCE01C3960E946B4C53
:10A900000E94FEC040904202509043026090440278
:10A9100070904502E0900C07F0900D0700910E0733
:10A9200010910F07A0900807B0900907C0900A0780
:10A93000D0900B079501A601B701C8010E9411F044
:10A94000181614F47501860120E030E040E251E46D
:10A95000B701C8010E94C7EE6093420270934302A0
:10A96000809344029093450240E0BE016F5E7F4FAA
:10A97000CE0101960E94B0AE409242025092430234
:10A9800060924402709245020E94614CA5E8B9E0D1
:10A990002496BFAFAEAF249722961FAE1EAE22976D
:10A9A00001E010E021960FAC219702C0000F111FAB
:10A9B0000A94E2F72296EEADFFAD229731962296E9
:10A9C000FFAFEEAF229721E030E021960FAC219748
:10A9D00002C0220F331F0A94E2F763963FAF2EAFF7
:10A9E000639787EB282E84E0382E87EF94E02A9631
:10A9F0009FAF8EAF2A97A7EDB4E02896BFAFAEAF5A
:10AA00002897E1E7F9E02696FFAFEEAF26972A9662
:10AA10002EAD3FAD2A9765963FAF2EAF6597D90112
:10AA20008D919C919C0120233123232B09F4ADC0EF
:10AA30006396EEADFFAD63978E239F23892B09F4B8
:10AA4000A4C02896AEADBFAD28978D919C91802370
:10AA50009123892B09F099C020E030E040E050E4D8
:10AA60002496AEADBFAD24976D917D918D919C9153
:10AA70000E94EBED6B017C0120E030E040E050E40F
:10AA80002496EEADFFAD2497648175818681978110
:10AA90000E94EAED4B015C0120E030E040E050EC28
:10AAA000C701B6010E946EE987FD70C120E030E069
:10AAB00046E553E4C701B6010E9411F0181634F4BC
:10AAC000C12CD12CB6E5EB2EB3E4FB2ECBA6DCA635
:10AAD000EDA6FEA62696AEADBFAD26974D905D9035
:10AAE0006D907C9020E030E040E85FE3C301B2016C
:10AAF0000E946EE987FD50C120E030E046E553E456
:10AB0000C301B2010E9411F0181634F4412C512CEB
:10AB1000F6E56F2EF3E47F2E4F8E58A269A27AA23B
:10AB20004FA258A669A67AA620E030E040E050EC9B
:10AB3000C501B4010E946EE987FD35C120E030E017
:10AB400046E553E4C501B4010E9411F0181634F42F
:10AB5000812C912C76E5A72E73E4B72E8BA29CA2B4
:10AB6000ADA2BEA2AE01495D5F4FC701B6010E9412
:10AB7000614A81111EC12896EEADFFAD28978081F4
:10AB80009181802B912B918380832A962EAD3FADAE
:10AB90002A972E5F3F4F2A963FAF2EAF2A97659692
:10ABA000AEADBFAD65978D919C9180239123892B8C
:10ABB00009F4A6C0F9018081918180239123892B1A
:10ABC00009F49EC0F1018081918180239123892B1A
:10ABD00009F096C020E030E040E050E42696AEADAB
:10ABE000BFAD26976D917D918D919C910E94EBED6B
:10ABF0002B013C0120E030E040E050E42696EEAD31
:10AC0000FFAD269764817581868197810E94EAED68
:10AC10004B015C012496AEADBFAD2497CD90DD9085
:10AC2000ED90FC9020E030E040E050ECC701B60130
:10AC30000E946EE987FDFDC020E030E046E553E468
:10AC4000C701B6010E9411F0181634F4C12CD12CA2
:10AC500056E5E52E53E4F52ECBA2DCA2EDA2FEA232
:10AC6000CBA6DCA6EDA6FEA620E030E040E85FE340
:10AC7000C301B2010E946EE987FDE1C020E030E02F
:10AC800046E553E4C301B2010E9411F0181634F4F2
:10AC9000412C512C36E5632E33E4732E4FA258A677
:10ACA00069A67AA620E030E040E85FE3C501B40180
:10ACB0000E946EE987FDCAC020E030E046E553E41B
:10ACC000C501B4010E9411F0181634F4812C912CA6
:10ACD00096E5A92E93E4B92E8F8E98A2A9A2BAA2C6
:10ACE000AE01495D5F4FC701B6010E94614A811103
:10ACF000B4C0F10180819181802B912B918380835D
:10AD0000F2E02F0E311C28962EAD3FAD28972E5F16
:10AD10003F4F28963FAF2EAF289726968EAD9FAD1A
:10AD20002697049626969FAF8EAF269791EC29160C
:10AD300094E0390609F06BCE2496AEADBFAD2497F2
:10AD400014962496BFAFAEAF24972296EEADFFAD1A
:10AD50002297359709F024CE8091CC188093CD1896
:10AD60002F962EAD3FAD2F97215031092F963FAF33
:10AD70002EAF2F97232B09F4B0C02D963FAD2D9702
:10AD800037FDABC08FAD87FF47CBA7C0C12CD12CFF
:10AD9000E12CA0ECFA2E9ACE412C512CE0E86E2E3C
:10ADA000EFE37E2EB9CE812C912CA12C60ECB62E37
:10ADB000D5CEAE01415E5F4FC501B4010E94614A2C
:10ADC000882309F4D8CE80912404882321F1B70187
:10ADD000A6018DE995E10E94D2B34FA158A569A5BE
:10ADE0007AA587E995E10E94D2B34BA15CA16DA140
:10ADF0007EA18DE895E10E94D2B34F8D58A169A143
:10AE00007AA187E895E10E94D2B389E20E94188A6C
:10AE10008AE00E94188A9E01215E3F4FAE014D5D7F
:10AE20005F4FBE01695D7F4FCE018B960E942EC1A0
:10AE3000A2CEC12CD12CE12C40ECF42E0DCF412C14
:10AE4000512C20E8622E2FE3722E28CF812C912CDA
:10AE500080E8A82E8FE3B82E3FCFAE01415E5F4F52
:10AE6000C701B6010E94614A882309F442CF80914C
:10AE70002404882321F1B701A60183E695E10E940D
:10AE8000D2B34FA158A569A57AA58DE595E10E9499
:10AE9000D2B34BA15CA16DA17EA183E595E10E9497
:10AEA000D2B34F8D58A169A17AA18DE495E10E949A
:10AEB000D2B389E20E94188A8AE00E94188A9E0111
:10AEC000215E3F4FAE014D5D5F4FBE01695D7F4F1B
:10AED000CE018B960E942EC10CCF0E94D2C080E082
:10AEE00090E0A0EAB0E48093151890931618A09310
:10AEF0001718B093181819821A821B821C829E019F
:10AF00002F5F3F4F45E158E161E178E18DE098E145
:10AF10000E946B4C80911B0590911C05A0911D0512
:10AF2000B0911E0580930D1890930E18A0930F18E2
:10AF3000B09310188091170590911805A0911905EC
:10AF4000B0911A058093111890931218A0931318BA
:10AF5000B093141819821A821B821C829E012F5FE3
:10AF60003F4F45E158E161E178E18DE098E10E94D1
:10AF70006B4C6096FFAD6097F11114C010924904BC
:10AF8000109248040E940B7D80E090E00E94B77B05
:10AF900009C02FADF42C052D162DE72C24300CF014
:10AFA00035CB22CBCC5ADF4F0FB6F894DEBF0FBEA5
:10AFB000CDBFDF91CF911F910F91FF90EF90DF9068
:10AFC000CF90BF90AF909F908F907F906F905F9049
:10AFD0004F903F902F9008951F920F920FB60F92AF
:10AFE00011240BB60F922F933F938F939F93EF9360
:10AFF000FF9320919A0E30919B0E80919C0E909120
:10B000009D0E2817390731F4809131018F7D80938F
:10B01000310114C0E0919C0EF0919D0EE65EF14F5F
:10B02000208180919C0E90919D0E01968F7799279B
:10B0300090939D0E80939C0E20933601FF91EF918B
:10B040009F918F913F912F910F900BBE0F900FBE4C
:10B050000F901F9018951F920F920FB60F92112408
:10B060000BB60F922F934F935F938F939F93EF9312
:10B07000FF938091300182FD1CC0209136018091A8
:10B080001E0F90911F0F4091200F5091210F01969C
:10B090008F7799274817590771F0E0911E0FF091AB
:10B0A0001F0FE256F14F208390931F0F80931E0FC6
:10B0B00002C080913601FF91EF919F918F915F9136
:10B0C0004F912F910F900BBE0F900FBE0F901F90BE
:10B0D00018950E94FBF03FB7F8948091E406909198
:10B0E000E506A091E606B091E70626B5A89B05C047
:10B0F0002F3F19F00196A11DB11D3FBFBA2FA92FF7
:10B10000982F8827820F911DA11DB11DBC01CD0173
:10B1100042E0660F771F881F991F4A95D1F708955F
:10B120002FB7F8946091E0067091E1068091E206F5
:10B130009091E3062FBF08951F920F920FB60F92C2
:10B1400011242F933F938F939F93AF93BF9380913D
:10B15000E0069091E106A091E206B091E3063091FD
:10B16000DF0623E0230F2D3720F40196A11DB11D2A
:10B1700005C026E8230F0296A11DB11D2093DF060E
:10B180008093E0069093E106A093E206B093E30675
:10B190008091E4069091E506A091E606B091E7065D
:10B1A0000196A11DB11D8093E4069093E506A0933E
:10B1B000E606B093E706BF91AF919F918F913F91C3
:10B1C0002F910F900FBE0F901F9018951F920F9206
:10B1D0000FB60F9211240BB60F922F933F934F93FC
:10B1E0005F936F937F938F939F93AF93BF93EF93EF
:10B1F000FF9380912F0590913005A0913105B0917A
:10B200003205892B8A2B8B2B59F190912E05E091D9
:10B210002C05F0912D0580818927808380912F0551
:10B2200090913005A0913105B0913205181619069C
:10B230001A061B060CF056C080912F059091300520
:10B24000A0913105B09132050197A109B109809310
:10B250002F0590933005A0933105B093320542C07D
:10B2600080911902E9E1F8E1E4919FEF90931902CE
:10B27000E230C9F050F4EE2399F0E13081F590917D
:10B280006F009D7F90936F002AC0E43019F1E0F0C9
:10B29000E53029F5909173009D7F909373001FC056
:10B2A00010926E001CC0909170009D7F9093700072
:10B2B00091E09093B0009091B100987F946090934A
:10B2C000B1001092B3000BC0909171009D7F9093DC
:10B2D000710005C0909172009D7F9093720060E0B4
:10B2E0000E948DC5FF91EF91BF91AF919F918F917A
:10B2F0007F916F915F914F913F912F910F900BBE76
:10B300000F900FBE0F901F9018952F923F924F9263
:10B310005F926F927F928F929F92AF92BF92CF92E5
:10B32000DF92EF92FF920F931F93CF93DF93CDB7EE
:10B33000DEB7C857D1090FB6F894DEBF0FBECDBF38
:10B34000E091820FF091830FEF2B11F00C94456286
:10B350002896DFAECEAE28976E2C79016A015B018C
:10B36000FC0120813181428153816C962CAF3DAF2D
:10B370004EAF5FAF6C972091F1173091F21740916B
:10B38000F3175091F4176C966CAD7DAD8EAD9FADFB
:10B390006C970E94D3E90E941CF0E0966CAF7DAFE1
:10B3A0008EAF9FAFE097D5018D919D910D90BC918F
:10B3B000A02DA0968CAF9DAFAEAFBFAFA097209150
:10B3C000F5173091F6174091F7175091F817BC0117
:10B3D000CD010E94D3E90E941CF0E4966CAF7DAFD2
:10B3E0008EAF9FAFE497D6012D913D914D915C9129
:10B3F000A4962CAF3DAF4EAF5FAFA4972091F91745
:10B400003091FA174091FB175091FC17A4966CAD40
:10B410007DAD8EAD9FADA4970E94D3E90E941CF034
:10B42000E8966CAF7DAF8EAF9FAFE897D7012D91B7
:10B430003D914D915C9122962CAF3DAF4EAF5FAFE9
:10B4400022972091FD173091FE174091FF175091E0
:10B45000001822966CAD7DAD8EAD9FAD22970E94F7
:10B46000D3E90E941CF060966CAF7DAF8EAF9FAFAA
:10B4700060978091250783FF1CC060962CAD3DAD81
:10B480004EAD5FAD609720936D0930936E09409388
:10B490006F095093700922968CAD9DADAEADBFADD6
:10B4A000229780935D0990935E09A0935F09B09302
:10B4B0006009D801BC91B9A7F801F181F9ABD801B5
:10B4C0001296BC91BEABF801F381FAAF80913B09B3
:10B4D00090913C09891B8F708F3019F40E945BAAF0
:10B4E000F5CF00913B09E9960FAFE99780913B09B1
:10B4F000082F10E01CA30BA38091610990916209B1
:10B50000A0916309B0916409E0968CAC9DACAEAC9F
:10B51000BFACE097881A990AAA0ABB0A809165090C
:10B5200090916609A0916709B0916809E4962CACE6
:10B530003DAC4EAC5FACE497281A390A4A0A5B0A64
:10B540008091690990916A09A0916B09B0916C0989
:10B55000E8962CAD3DAD4EAD5FADE897281B390B9D
:10B560004A0B5B0B2DA33EA34FA358A780916D09F7
:10B5700090916E09A0916F09B091700960960CAD21
:10B580001DAD2EAD3FAD6097081B190B2A0B3B0B71
:10B590000DA71EA72FA738AB012B022B032B09F4F5
:10B5A000BCC08091240781114BC060915004709100
:10B5B000510480915204909153040E942FEF2091E6
:10B5C000250230912602621773070CF039C060968D
:10B5D0002CAD3DAD4EAD5FAD609720936D093093BE
:10B5E0006E0940936F095093700922968CAD9DAD02
:10B5F000AEADBFAD229780935D0990935E09A09395
:10B600005F09B0936009E3E3FAE184918F010F5F72
:10B610001F4F811103C0EDE8F9E104C00E94188AB0
:10B62000F801F3CF84918F010F5F1F4F882321F022
:10B630000E94188AF801F6CF1DA61EA61FA618AAFA
:10B6400094E0699E800111240F5D1D4F6DA57EA5BC
:10B650008FA598A90E9474E9D8012D913D914D9133
:10B660005C910E94D3E96B017C0120E030E0A901EC
:10B670000E9411F087FF04C0F7FAF094F7F8F094F5
:10B680006091FD177091FE178091FF17909100183F
:10B690000E942FEF9B01AC01A8ECB0E00E94CBED23
:10B6A0000E9474E9A70196010E946EE987FF39C0E4
:10B6B00060960CAD1DAD2EAD3FAD609700936D094A
:10B6C00010936E0920936F093093700922962CAD68
:10B6D0003DAD4EAD5FAD229720935D0930935E097D
:10B6E00040935F0950936009E3E3FAE184918F018D
:10B6F0000F5F1F4F811103C0EEE6F9E104C00E9405
:10B70000188AF801F3CF84918F010F5F1F4F8823B0
:10B7100021F00E94188AF801F6CF1DA61EA61FA6CA
:10B7200018AAD501C4018827B7FD83959927AA27B0
:10B73000BB27782E57FE03C0382F3260732E8DA1A1
:10B740009EA1AFA1B8A5B7FF03C0972D9460792E35
:10B750000DA51EA52FA538A937FF03C0172D18600A
:10B76000712E24E0629E800111240F5D1D4F6DA596
:10B770007EA58FA598A90E9474E9D8012D913D91CD
:10B780004D915C910E94D3E96B017C0120E030E097
:10B79000A9010E9411F087FF04C0C701B6019058AB
:10B7A00002C0C701B60120E030E040E05FE30E9444
:10B7B000EBED0E9434EF6AAB7BAB8CAB9DAB88E6C4
:10B7C0000BA11CA1809FF001819FF00D1124EA5272
:10B7D000FF4E1082EA5BFF4F7082B501A401B7FEF5
:10B7E00007C044275527BA01481959096A097B0936
:10B7F00088E60BA11CA1809FF001819FF00D112410
:10B80000EA52FF4E458B568B678B708F2C962CAE71
:10B810003DAE4EAE5FAE2C9757FE0DC088279927E0
:10B82000DC0182199309A409B5092C968CAF9DAF50
:10B83000AEAFBFAF2C9728E60BA11CA1209FF00153
:10B84000219FF00D1124EA52FF4E2C968CAD9DAD38
:10B85000AEADBFAD2C97818F928FA38FB48F0DA10A
:10B860001EA12FA138A537FF07C030952095109550
:10B8700001951F4F2F4F3F4FE8E67E2EABA1BCA195
:10B880007A9EF0017B9EF00D1124EA52FF4E058F47
:10B89000168F278F30A38AA99BA9ACA9BDA981A324
:10B8A00092A3A3A3B4A323964FAF2397752EF62F8D
:10B8B000E72F2C968CAD9DADAEADBFAD2C97481744
:10B8C00059076A077B0778F429969FAD2997239635
:10B8D0009FAF23972A967FAC2A972B96FFAD2B9785
:10B8E0002C96EFAD2C9723968FAD2397972DAF2FE6
:10B8F000BE2F80179107A207B30710F4D901C80122
:10B900000AA91BA92CA93DA980179107A207B30773
:10B9100010F4D901C80128E60BA11CA1209FF00159
:10B92000219FF00D1124EA52FF4E85A396A3A7A3F1
:10B93000B0A70697A105B10508F4A0C5DF01AE596F
:10B94000BF4F80914604909147048D939C9361A6CC
:10B95000452B462B472B09F05F9888E60BA11CA1CD
:10B96000809FF001819FF00D1124EA52FF4E818DDE
:10B97000928DA38DB48D892B8A2B8B2B11F08A98F5
:10B98000479888E60BA11CA1809FF001819FF00DD4
:10B990001124EA52FF4E858D968DA78DB0A1892B7B
:10B9A0008A2B8B2B31F080910801817080930601E6
:10B9B00047982AA93BA94CA95DA9232B242B252B09
:10B9C00009F465C580912A07882319F08150809376
:10B9D0002A07611004C0129880E280932A076090C1
:10B9E00020077090210700912207109123079301EF
:10B9F000A80169A579A98EA99AAD0E946EE987FF71
:10BA000004C069A679AA0EAB1AAFC501B4010E94A1
:10BA100074E92091C2103091C3104091C41050912C
:10BA2000C5100E94D3E926966CAF7DAF8EAF9FAF55
:10BA30002697698B7A8B8B8B9C8BC201B1010E94FC
:10BA400074E92091C6103091C7104091C8105091F0
:10BA5000C9100E94D3E92B013C016D8B7E8B8F8B2B
:10BA6000988F6DA17EA18FA198A50E9474E9209165
:10BA7000CA103091CB104091CC105091CD100E9443
:10BA8000D3E94B015C01698F7A8F8B8F9C8F20915A
:10BA9000CE103091CF104091D0105091D110C701ED
:10BAA000B6010E94D3E96B017C016D8F7E8F8F8F71
:10BAB00098A388E60BA11CA1809FF001819FF00D47
:10BAC0001124EA52FF4E258936894789508D2DA3CE
:10BAD0003EA34FA358A7263031054105510508F470
:10BAE000DFC42896AEADBFAD2897CD90DD90ED9028
:10BAF000FC9020E030E0A901C701B6010E946EE988
:10BB00008111EDC426962CAD3DAD4EAD5FAD2697AF
:10BB1000CA01B9010E94D3E96B017C01A301920122
:10BB2000C301B2010E94D3E99B01AC01C701B60178
:10BB30000E94EBED6B017C01A5019401C501B401EC
:10BB40000E94D3E99B01AC01C701B6010E94EBED55
:10BB50000E9456F028E60BA11CA1209FF001219F16
:10BB6000F00D1124EA52FF4E658776878787908B08
:10BB700088E60BA11CA1809FF001819FF00D11248C
:10BB8000EA52FF4E4584568467847088A30192016F
:10BB900060E070E080E89FE30E94C7EE64966CAFBF
:10BBA0007DAF8EAF9FAF649729A539A94EA95AAD35
:10BBB0000E94D3E94B015C0180913B0990913909C6
:10BBC000891B8F7027968FAF2797A501940160E09E
:10BBD00074E284E799E40E94C7EE0E941CF06B01B6
:10BBE0007C0127968FAD27978250863008F486C453
:10BBF000A5019401C301B2010E94D3E99B01AC01EC
:10BC00000E94D3E968966CAF7DAF8EAF9FAF689707
:10BC100088E6ABA1BCA18A9F80018B9F100D1124E7
:10BC20000A521F4E68962CAD3DAD4EAD5FAD689784
:10BC3000D80111962D933D934D935C93149795964F
:10BC40002D913D914D915C9198972EAB3FAB48AFB4
:10BC500059AFCA01B9010E9472E96AAF7BAF8CAFDC
:10BC60009DAF9B01AC01C501B4010E94D3E90E94C4
:10BC7000B1EE0E9434EFA8966CAF7DAF8EAF9FAF50
:10BC8000A897F801EE5AFF4F6083718382839383F4
:10BC90008E010F5E1F4F2A961FAF0EAF2A970051DD
:10BCA000110924961FAF0EAF249708E017E0AC9659
:10BCB0001FAF0EAFAC978E010F5D1F4F1AA309A3E4
:10BCC00024960EAD1FAD2497AA961FAF0EAFAA976C
:10BCD000312C212C10E819A70FE309AB2A96AEAD41
:10BCE000BFAD2A972D913D914D915D912A96BFAFA1
:10BCF000AEAF2A97C501B4010E94D3E96B017C0164
:10BD0000AA96EEADFFADAA9761937193819391933B
:10BD1000AA96FFAFEEAFAA9720E030E0A9010E94FB
:10BD200011F087FF04C0F7FAF094F7F8F094AC969E
:10BD3000AEADBFADAC974D905D906D907D90AC96E3
:10BD4000BFAFAEAFAC97A7019601C301B2010E948D
:10BD50006EE987FD0DC409A11AA12A962EAD3FAD4B
:10BD60002A970217130709F0B9CF20E030E040E826
:10BD70005FE3632D722D89A599A90E946EE987FF63
:10BD800058C07E0131E1E30EF11C24960EAD1FADCB
:10BD90002497232D322D49A559A9D8016D917D9164
:10BDA0008D919C910E94D3E9F801619371938193E5
:10BDB00091938F01EE16FF0661F728E60BA11CA1F7
:10BDC000209FC001219F900D11249C012A523F4EBB
:10BDD000790189010E5A1F4FA8966CAD7DAD8EADCD
:10BDE0009FADA8970E9472E9232D322D49A559A92C
:10BDF0000E94D3E90E9434EFD8016D937D938D9317
:10BE00009C931397232D322D49A559A9632D722D8B
:10BE100089A599A90E94D3E968962CAD3DAD4EAD98
:10BE20005FAD68970E94D3E9F701618372838383D2
:10BE300094832AAD3BAD4CAD5DAD64966CAD7DADEC
:10BE40008EAD9FAD64970E94D3E969A77AA78BA7AF
:10BE50009CA70DA11EA12FA138A5012B022B032BFE
:10BE600009F09EC388E62BA13CA1829F8001839F9D
:10BE7000100D11240A521F4EF801818D928DA38D51
:10BE8000B48D892B8A2B8B2B09F08AC3858D968DD7
:10BE9000A78DB0A1892B8A2B8B2B09F081C3209110
:10BEA000040730910507409106075091070769A5DF
:10BEB0007AA58BA59CA50E94D3E90E94B1EE0E94B1
:10BEC00034EF2B013C01F801E95BFF4F108288E65B
:10BED0002BA13CA1829F8001839F100D11240A5247
:10BEE0001F4EF801E25AFF4F4082518262827382F4
:10BEF000C301B2010E9472E929A53AA54BA55CA530
:10BF00000E94C7EE6AAF7BAF8CAF9DAFD801519650
:10BF10006D937D938D939C935497F801E95BFF4F4C
:10BF20008081882381F17801B8E4EB0EF11C37960B
:10BF30002091F8063091F9064091FA065091FB06DF
:10BF400060817181828193810E94D3E92AAD3BADEA
:10BF50004CAD5DAD0E94D3E92091FD173091FE17E5
:10BF60004091FF17509100180E94D3E99B01AC014A
:10BF700060E074E284EF99E40E94C7EE0E9434EF1F
:10BF8000F7017183608388E60BA11CA1809FF001FB
:10BF9000819FF00D1124EA52FF4E218132814381AD
:10BFA00054812C962CAF3DAF4EAF5FAF2C97CA019A
:10BFB000B9010E9456F0362E272E8C0148EE56E02D
:10BFC00062965FAF4EAF62973E0151E1650E711C04
:10BFD00088EE96E09FAB8EAB24964EAC5FAC249778
:10BFE0003DA62DA209A719AB1AAAD201CD90DD90CA
:10BFF000ED90FD902D0120E030E0A901C701B601D0
:10C000000E9411F087FF04C0F7FAF094F7F8F0945B
:10C01000EEA9FFA981909190A190B190FFABEEABFA
:10C02000A7019601C501B4010E946EE987FDD8C53C
:10C0300064147504D1F627965FAD2797552309F44C
:10C0400048C6C0903D09D0903E09E0903F09F0906D
:10C0500040092DEB37E346E855E3C701B6010E94DE
:10C060006EE987FD36C6C701B6010E9456F06B0126
:10C070007C019B01AC01632D722DC8010E946EE909
:10C0800087FD03C03C2C2D2C87019601A701632D51
:10C09000722DC8010E94C7EE68966CAF7DAF8EAF5F
:10C0A0009FAF689781E499E028969FAF8EAF28975D
:10C0B00020E030E040E85FE32AAB3BAB4CAB5DAB4C
:10C0C0001EAA2896AEADBFAD28972D913D914D91FA
:10C0D0005D912896BFAFAEAF289768966CAD7DADE9
:10C0E0008EAD9FAD68970E94D3E94B015C01249609
:10C0F000EEADFFAD2497C190D190E190F1902496E0
:10C10000FFAFEEAF2497FEA9FF2391F02AA93BA928
:10C110004CA95DA90E94D3E94B015C012AA93BA966
:10C120004CA95DA9C701B6010E94D3E96B017C014E
:10C13000A7019601C501B4010E9411F020E030E092
:10C14000A90118160CF092C5C701B6010E9411F0A2
:10C1500018160CF486C520E030E0A901C501B40131
:10C160000E946EE987FD7DC52601370177FA70943C
:10C1700077F87094A3019201C501B4010E9411F0F7
:10C18000181614F4240135016296AEADBFAD629766
:10C19000CD90DD90ED90FD906296BFAFAEAF62970F
:10C1A000A3019201C701B6010E946EE987FF15C085
:10C1B000A3019201C701B6010E94C7EE9B01AC0129
:10C1C0006AA97BA98CA99DA90E94D3E96AAB7BAB24
:10C1D0008CAB9DABBEA9BF5FBEABE1E5F9E0289695
:10C1E0002EAD3FAD2897E217F30709F06ACF3EA9BD
:10C1F000332361F02AA93BA94CA95DA9632D722DB7
:10C20000C8010E94D3E9362E272E8C0124EA30E79C
:10C210004DE75FE3632D722DC8010E94D3E96B01E6
:10C220007C012091260730912707409128075091E3
:10C2300029070E946EE987FD42C58DA59DA1A9A58C
:10C24000B9A98093260790932707A0932807B09356
:10C25000290728E64BA15CA1249FC001259F900DD2
:10C260001124DC01AA52BF4E7D01232D322DA801DD
:10C27000632D722DC8010E94D3E9F701618772878F
:10C28000838794876AAD7BAD8CAD9DAD90589B0143
:10C29000AC010E94EBEDD7011D962D913D914D9182
:10C2A0005C9150970E94D3E99B01AC016BE077ED64
:10C2B00083E29BE30E94EAED9B01AC018BE097EDEA
:10C2C000A3E2BBE3F70185839683A783B087108140
:10C2D0002C966CAD7DAD8EAD9FAD2C970E946EE916
:10C2E00018160CF4FBC483E0182B88E62BA13CA1A4
:10C2F000829FF001839FF00D1124EA52FF4E1083BC
:10C3000080E1FE013196A1E4B9E001900D928A9599
:10C31000E1F72C968CAD9DADAEADBFAD2C97809363
:10C320003D0990933E09A0933F09B0934009E096E0
:10C330000CAD1DAD2EAD3FADE0970093610910939C
:10C3400062092093630930936409E4962CAD3DADF6
:10C350004EAD5FADE4972093650930936609409335
:10C36000670950936809E8968CAD9DADAEADBFAD41
:10C37000E8978093690990936A09A0936B09B09339
:10C380006C0960960CAD1DAD2EAD3FAD609700936E
:10C390006D0910936E0920936F09309370096C96A4
:10C3A0002CAD3DAD4EAD5FAD6C97209351093093F0
:10C3B00052094093530950935409A0968CAD9DADFA
:10C3C000AEADBFADA0978093550990935609A09349
:10C3D0005709B0935809A4960CAD1DAD2EAD3FADD5
:10C3E000A4970093590910935A0920935B0930933D
:10C3F0005C0922962CAD3DAD4EAD5FAD22972093EA
:10C400005D0930935E0940935F09509360099091F4
:10C410003B0980913C09981303C084E68093380956
:10C42000E9968FADE9978F5F8F7080933B0980917C
:10C430003B0990913A0981508F70891351C4109132
:10C440003C091BA300913B090DA728E61BA10DA5E4
:10C450001013D1C4812C912CA12CB12C1DA219A692
:10C4600019AA1EAE212C312C00E010E02DA53BA115
:10C470002313CEC42114310409F07FC580916F00CD
:10C48000826080936F0081E0ECC680E0EAC6609035
:10C490001C0770901D0700911E0710911F07A7CA67
:10C4A000818D928DA38DB48D0697A105B10508F0FD
:10C4B00018CB858D968DA78DB0A10697A105B105E6
:10C4C00008F00FCB20E030E0A901C701B6010E94BF
:10C4D00011F087FF04C0F7FAF094F7F8F09488E6BB
:10C4E0000BA11CA1809FF001819FF00D1124EA5245
:10C4F000FF4EC586D686E786F08A3ACB809118072C
:10C5000090911907A0911A07B0911B07C816D90678
:10C51000EA06FB0608F06CCB8C199D09AE09BF0931
:10C52000BC01CD01660F771F881F991F27964FAD5D
:10C530002797042F10E020E030E0A90198010E9425
:10C540008DEDCA01B9010E9472E90E941CF06C0DC8
:10C550007D1D8E1D9F1D0E9472E99B01AC0160E054
:10C5600074E284E799E40E94C7EE4B015C0140CB82
:10C57000A7019601C301B2010E94C7EE7B018C01A5
:10C580009B01AC01632D722D89A599A90E9411F020
:10C5900018160CF0E0CB3E2C2F2C09A719ABDBCBE7
:10C5A0000AA91BA92CA93DA9012B022B032B49F099
:10C5B0002091000730910107409102075091030735
:10C5C00008C02091FC063091FD064091FE06509176
:10C5D000FF0669A57AA58BA59CA50E94D3E90E94B8
:10C5E000B1EE0E9434EF2B013C012AA93BA94CA9D2
:10C5F0005DA9232B242B252BC9F020E030E0A901D5
:10C600006091F8067091F9068091FA069091FB0608
:10C610000E946EE9882351F081E00DA51EA52FA58B
:10C6200038A910161106120613060CF080E098E6E1
:10C630002BA13CA1929F8001939F100D11240A52BF
:10C640001F4E180137E4230E311CD1018C9388232F
:10C6500009F4B3C020915109309152094091530916
:10C66000509154096C966CAD7DAD8EAD9FAD6C97BD
:10C670000E94EAED6DA77EA78FA798AB2091550980
:10C68000309156094091570950915809A0966CADC8
:10C690007DAD8EAD9FADA0970E94EAED4B015C0190
:10C6A0002091590930915A0940915B0950915C09D8
:10C6B000A4966CAD7DAD8EAD9FADA4970E94EAEDC2
:10C6C0006B017C012DA53EA54FA558A9CA01B90152
:10C6D0000E94D3E96DA77EA78FA798ABA50194010F
:10C6E000C501B4010E94D3E99B01AC016DA57EA5F3
:10C6F0008FA598A90E94EBED4B015C01A701960163
:10C70000C701B6010E94D3E99B01AC01C501B40188
:10C710000E94EBED0E9456F06B017C0120915D09B7
:10C7200030915E0940915F095091600922966CAD8D
:10C730007DAD8EAD9FAD22970E94EAEDA7019601D7
:10C740000E94C7EE6B017C01F801E25BFF4F608342
:10C7500071838283938320E030E040E450E40E94C0
:10C7600011F018161CF4F101108227C02091F80670
:10C770003091F9064091FA065091FB06C701B601C7
:10C780000E94D3E99B01AC016091F4067091F5061B
:10C790008091F6069091F7060E94C7EE29A53AA56A
:10C7A0004BA55CA50E94D3E90E9434EF6415750582
:10C7B0008605970510F42B013C0180919E10909105
:10C7C0009F10A091A010B091A1100EA91FA928AD93
:10C7D00039AD80179107A207B30708F4DFC02DA178
:10C7E0003EA14FA158A5232B242B252B41F160916D
:10C7F000A2107091A3108091A4109091A5106415BF
:10C80000750586059705D8F42EA93FA948AD59AD01
:10C810000E947EED6B017C012DA13EA14FA158A588
:10C82000C301B2010E947EEDC616D706E806F906DE
:10C8300030F4C701B6010E948DED29013A0188E666
:10C840000BA11CA1809FF001819FF00D1124EA52E1
:10C85000FF4EC18CD28CE38CF48CC114D104E10462
:10C86000F10431F16091A6107091A7108091A81089
:10C870009091A9106415750586059705C8F42EA931
:10C880003FA948AD59AD0E947EED4B015C01A70167
:10C890009601C301B2010E947EED86169706A80696
:10C8A000B90630F4C501B4010E948DED29013A01A9
:10C8B00088E60BA11CA1809FF001819FF00D11243F
:10C8C000EA52FF4EC58CD68CE78CF0A0C114D1047F
:10C8D000E104F10431F16091AA107091AB108091E4
:10C8E000AC109091AD106415750586059705C8F4D8
:10C8F0002EA93FA948AD59AD0E947EED4B015C01C8
:10C90000A7019601C301B2010E947EED861697062B
:10C91000A806B90630F4C501B4010E948DED2901C5
:10C920003A0188E60BA11CA1809FF001819FF00DC8
:10C930001124EA52FF4EC1A0D2A0E3A0F4A0C1147A
:10C94000D104E104F10409F4C2CA6091AE107091FF
:10C95000AF108091B0109091B110641575058605E7
:10C96000970508F0B4CA2EA93FA948AD59AD0E9459
:10C970007EED4B015C01A7019601C301B2010E944B
:10C980007EED86169706A806B90608F0A0CAC5016E
:10C99000B4010E948DED29013A0199CA2DA13EA151
:10C9A0004FA158A5232B242B252BC9F16091A21050
:10C9B0007091A3108091A4109091A5106415750535
:10C9C0008605970560F50E9472E92AAD3BAD4CAD36
:10C9D0005DAD0E94D3E96B017C016DA17EA18FA1A9
:10C9E00098A50E9472E94B015C01C301B2010E944B
:10C9F00072E9A50194010E94D3E99B01AC01C70132
:10CA0000B6010E946EE987FF0AC0A5019401C70123
:10CA1000B6010E94C7EE0E9434EF2B013C0188E66C
:10CA20000BA11CA1809FF001819FF00D1124EA52FF
:10CA3000FF4E818C928CA38CB48C81149104A10440
:10CA4000B104B9F16091A6107091A7108091A8105F
:10CA50009091A910641575058605970550F50E94FB
:10CA600072E92AAD3BAD4CAD5DAD0E94D3E96B01DF
:10CA70007C01C501B4010E9472E94B015C01C30154
:10CA8000B2010E9472E9A50194010E94D3E99B01C1
:10CA9000AC01C701B6010E946EE987FF0AC0A5017B
:10CAA0009401C701B6010E94C7EE0E9434EF2B012A
:10CAB0003C0188E60BA11CA1809FF001819FF00D35
:10CAC0001124EA52FF4E858C968CA78CB0A081145D
:10CAD0009104A104B104B9F16091AA107091AB1056
:10CAE0008091AC109091AD10641575058605970581
:10CAF00050F50E9472E92AAD3BAD4CAD5DAD0E9490
:10CB0000D3E96B017C01C501B4010E9472E94B01BC
:10CB10005C01C301B2010E9472E9A50194010E9467
:10CB2000D3E99B01AC01C701B6010E946EE987FF02
:10CB30000AC0A5019401C701B6010E94C7EE0E9478
:10CB400034EF2B013C0188E60BA11CA1809FF00172
:10CB5000819FF00D1124EA52FF4EC1A0D2A0E3A0A4
:10CB6000F4A0C114D104E104F10409F4B0C9609146
:10CB7000AE107091AF108091B0109091B11064150B
:10CB800075058605970508F0A2C90E9472E92AADCD
:10CB90003BAD4CAD5DAD0E94D3E94B015C01C701DB
:10CBA000B6010E9472E96B017C01C301B2010E94CF
:10CBB00072E9A70196010E94D3E99B01AC01C5016E
:10CBC000B4010E946EE987FF82C9A7019601C501E1
:10CBD000B4010E94C7EE0E9434EF2B013C0177C9DB
:10CBE000FAA9FF2331F1A5019401632D722DC8012B
:10CBF0000E94D3E94B015C012DA53DA149A559A98E
:10CC0000C701B6010E94D3E99B01AC01C501B40183
:10CC10000E946EE987FF22C0A7019601C501B401F9
:10CC20000E94C7EE6DA77DA389A799AB21E02AAB2F
:10CC3000FFC9A7019601C501B4010E94C7EE9B017F
:10CC4000AC016DA57DA189A599A90E94D3E96DA725
:10CC50007DA389A799AB31E03AABEAC941E04AAB81
:10CC6000E7C9A7019601C501B40113C0C701B60108
:10CC70000E946EE987FD09C020E030E0A901C501EE
:10CC8000B4010E9411F018164CF4A5019401C701DB
:10CC9000B6010E94EAED2B013C0176CA2401350160
:10CCA00077FA709477F87094A3019201C701B601E6
:10CCB0000E946EE987FD68CA2601370165CA2DA565
:10CCC0003DA149A559A9C701B6010E946EE987FF98
:10CCD000B4CA3DA42DA009A519A9AFCA81E004CB0F
:10CCE000F0903B098FEF8F0D8F708BA3B0903A09B6
:10CCF00080913B09B81609F454C0C12CD12C0BA16A
:10CD00000B1509F44EC0602E712C28E6269D80017B
:10CD1000279D100D11240A521F4ED8018C9183FDBE
:10CD20002BC00EAF1AAB0115110541F11996BC913C
:10CD3000BDA7F801F285FDA3D8011B96BC91B9A748
:10CD4000F801F485F9ABD80115962D903D904D90E2
:10CD50005C901897A20191016DA57DA189A59F2FD7
:10CD60000E946EE9811186C1C114D10439F0F60127
:10CD7000808180FD7FC102C0CEAEDAAA8BA1815036
:10CD80008F708BA380913A098B1103C0CEACDAA8C7
:10CD9000B6CF0BA10B1529F081E08B0D8F70B82E4B
:10CDA000F1CF10913A091BA3C12CD12C80913B09E2
:10CDB0000BA1801709F443CB802E912C28E6289DE7
:10CDC0008001299D100D11240A521F4ED8018C910B
:10CDD00083FD0AC05801C114D10439F0C6010E9474
:10CDE000FE84811102C0C5C156018BA18F5F8F7077
:10CDF0008BA36501DBCF802F81508F70289FF001BE
:10CE00001124EA52FF4E908193FF24CB8DA71ECBB5
:10CE100048E6439FC0011124DC01AA52BF4E1D0108
:10CE20008C9183FD19C015966D917D918D919C918A
:10CE300018970E9456F0F62EE72ED82EC92E01150F
:10CE4000110509F48CC0F801808180FD0AC0D10170
:10CE50008C9180FD06C083C0FDA0E9A4D9A8CEAC0A
:10CE600083C0F801808181608083C8010E94FE84B4
:10CE7000811171C0F80161817281838194810E9466
:10CE800056F02B013C019B01AC0160E070E080E8B2
:10CE90009FE30E94C7EE4B015C019B01AC016F2D2B
:10CEA0007E2D8D2D9C2D0E94D3E969837A838B83FF
:10CEB0009C832DA139A549A95EADC501B4010E948D
:10CEC000D3E9698B7A8B8B8B9C8BAE014F5F5F4F65
:10CED000BE016F5E7F4FC8010E940CBAF801E95B8A
:10CEE000FF4F80818823B9F12091F8063091F9062F
:10CEF0004091FA065091FB063796608171818281DC
:10CF000093810E94D3E92091FD173091FE17409143
:10CF1000FF17509100180E94D3E94B015C019B015F
:10CF2000AC01C301B2010E94D3E90E9434EFF801C1
:10CF3000E65BFF4F71836083A50194016F2D7E2D09
:10CF40008D2D9C2D0E94D3E90E9434EFF801E45B03
:10CF5000FF4F71836083D8018C918E7F8C938F2CCF
:10CF60009E2CAD2CBC2C81018BA18F5F8F708BA36D
:10CF7000FDA2E9A6D9AACEAE79CAF101808181606D
:10CF80008083C8010E94FE8481116FC0D101119677
:10CF90006D917D918D919C9114970E9456F06B013B
:10CFA0007C019B01AC0160E070E080E89FE30E949F
:10CFB000C7EE2B013C012DEC3CEC4CE45DE30E9400
:10CFC000D3E969837A838B839C839401A501C30190
:10CFD000B2010E94D3E9698B7A8B8B8B9C8BAE015B
:10CFE0004F5F5F4FBE016F5E7F4FC1010E940CBA61
:10CFF000F101E95BFF4F80818823B9F12091F806A8
:10D000003091F9064091FA065091FB0637966081FF
:10D010007181828193810E94D3E92091FD17309123
:10D02000FE174091FF17509100180E94D3E94B0161
:10D030005C019B01AC01C701B6010E94D3E90E94CB
:10D0400034EFF101E65BFF4F718360832DEC3CEC24
:10D050004CE45DE3C501B4010E94D3E90E9434EFC2
:10D06000F101E45BFF4F71836083F10180818E7F6A
:10D07000808304CA28E6269DF001279DF00D112427
:10D08000EA52FF4E808181FD43C0C114D10441F0BA
:10D09000D6011596CD90DD90ED90FC90189708C0C4
:10D0A0008BE0C82E87EDD82E83E2E82E8BE3F82E96
:10D0B000B8E6B69DF001B79DF00D1124EA52FF4E7F
:10D0C00081899289A389B489BC01CD0190589B01C3
:10D0D000AC010E94EBEDF801258536854785508926
:10D0E0000E94D3E99B01AC01C701B6010E94EAEDA1
:10D0F000E62E872E982EA92E262F372F482F592F10
:10D100006DA57DA189A599A90E946EE987FF04C03C
:10D11000EDA48DA099A4A9A82E2D382D492D5A2D06
:10D12000C201B1010E946EE9882309F427CEF8E616
:10D13000F69DC001F79D900D11249C012A523F4E8F
:10D140006901D9018C9181608C93C8010E94FE8491
:10D15000882329F0F60180818E7F80830FCE8E2D6B
:10D16000982DA92DBA2DF60185839683A783B087C4
:10D1700005CED6018C9181FD52C0D60115962D9118
:10D180003D914D915C9118972DA73EA74FA758ABA5
:10D190001501B5E02B0E311CF801458056806780E3
:10D1A0007084A30192016DA57EA58FA598A90E9408
:10D1B0006EE987FF34C0F60181899289A389B48919
:10D1C000BC01CD0190589B01AC010E94EBEDD60152
:10D1D0001D962D913D914D915C9150970E94D3E900
:10D1E0009B01AC016DA57EA58FA598A90E94EAEDD3
:10D1F0006B017C019B01AC01C301B2010E9411F0E3
:10D2000018166CF4D8018C9181608C93C5010E9432
:10D21000FE848823E1F0F80180818E7F808318E608
:10D22000189DF001199DF00D1124EA52FF4E218541
:10D2300032854385548565817681878190850E94FA
:10D240006EE98111D2CD0BA100933A09CECDD10167
:10D25000CD92DD92ED92FC9213970BA100933A09C7
:10D26000DECFC858DF4F0FB6F894DEBF0FBECDBF7C
:10D27000DF91CF911F910F91FF90EF90DF90CF90B2
:10D28000BF90AF909F908F907F906F905F904F90E6
:10D290003F902F90089580913B0990913C09891B04
:10D2A0008F708F3019F40E945BAAF5CF80913B09F3
:10D2B0008F5F8F70E0913B0998E69E9FF0011124EB
:10D2C000EA52FF4EDF011D929A95E9F798E09083AC
:10D2D00040916109509162096091630970916409FC
:10D2E000458B568B678B708F40916509509166090D
:10D2F0006091670970916809418F528F638F748FB5
:10D300004091690950916A0960916B0970916C09AB
:10D31000458F568F678F70A340916D0950916E09AC
:10D3200060916F097091700941A352A363A374A324
:10D3300020913B0990913C09291303C094E69093F6
:10D34000380980933B0980916F00826080936F0061
:10D35000089590913B0980913C09981306C08091F3
:10D36000820F9091830F892B19F00E945BAAF1CF55
:10D3700008958F929F92AF92BF92CF92DF92EF92D9
:10D38000FF921F93CF93DF93C82F8BE59BE0909381
:10D390003709809336091092770B82E090E0A0E085
:10D3A000B0E08093600B9093610BA093620BB093FD
:10D3B000630B1092350910923109109232091092C4
:10D3C0003309109234098FEF9FEFDC0180932D0910
:10D3D00090932E09A0932F09B0933009CC2379F1B3
:10D3E000C53008F0F8C040E060E070E0CB010E947A
:10D3F000B9D4882309F4EFC020E1C29FC0011124F1
:10D40000835E984FFC01E254FE4F20812F7709F094
:10D41000E2C03C964081518162817381443651055E
:10D420006105710508F4D7C03497C080D180E280CF
:10D43000F380C114D104E104F10421F4CCC0C12C67
:10D44000D12C760140E0C701B6010E94B9D4182F53
:10D45000882309F4C0C0809138079091390781155D
:10D46000924009F0B8C0A0913D07AA2309F4B3C0C7
:10D4700060913B0770913C076115710509F4ABC0E1
:10D4800020913A07222309F4A6C0A093720B20939F
:10D49000640B80E030E041E050E0C82FFA01082E34
:10D4A00002C0EE0FFF1F0A94E2F72E173F0739F074
:10D4B0008F5FC83091F789E080936D0B8CC08093AB
:10D4C0006D0B20914307309144072115310519F068
:10D4D00040E050E008C02091510730915207409140
:10D4E0005307509154072093650B3093660B40937C
:10D4F000670B5093680B46015701860E971EA11CBF
:10D50000B11C8092730B9092740BA092750BB09229
:10D51000760BE0913E07F0913F07F093790BE09393
:10D52000780BB0E00E94CBED860E971EA81EB91EA8
:10D5300080927A0B90927B0BA0927C0BB0927D0B29
:10D5400085E0EE0FFF1F8A95E1F7E150FE4FEF2FC8
:10D55000FF27E6958E0E9F1EA11CB11C80926E0BBC
:10D5600090926F0BA092700BB092710B20914007BC
:10D57000309141072115310521F0A90160E070E0EB
:10D5800008C040914D0750914E0760914F07709130
:10D590005007D701C60188199909AA09BB09840F48
:10D5A000951FA61FB71F04C0B695A7959795879599
:10D5B000CA95D2F78093690B90936A0BA0936B0B7B
:10D5C000B0936C0B853F2FE09207A105B10528F4BD
:10D5D0008CE08093770B10E01AC0853F9F4FA10528
:10D5E000B10510F480E111C08091590790915A075C
:10D5F000A0915B07B0915C0780937A0B90937B0BB3
:10D60000A0937C0BB0937D0B80E28093770B812FEE
:10D61000DF91CF911F91FF90EF90DF90CF90BF905F
:10D62000AF909F908F900895682F82E29FE00C94B6
:10D630009E4ACF92DF92EF92FF921F93CF93DF9398
:10D640001092BA098091ED09882321F08AEE99E0C1
:10D650000E9438A210925F0B10925C0B85E38093BE
:10D660005B0B0E949058EB01A89561E080915B0BE9
:10D670000E94BBC58BE59BE00E9499A32398229A48
:10D68000219A209A289A85E080935D0B82E58CBDD3
:10D690001DBC1AE08FEF0E949EA31150D9F720E025
:10D6A00030E0A90160E08BE59BE00E94A3A3182F66
:10D6B00080935E0B813049F00E9490586C1B7D0B6B
:10D6C000613D774060F381E054C02AEA31E040E0F8
:10D6D00050E068E08BE59BE00E94A3A382FF03C0BB
:10D6E00010935F0B0EC014E00E94B1A880935E0BF4
:10D6F0001150D1F78A3A11F082E03BC082E080936A
:10D700005F0B80915F0B823021F0C12CD12C760110
:10D7100005C0C12CD12CE12C80E4F82E20E030E0B3
:10D72000A90167E38BE59BE00E94A3A3A7019601F3
:10D7300069E28BE59BE00E94A3A380935E0B8823A4
:10D7400049F00E9490586C1B7D0B613D774030F38F
:10D750008AE00FC080915F0B823011F520E030E04D
:10D76000A9016AE38BE59BE00E94A3A3882351F003
:10D7700088E080935C0B8BE59BE00E9499A3E3E338
:10D78000FAE119C00E94B1A8807C803C19F483E0C2
:10D7900080935F0B0E94B1A80E94B1A80E94B1A81B
:10D7A0008BE59BE00E9499A310925D0B81E0E1DD87
:10D7B000811131C015C08491EF012196882321F099
:10D7C0000E94188AFE01F7CFE5E2FAE18491EF01A9
:10D7D0002196882309F456C00E94188AFE01F6CFCC
:10D7E00080E0C7DD811117C0EEE1FAE18491EF011D
:10D7F0002196882321F00E94188AFE01F7CFEAE0E3
:10D80000FAE18491EF012196882309F43BC00E943C
:10D81000188AFE01F6CF60E67BE08AEE99E00E946E
:10D82000E5A1811116C0EEE1FAE18491EF012196A4
:10D83000882321F00E94188AFE01F7CFE9EFF9E171
:10D840008491EF0121968823E9F00E94188AFE0155
:10D85000F7CF81E08093BA09E3E3FAE18491EF0125
:10D860002196882321F00E94188AFE01F7CFEDEE61
:10D87000F9E18491EF012196882321F00E94188A12
:10D88000FE01F7CF8BE1EAEEF9E0A9E0BAE0019002
:10D890000D928A95E1F78091E8099091E9099093BA
:10D8A000080A8093070ADF91CF911F91FF90EF90B4
:10D8B000DF90CF9008958091C70D823041F488EDBC
:10D8C00099E190932C0780932B070E94448A0E9431
:10D8D00090586093CB0D7093CC0D8093CD0D9093A9
:10D8E000CE0D8091BA09882319F081E08093B9099F
:10D8F00081E08093C70D0895CF93DF931092B9090B
:10D9000083E08093C70D8091140E8823B1F0E0ED81
:10D91000F9E18491EF01882341F0082E000C990B66
:10D9200083DE2196FE018491F6CF8DE090E07CDECF
:10D930008AE090E0DF91CF9177CEE4EDF9E1849138
:10D94000EF01882391F3082E000C990B6DDE2196D0
:10D95000FE018491F6CF8F929F92AF92BF92CF92A9
:10D96000DF92EF92FF920F931F93CF93DF9300D03C
:10D970001F92CDB7DEB7FC018381813079F58181BB
:10D9800081FF2CC081899289A389B489892B8A2B34
:10D990008B2B09F448C07F0140E050E0BA01CF0171
:10D9A0000E944EA18823D1F0F70185889688A78828
:10D9B000B08CC18CD28C82E090E0A0E0B0E0F601A7
:10D9C00080839183A283B3839E012F5F3F4FB50174
:10D9D000A401C6010E9482D5811102C080E03CC032
:10D9E00000E010E09801B501A401C6010E94F1D445
:10D9F0008823A1F389809A80AB80BC80F601878957
:10DA0000803141F4F8EF8F16FFEF9F06A104B104B7
:10DA100060F4DACF88EF88168FEF9806A8068FE0BB
:10DA2000B80618F4D1CF81E017C0F701158A168A1D
:10DA3000178A108E118A128A138A148A818180684B
:10DA40008183C7010E94D0D6882341F240E050E094
:10DA5000BA01C7010E944EA10F900F900F900F9036
:10DA6000DF91CF911F910F91FF90EF90DF90CF90BA
:10DA7000BF90AF909F908F9008951092BC09109224
:10DA8000B9098091850B882321F082E89BE00C94F2
:10DA900038A208952F923F924F925F926F927F9299
:10DAA0008F929F92AF92BF92CF92DF92EF92FF92AE
:10DAB0000F931F93CF93DF93CDB7DEB7C257D10932
:10DAC0000FB6F894DEBF0FBECDBF8C013B014A01FB
:10DAD0004DB75EB7E1965FAF4EAFE197AD961FAE23
:10DAE000AD971B0154E0250E311C7E018FE5E80E39
:10DAF000F11C95E6492E92E0592EE0E4F0E0EC0F9F
:10DB0000FD1F3496E396FFAFEEAFE397F3018781F5
:10DB1000823008F462C184859585A685B7858F71AA
:10DB20009927AA27BB27892B8A2B8B2B09F055C154
:10DB30001092CA094AEC59E0BE016F5F7F4FC101E4
:10DB40000E9468D618160CF048C18C85982F9871E1
:10DB5000903129F42091370C2150223078F429811A
:10DB6000222309F43AC1253E89F22E3279F220911E
:10DB7000CA092E3259F28A7049F6B8C04DB75EB75D
:10DB8000AF965FAF4EAFAF97BE016F5F7F4FC701DC
:10DB90000E9463D40115110521F0F80180818111E3
:10DBA0009BC021E081E090E0F70101900020E9F7BF
:10DBB0003197EE19FF098E0F9F1F02964DB75EB782
:10DBC000481B590B0FB6F8945EBF0FBE4DBF8DB703
:10DBD0009EB701965C01211102C0B80102C062E249
:10DBE00073E0C5010E944FF1B701C5010E9430F1F9
:10DBF00062E273E0C5010E9430F125961FAE2597C1
:10DC000028961FAE289724961FAE1EAE2497229604
:10DC10005FAE4EAE229721E0A701B101E3968EAD33
:10DC20009FADE3970E94C4A781112AC08091370C51
:10DC3000811126C0E3E3FAE184916F019FEFC91AD5
:10DC4000D90A882321F00E94188AF601F5CFECEB5F
:10DC5000F9E184916F012FEFC21AD20A882321F0D3
:10DC60000E94188AF601F5CF6701F60181916F01D4
:10DC7000882319F00E94188AF8CF8AE00E94188A37
:10DC80008BE1FE01EC5BFF4FDE01959601900D925A
:10DC90008A95E1F724968EAD9FAD24979CA38BA324
:10DCA0005AA249A240E050E0BE016F5D7F4FC5011E
:10DCB000F1DECE0181960E94F1A9CE01805C9F4FDA
:10DCC0000E94F1A9AF964EAD5FADAF970FB6F89435
:10DCD0005EBF0FBE4DBF1ACFF80101900020E9F7DB
:10DCE0003197CF01801B910B20E05ECF81E0903116
:10DCF00009F080E08093BB09903141F08985873439
:10DD000009F004CF8A858E3709F400CF8091370C53
:10DD1000813029F08230D9F18111F8CE0AC080918A
:10DD2000380C9091390C01969093390C8093380CF3
:10DD3000EDCEBE016F5F7F4F8DEB99E00E9463D403
:10DD40000115110529F48DEBC82E89E0D82E09C0E4
:10DD50006801F60181916F018823A9F30E94188A56
:10DD6000F8CFF60181916F01882319F00E94188A7B
:10DD7000F8CF80E20E94188A6D8D7E8D8F8D98A1DC
:10DD80004AE00E943B8D8AE00E94188ABFCEBE0105
:10DD90006F5F7F4F8DEB99E00E9463D481149104F3
:10DDA00041F06DEB79E0C4010E941DF1892B69F40B
:10DDB00014C0AD96FFADAD978F2F90E02091440F2A
:10DDC0003091450F8217930741F0AD962FADAD9777
:10DDD0002F5FAD962FAFAD9799CEE1968EAD9FADEB
:10DDE000E1970FB6F8949EBF0FBE8DBFCE58DF4FA0
:10DDF0000FB6F894DEBF0FBECDBFDF91CF911F915C
:10DE00000F91FF90EF90DF90CF90BF90AF909F90D9
:10DE10008F907F906F905F904F903F902F900895DC
:10DE20000F931F93CF93DF93CDB7DEB76F970FB6E6
:10DE3000F894DEBF0FBECDBF8B0122E02093370CDC
:10DE40009093450F8093440F89E09AE00E9495A338
:10DE50008BE1E9E0FAE0DE01159601900D928A95DA
:10DE6000E1F78091070A9091080A9C838B8385E6ED
:10DE700092E09A838983A801BE016F5F7F4F80E0A3
:10DE800090E008DECE0101960E94F1A96F960FB6D0
:10DE9000F894DEBF0FBECDBFDF91CF911F910F91E0
:10DEA00008952F923F924F925F926F927F928F923E
:10DEB0009F92AF92BF92CF92DF92EF92FF920F9319
:10DEC0001F93CF93DF93CDB7DEB76F970FB6F8945C
:10DED000DEBF0FBECDBF6C012DB63EB61D821886CB
:10DEE0001C821B8285E692E09A838983FB018081F4
:10DEF0009E012F5F3F4F39018F3241F085E09AE05C
:10DF0000F60191838083F62E172F64C086EE99E088
:10DF1000F601918380838B010F5F1F4F011511055F
:10DF200009F456C04DB65EB66FE270E0C8010E94BB
:10DF30003BF14C010817190708F048C07C01E01AB2
:10DF4000F10AFF24C70101962DB73EB7281B390BF4
:10DF50000FB6F8943EBF0FBE2DBF8DB79EB701968A
:10DF60005C01A701B8010E9464F1F501EE0DFF1DEF
:10DF70001082F601608171816115710511F06C5F8D
:10DF80007F4F21E0A501CE0105960E94C4A7811113
:10DF900011C0B50188EA99E10E9408B48EE20E949E
:10DFA000188A8AE00E94188A0FB6F8945EBE0FBEE7
:10DFB0004DBE0EC0F6017182608284010F5F1F4F5B
:10DFC0000FB6F8945EBE0FBE4DBEA8CFF02E02C0B5
:10DFD000F12C10E0C3010E94F1A98F2D912F0FB6F3
:10DFE000F8943EBE0FBE2DBE6F960FB6F894DEBFFE
:10DFF0000FBECDBFDF91CF911F910F91FF90EF909A
:10E00000DF90CF90BF90AF909F908F907F906F9058
:10E010005F904F903F902F900895CF93DF938B3D6B
:10E020009240B1F0EEE1FAE18491EF01219688236C
:10E0300021F00E94188AFE01F7CFE9E3FAE184910A
:10E04000EF012196882331F00E94188AFE01F7CF54
:10E0500080E001C081E0DF91CF9108952F923F923F
:10E060004F925F926F927F928F929F92AF92BF92E8
:10E07000CF92DF92EF92FF920F931F93CF93DF9394
:10E08000CDB7DEB7C757D1090FB6F894DEBF0FBEC4
:10E09000CDBF2DB63EB6A7961FAE1EAEA79784E69F
:10E0A00090E0A9969FAF8EAFA99701E09E012B59F2
:10E0B0003F4F44E050E0BE01655A7F4FCE01895981
:10E0C0009F4F0E940FD39E012B593F4F42E050E0DB
:10E0D000BE0167597F4FCE0189599F4F0E940FD3D0
:10E0E00043E050E0BE01655A7F4F8FE093E00E940D
:10E0F00056F1892B09F43FC06F968FAD6F97882337
:10E1000039F08FE36C968FAF6C976D961FAE6D975D
:10E11000E3E3FAE184917F012FEFE21AF20A811121
:10E1200003C0ECEFFAE104C00E94188AF701F2CFB5
:10E1300084917F013FEFE31AF30A882321F00E94C4
:10E14000188AF701F5CFBE01655A7F4F83EF9AE138
:10E150000E9408B4E5EEFAE184917F019FEFE91A8D
:10E16000F90A882321F00E94188AF701F5CF81E08F
:10E170008093460F4EC5EDB7FEB7E696FFAFEEAF04
:10E18000E6976B961CAE1DAE1EAE1FAE6B97A796A4
:10E190001FAE1EAEA79701E09E012B593F4F41E0F5
:10E1A00050E0BE0160597F4FCE0189599F4F0E94B8
:10E1B0000FD380E1EBE8F2E0DE01919601900D9241
:10E1C0008A95E1F780E1EBE9F2E0DE0151960190FA
:10E1D0000D928A95E1F780E1EBEAF2E0DE0111961B
:10E1E00001900D928A95E1F7E1964FADE19750E0ED
:10E1F0004D5F5F4F440F551F440F551F2DB73EB75E
:10E20000241B350B0FB6F8943EBF0FBE2DBF8DB744
:10E210009EB701967C0100E09E012B593F4FBC0147
:10E22000CE0189599F4F0E940FD39E012B593F4F1A
:10E2300044E050E068E177E0CE0189599F4F0E94A9
:10E240000FD3E1968FACE197912C93E0890E911C4E
:10E25000880C991C880C991CEDB7FEB7E819F909D0
:10E260000FB6F894FEBF0FBEEDBF2DB73EB72F5FC0
:10E270003F4F69018DB79EB7881999090FB6F89479
:10E280009EBF0FBE8DBFEDB7FEB731965F019E01F9
:10E290002B593F4FA401B601CE0189599F4F0E94CF
:10E2A0000FD39E012B593F4FA401B501CE018959CF
:10E2B0009F4F0E940FD31091470F112309F4A7C05D
:10E2C00000E09E012B593F4F44E050E060E077E0D2
:10E2D000CE0189599F4F0E940FD39E012B593F4F6A
:10E2E00044E050E064E077E0CE0189599F4F0E94FE
:10E2F0000FD39E012B593F4F44E050E06CEF76E086
:10E30000CE0189599F4F0E940FD39E012B593F4F39
:10E3100044E050E060E277E0CE0189599F4F0E94CF
:10E320000FD39E012B593F4F44E050E06CE177E062
:10E33000CE0189599F4F0E940FD39E012B593F4F09
:10E3400040E150E068EE76E0CE0189599F4F0E948F
:10E350000FD39E012B593F4F44E050E0BE01695A54
:10E360007F4FCE0189599F4F0E940FD39E012B5999
:10E370003F4F4CE050E06DE475E0CE0189599F4F6E
:10E380000E940FD39E012B593F4F44E050E061E2C1
:10E3900078E1CE0189599F4F0E940FD39E012B59DE
:10E3A0003F4F44E050E0BE01695A7F4FCE0189598A
:10E3B0009F4F0E940FD301E09E012B593F4F41E038
:10E3C00050E0BE0161597F4FCE0189599F4F0E9495
:10E3D0000FD39E012B593F4F41E050E0BE016259DF
:10E3E0007F4FCE0189599F4F0E940FD311118AC0D0
:10E3F0006B968CAD9DADAEADBFAD6B9780935A174C
:10E4000090935B17A0935C17B0935D177BC0E19668
:10E410008FADE19790E0029628E037E0E4963FAFB9
:10E420002EAFE497B501DE011196E1EF8E2EE7E104
:10E430009E2EAE014F5E5F4FF2EBAF2EF0E1BF2E8E
:10E44000E896FFAEEEAEE8977E0131E2E30EF11CF6
:10E4500020E030E0821793072CF0E896EEADFFAD98
:10E46000E89701C0F7014080518062807380F50118
:10E4700041925192619271925F018217930714F059
:10E48000F60101C0FA014080518062807380F4017E
:10E4900041925192619271924F018217930734F029
:10E4A000FB01408051806280738005C04D905D907B
:10E4B0006D907C901397E496EEADFFADE49741929A
:10E4C000519261927192E496FFAFEEAFE4972F5FA5
:10E4D0003F4F6C5F7F4F1496F4E0CF0ED11C4C5F22
:10E4E0005F4FE896EEADFFADE8973496E896FFAF44
:10E4F000EEAFE897F4E0EF0EF11C2430310509F09F
:10E50000A9CFDECEE0968FADE097853099F4AF9637
:10E510008FADAF97853071F400E09E012B593F4FCE
:10E5200044E650E06EE577E1CE0189599F4F0E94A5
:10E530000FD324C0111102C00E9472BFE0968FADAC
:10E54000E097AF96CFACAF978C9D60011124E12C82
:10E55000F12CEC14FD0491F000E09E012B593F4F8B
:10E5600044E050E0BE01695A7F4FCE0189599F4F68
:10E570000E940FD32FEFE21AF20AEBCF00E09E01C8
:10E580002B593F4F44E050E0BE016D5A7F4FCE0102
:10E5900089599F4F0E940FD31AE0115079F000E083
:10E5A0009E012B593F4F44E050E0BE01695A7F4F16
:10E5B000CE0189599F4F0E940FD3EFCF01E09E01FA
:10E5C0002B593F4F41E050E0BE0163597F4FCE01D0
:10E5D00089599F4F0E940FD39E012B593F4F41E015
:10E5E00050E0BE0164597F4FCE0189599F4F0E9470
:10E5F0000FD300E09E012B593F4F44E050E0BE0195
:10E60000635C7F4FCE0189599F4F0E940FD39E01BB
:10E610002B593F4F44E050E0BE016F5C7F4FCE016D
:10E6200089599F4F0E940FD3AE968FADAE97AD968E
:10E63000CFACAD978C9D60011124E12CF12C00E052
:10E640009E012B593F4FEC14FD0471F044E050E063
:10E65000BE01695A7F4FCE0189599F4F0E940FD347
:10E660003FEFE31AF30AEBCF41E050E0BE016F58F1
:10E670007F4FCE0189599F4F0E940FD39E012B5986
:10E680003F4F41E050E0BE0165597F4FCE018959AF
:10E690009F4F0E940FD39E012B593F4F44E050E003
:10E6A000BE01695A7F4FCE0189599F4F0E940FD3F7
:10E6B0009E012B593F4F44E050E0BE01695A7F4F05
:10E6C000CE0189599F4F0E940FD39E012B593F4F76
:10E6D00044E050E065E278E1CE0189599F4F0E9405
:10E6E0000FD39E012B593F4F44E050E0BE01615BC8
:10E6F0007F4FCE0189599F4F0E940FD39E012B5906
:10E700003F4F44E050E0BE01655B7F4FCE01895929
:10E710009F4F0E940FD39E012B593F4F44E050E082
:10E72000BE01695B7F4FCE0189599F4F0E940FD375
:10E7300010E000E09E012B593F4F44E050E0BE0145
:10E74000695A7F4FCE0189599F4F0E940FD31111F3
:10E7500010C06B96CCACDDACEEACFFAC6B9720E0A0
:10E7600030E84BE355E4C701B6010E946EE9811120
:10E7700003C054E0F52E33C08091470F811108C0CB
:10E78000C092740FD092750FE092760FF092770FCF
:10E7900000E09E012B593F4F44E050E060E77FE0EE
:10E7A000CE0189599F4F0E940FD39E012B593F4F95
:10E7B00044E050E068E77FE0CE0189599F4F0E9416
:10E7C0000FD39E012B593F4F44E050E0BE01695AE0
:10E7D0007F4FCE0189599F4F0E940FD312C0FA94E8
:10E7E000FF2079F000E09E012B593F4F44E050E0BC
:10E7F000BE01695A7F4FCE0189599F4F0E940FD3A6
:10E80000EECF1F5F153009F094CF00E09E012B5929
:10E810003F4F42E050E0BE016D597F4FCE01895914
:10E820009F4F0E940FD39E012B593F4F44E050E071
:10E83000BE01695A7F4FCE0189599F4F0E940FD365
:10E840006B96CCACDDACEEACFFAC6B9720E030E867
:10E850004BE355E4C701B6010E946EE9882329F114
:10E860008091470F811108C0C0926C0FD0926D0F3C
:10E87000E0926E0FF0926F0F00E09E012B593F4F18
:10E8800044E050E068E67FE0CE0189599F4F0E9446
:10E890000FD39E012B593F4F44E050E064E67FE0E8
:10E8A000CE0189599F4F0E940FD300E09E012B5942
:10E8B0003F4F42E050E0BE016F597F4FCE01895972
:10E8C0009F4F0E940FD39E012B593F4F41E050E0D4
:10E8D000BE016F587F4FCE0189599F4F0E940FD3C1
:10E8E00019E0115000E09E012B593F4F112359F0C0
:10E8F00044E050E0BE01695A7F4FCE0189599F4FD5
:10E900000E940FD3EECF41E050E062EC77E1CE0100
:10E9100089599F4F0E940FD3F12C00E09E012B5983
:10E920003F4F44E050E0BE01695A7F4FCE01895904
:10E930009F4F0E940FD31091470F111110C0F1107B
:10E940000EC06B968CAD9DADAEADBFAD6B97809399
:10E95000C7179093C817A093C917B093CA17F39419
:10E9600085E0F812DACF111102C00E9450B34CE0DA
:10E97000F42EFA94F11003C03CE0F32E0FC000E037
:10E980009E012B593F4F42E050E0BE01615A7F4F3C
:10E99000CE0189599F4F0E940FD3EBCFFA9400E02C
:10E9A0009E012B593F4FFF2059F044E050E0BE013B
:10E9B0006D5B7F4FCE0189599F4F0E940FD3EECFE1
:10E9C00046E050E0BE01635C7F4FCE0189599F4F06
:10E9D0000E940FD39E012B593F4F44E050E068EF57
:10E9E00076E0CE0189599F4F0E940FD39E012B598B
:10E9F0003F4F4CE050E0BE016F5C7F4FCE01895924
:10EA00009F4F0E940FD32CE1F22EFA94F11003C015
:10EA100094E0F92E1DC000E09E012B593F4F44E0C9
:10EA200050E0BE01695A7F4FCE0189599F4F0E9425
:10EA30000FD3EBCF00E09E012B593F4F44E050E055
:10EA4000BE01695A7F4FCE0189599F4F0E940FD353
:10EA5000FA94F110EFCF8BE0F82EFA94FF2079F0C2
:10EA600000E09E012B593F4F44E050E0BE01695A3F
:10EA70007F4FCE0189599F4F0E940FD3EECFA996A9
:10EA80008EAD9FADA99784569109C7DA8093460F42
:10EA9000882309F1E3E3FAE184917F019FEFE91A0A
:10EAA000F90A882321F00E94188AF701F5CFA99668
:10EAB0006EAD7FADA997645671098DED9AE10E9404
:10EAC000EFB36BED72E085ED9AE10E94EFB38AE05F
:10EAD0000E94188A93C0A7962EAD3FADA797AB961C
:10EAE0008EAD9FADAB972817390709F445C081E07B
:10EAF0008093460FEEE1FAE184917F012FEFE21A55
:10EB0000F20A811103C0E5EBFAE104C00E94188A01
:10EB1000F701F2CF84917F013FEFE31AF30A8823D4
:10EB200021F00E94188AF701F5CFAB968EAD9FAD0C
:10EB3000AB970E94D9DAE0EBFAE184917F019FEF75
:10EB4000E91AF90A882321F00E94188AF701F5CF03
:10EB5000A7968EAD9FADA7970E94D9DAE0EAFAE1B9
:10EB600084917F012FEFE21AF20A882309F446C04C
:10EB70000E94188AF701F4CF111142C0E3E3FAE1D1
:10EB800084917F013FEFE31AF30A811103C00FE084
:10EB900013E004C00E94188AF701F2CFF8018191B6
:10EBA0008F01882319F00E94188AF8CFA9966EADBC
:10EBB0007FADA9976456710983E89AE10E94EFB38B
:10EBC000A7964EAD5FADA79760E070E086E79AE14B
:10EBD0000E94B5B3E3E7FAE184917F012FEFE21AD7
:10EBE000F20A811107C08091460F811109C00E946D
:10EBF000D0D306C00E94188AF701EECF112399F3F3
:10EC0000E6968EAD9FADE6970FB6F8949EBF0FBE09
:10EC10008DBF8091470F811102C00E94F8C690916C
:10EC2000460F81E089270FB6F8943EBE0FBE2DBE79
:10EC3000C958DF4F0FB6F894DEBF0FBECDBFDF91CE
:10EC4000CF911F910F91FF90EF90DF90CF90BF90E9
:10EC5000AF909F908F907F906F905F904F903F907C
:10EC60002F90089581E08093470FF8D91092470FB5
:10EC70008111F4C90E948DCB81E008958F929F92FB
:10EC8000AF92BF92CF92DF92EF92FF920F931F93BA
:10EC9000CF93DF93CDB7DEB7CA5AD1090FB6F89438
:10ECA000DEBF0FBECDBFE9961CAE1DAE1EAE1FAEC1
:10ECB000E9978091F1039091F203A091F303B09151
:10ECC000F403ED968CAF9DAFAEAFBFAFED97C556D9
:10ECD000DF4F19821882CB59D04084E690E0C356AA
:10ECE000DF4F99838883CD59D0401092460F9E0103
:10ECF00025563F4F44E050E0BE0167587F4FCE019C
:10ED000083569F4F0E945CD3C356DF4F8881998101
:10ED1000CD59D0400296C356DF4F99838883CD5991
:10ED2000D040C556DF4F19821882CB59D04081E0C0
:10ED3000CD55DF4F8883C35AD0409E0125563F4FA3
:10ED400041E050E0BE016D557F4FCE0183569F4F8D
:10ED50000E945CD39E0125563F4F40E150E062EB9C
:10ED600070E1CE0183569F4F0E945CD39E012556D1
:10ED70003F4F44E050E068E177E0CE0183569F4F7B
:10ED80000E945CD39E0125563F4F40E150E061EF69
:10ED900077E1CE0183569F4F0E945CD39E0125569A
:10EDA0003F4F40E150E068E077E0CE0183569F4F4F
:10EDB0000E945CD39E0125563F4F44E050E060E046
:10EDC00077E0CE0183569F4F0E945CD39E0125566B
:10EDD0003F4F44E050E064E077E0CE0183569F4F20
:10EDE0000E945CD39E0125563F4F44E050E06CEFFB
:10EDF00076E0CE0183569F4F0E945CD39E0125563C
:10EE00003F4F44E050E060E277E0CE0183569F4FF1
:10EE10000E945CD39E0125563F4F44E050E06CE1D8
:10EE200077E0CE0183569F4F0E945CD39E0125560A
:10EE30003F4F40E150E068EE76E0CE0183569F4FB1
:10EE40000E945CD38AE097EDA3EABCE3E9968CAF1D
:10EE50009DAFAEAFBFAFE9979E0125563F4F44E04F
:10EE600050E0BE016B587F4FCE0183569F4F0E94EA
:10EE70005CD39E0125563F4F4CE050E06DE475E0B9
:10EE8000CE0183569F4F0E945CD38091DC179091F6
:10EE9000DD17A091DE17B091DF17C358DF4F8883CD
:10EEA0009983AA83BB83CD57D0409E0125563F4FFF
:10EEB00044E050E0BE0163587F4FCE0183569F4F20
:10EEC0000E945CD385E0CC55DF4F8883C45AD04084
:10EED000CB55DF4F8883C55AD0409E0125563F4F02
:10EEE00044E050E06AE577E1CE0183569F4F0E94EF
:10EEF0005CD39E0125563F4F41E050E0BE016C556A
:10EF00007F4FCE0183569F4F0E945CD39E012556B2
:10EF10003F4F41E050E0BE016B557F4FCE0183561D
:10EF20009F4F0E945CD39E0125563F4F44E650E020
:10EF30006EE577E1CE0183569F4F0E945CD3CF5799
:10EF4000DF4F188219821A821B82C158D0409E015D
:10EF500025563F4F44E050E0BE016F577F4FCE0132
:10EF600083569F4F0E945CD3E9961CAE1DAE1EAE29
:10EF70001FAEE9971AE0115071F09E0125563F4FE0
:10EF800044E050E0BE016B587F4FCE0183569F4F47
:10EF90000E945CD3F0CF83E0CA55DF4F8883C65A06
:10EFA000D040C955DF4F8883C75AD040CB57DF4F79
:10EFB000188219821A821B82C558D040C757DF4F6A
:10EFC000188219821A821B82C958D040E9961CAE59
:10EFD0001DAE1EAE1FAEE9979E0125563F4F41E084
:10EFE00050E0BE016A557F4FCE0183569F4F0E946D
:10EFF0005CD39E0125563F4F41E050E0BE0169556C
:10F000007F4FCE0183569F4F0E945CD39E012556B1
:10F010003F4F44E050E0BE0167577F4FCE0183561B
:10F020009F4F0E945CD39E0125563F4F44E050E025
:10F03000BE016B577F4FCE0183569F4F0E945CD31A
:10F040000AE010E00150110971F09E0125563F4F72
:10F0500044E050E0BE016B587F4FCE0183569F4F76
:10F060000E945CD3EFCFC855DF4F1882C85AD040FA
:10F070008FEFC755DF4F8883C95AD0409E01255670
:10F080003F4F41E050E0BE0168557F4FCE018356AF
:10F090009F4F0E945CD39E0125563F4F41E050E0B8
:10F0A000BE0167557F4FCE0183569F4F0E945CD3B0
:10F0B000E9961CAE1DAE1EAE1FAEE9979E01255609
:10F0C0003F4F44E050E0BE016B587F4FCE01835666
:10F0D0009F4F0E945CD39E0125563F4F44E050E075
:10F0E000BE016B587F4FCE0183569F4F0E945CD369
:10F0F0009E0125563F4F44E050E065E278E1CE01A5
:10F1000083569F4F0E945CD38091BB029091BC02BA
:10F11000A091BD02B091BE02C357DF4F888399838F
:10F12000AA83BB83CD58D0408091BF029091C0028A
:10F13000A091C102B091C202CF56DF4F888399835C
:10F14000AA83BB83C159D040CB56DF4F19821882A6
:10F15000C559D040C956DF4F19821882C759D040CF
:10F160009E0125563F4F44E050E0BE0163577F4F5C
:10F17000CE0183569F4F0E945CD39E0125563F4F80
:10F1800044E050E0BE016F567F4FCE0183569F4F43
:10F190000E945CD39E0125563F4F44E050E0BE01E3
:10F1A0006B567F4FCE0183569F4F0E945CD310E079
:10F1B000C12C80E8D82E8BE3E82E85E4F82E812C34
:10F1C000912C90E8A92E9FE3B92E111138C09E0111
:10F1D00025563F4F44E050E064E77FE0CE01835680
:10F1E0009F4F0E945CD39E0125563F4F44E050E064
:10F1F00060E77FE0CE0183569F4F0E945CD39E0163
:10F2000025563F4F44E050E068E77FE0CE0183564B
:10F210009F4F0E945CD3E9968CAE9DAEAEAEBFAE62
:10F22000E9979E0125563F4F44E050E0BE016B58E0
:10F230007F4FCE0183569F4F0E945CD32AC0E99630
:10F24000CCAEDDAEEEAEFFAEE9979E0125563F4F48
:10F2500044E050E0BE016B587F4FCE0183569F4F74
:10F260000E945CD3E9961CAE1DAE1EAE1FAEE997A0
:10F2700004E0015071F09E0125563F4F44E050E0FC
:10F28000BE016B587F4FCE0183569F4F0E945CD3C7
:10F29000F0CF1F5F153009F098CF84E190E0C156A0
:10F2A000DF4F99838883CF59D0409E0125563F4F29
:10F2B00042E050E0BE0161567F4FCE0183569F4F22
:10F2C0000E945CD39E0125563F4F44E050E06CE61F
:10F2D0007FE0CE0183569F4F0E945CD39E0125564E
:10F2E0003F4F44E050E068E67FE0CE0183569F4FF9
:10F2F0000E945CD39E0125563F4F44E050E064E6F7
:10F300007FE0CE0183569F4F0E945CD380E290E065
:10F31000CF55DF4F99838883C15AD0409E0125562F
:10F320003F4F42E050E0BE016F557F4FCE01835604
:10F330009F4F0E945CD3C655DF4F1882CA5AD040F7
:10F3400080E2E3ECF2E0DE019D9601900D928A9559
:10F35000E1F79E0125563F4F41E050E0BE01665562
:10F360007F4FCE0183569F4F0E945CD39E0125564E
:10F370003F4F40E250E0BE01635D7F4FCE018356B8
:10F380009F4F0E945CD39E0125563F4F41E050E0C5
:10F3900062EC77E1CE0183569F4F0E945CD310E070
:10F3A00011110EC08091C7179091C817A091C9176D
:10F3B000B091CA17E9968CAF9DAFAEAFBFAFE997DA
:10F3C0009E0125563F4F44E050E0BE016B587F4FF1
:10F3D000CE0183569F4F0E945CD31F5F153001F70B
:10F3E000BE01635B7F4F86E1FB0111928A95E9F7CD
:10F3F0009E0125563F4F46E150E0CE0183569F4F78
:10F400000E945CD38CE2E3EEF2E0DE011196019003
:10F410000D928A95E1F79E0125563F4F4CE250E050
:10F42000BE016F5F7F4FCE0183569F4F0E945CD31A
:10F43000BE0161597F4F86E0FB0111928A95E9F781
:10F440009E0125563F4F46E050E0CE0183569F4F28
:10F450000E945CD39E0125563F4F44E050E068EF88
:10F4600076E0CE0183569F4F0E945CD3BE016D595A
:10F470007F4F8CE0FB0111928A95E9F79E0125569A
:10F480003F4F4CE050E0CE0183569F4F0E945CD32B
:10F49000E9961CAE1DAE1EAE1FAEE9971CE11150E1
:10F4A00071F09E0125563F4F44E050E0BE016B587D
:10F4B0007F4FCE0183569F4F0E945CD3F0CFE996D9
:10F4C0001CAE1DAE1EAE1FAEE99714E0115071F0D8
:10F4D0009E0125563F4F44E050E0BE016B587F4FE0
:10F4E000CE0183569F4F0E945CD3F0CFE9961CAEAD
:10F4F0001DAE1EAE1FAEE9971BE0115071F09E01CC
:10F5000025563F4F44E050E0BE016B587F4FCE017F
:10F5100083569F4F0E945CD3F0CF8091460F81119C
:10F5200067C0C356DF4FE880F980CD59D040F4E67C
:10F53000EF1AF108C556DF4F88819981CB59D04029
:10F54000C756DF4F99838883C959D04084E690E03D
:10F55000C356DF4F99838883CD59D0409E012556ED
:10F560003F4F44E050E06FE073E0CE0183569F4F81
:10F570000E945CD39E0125563F4F42E050E0BE0101
:10F5800067567F4FCE0183569F4F0E945CD3E3E3C3
:10F59000FAE184918F010F5F1F4F882321F00E94B1
:10F5A000188AF801F6CFB70181E69AE10E94EFB31D
:10F5B000C756DF4F48815981C959D04060E070E09B
:10F5C00084E59AE10E94B5B3E1E5FAE184918F0107
:10F5D0000F5F1F4F882321F00E94188AF801F6CF91
:10F5E000C7010E940D709091460F892B8093460FA2
:10F5F0009091460F81E08927C655DF4F0FB6F894EA
:10F60000DEBF0FBECDBFDF91CF911F910F91FF9055
:10F61000EF90DF90CF90BF90AF909F908F90089524
:10F62000CF92DF92EF92FF920F931F93CF93DF93CE
:10F630006C017A018B01C0E0D0E0CE15DF0581F0CE
:10F64000D8016D918D01D601ED91FC910190F08171
:10F65000E02DC6011995892B11F02196EECF7E0180
:10F66000C701DF91CF911F910F91FF90EF90DF9035
:10F67000CF900895FF920F931F93CF93DF938C0148
:10F68000EB01F42E80E20E94188A8FEFF81611F039
:10F6900084E501C082E40E94188A8AE30E94188AE5
:10F6A000F801608171818281938142E00E94C08D66
:10F6B000488159816A817B8180EB9DE10E94D2B3B0
:10F6C00062E070E080E090E0DF91CF911F910F91B8
:10F6D000FF900C94BEC6CF92DF92EF92FF92C09043
:10F6E0005004D0905104E0905204F0905304609183
:10F6F0004E0470914F0467507109072E000C880B5F
:10F70000990B0E9474E99B01AC01C701B6010E94EC
:10F710006EE987FF1FC020E030E040E450E4C701FD
:10F72000B6010E94EBED0E9434EF7093B00F60932E
:10F73000AF0F0E949058DC01CB01805A9541AF4F2A
:10F74000BF4F8093AB0F9093AC0FA093AD0FB093CE
:10F75000AE0F08C01092AB0F1092AC0F1092AD0F0D
:10F760001092AE0FFF90EF90DF90CF90089590939E
:10F770004F0480934E0480E0AECF8F929F92AF9261
:10F78000BF92CF92DF92EF92FF920F931F93CF938E
:10F79000DF93F0E2FF2EE12CAE2DB0E0BD016F0D46
:10F7A000711D759567956E1511F0F6120BC0E3E9A2
:10F7B000FBE165917491072E000C880B990B0E9458
:10F7C00074E962C09B0121503109220F331F220FBF
:10F7D000331FF901EB5EF44E05911491AB01440F18
:10F7E000551F440F551FFA01EB5EF44EC591D4919D
:10F7F0008017910714F4F62ED1CFC817D90714F447
:10F80000E62ECACFF901E95EF44EE590F490FA01D4
:10F81000E95EF44EC590D490BC01601B710B072EBD
:10F82000000C880B990B0E9474E94B015C01B60136
:10F830006E197F09072E000C880B990B0E9474E942
:10F840009B01AC01C501B4010E94D3E94B015C01ED
:10F85000C01BD10BBE01DD0F880B990B0E9474E910
:10F860009B01AC01C501B4010E94C7EE4B015C01D4
:10F87000B701FF0C880B990B0E9474E99B01AC0146
:10F88000C501B4010E94EBEDDF91CF911F910F9163
:10F89000FF90EF90DF90CF90BF90AF909F908F90B0
:10F8A00008950F931F93CF93DF93CDB7DEB72897BB
:10F8B0000FB6F894DEBF0FBECDBF60914E047091BD
:10F8C0004F04072E000C880B990B0E9474E96D837E
:10F8D0007E838F8398878091500490915104A091EA
:10F8E0005204B091530489839A83AB83BC834DEF58
:10F8F000BE016B5F7F4FCE010196BCDE6091480474
:10F9000070914904072E000C880B990B0E9474E932
:10F910006D837E838F83988780914A0490914B04F6
:10F92000A0914C04B0914D0489839A83AB83BC832E
:10F930004FEFBE016B5F7F4FCE0101969BDEE8EB80
:10F94000FDE184918F010F5F1F4F882321F00E94FA
:10F95000188AF801F6CFE091860FF0E0EC57F04FEF
:10F96000608170E080E090E00E94A68DE3EBFDE115
:10F9700084918F010F5F1F4F882321F00E94188A06
:10F98000F801F6CF6091850F70E080E090E00E9472
:10F99000A68D28960FB6F894DEBF0FBECDBFDF91BF
:10F9A000CF911F910F9108950F930FB70F9300916F
:10F9B0006E000B7F00936E0078940F930BB70F933C
:10F9C0000CB70F921F922F933F934F935F936F93B8
:10F9D0007F938F939F93AF93BF93EF93FF931124E4
:10F9E00094D1FF91EF91BF91AF919F918F917F91B2
:10F9F0006F915F914F913F912F911F900F900CBF8E
:10FA00000F910BBF0F910460F89400936E000F915B
:10FA10000FBF0F911895CF92DF92EF92FF92C09097
:10FA20004A04D0904B04E0904C04F0904D04609157
:10FA300048047091490466507109072E000C880B28
:10FA4000990B0E9474E99B01AC01C701B6010E94A9
:10FA50006EE987FF1FC020E030E040E050E4C701BE
:10FA6000B6010E94EBED0E9434EF7093B60F6093E5
:10FA7000B50F0E949058DC01CB01805A9541AF4FE1
:10FA8000BF4F8093B10F9093B20FA093B30FB09379
:10FA9000B40F08C01092B10F1092B20F1092B30FB2
:10FAA0001092B40FFF90EF90DF90CF9008951092D6
:10FAB000800F80E090E05BDE1092490410924804D1
:10FAC000AADF0E946AB480E090E051DE1092840FB9
:10FAD0002C9810924904109248041092850F80913E
:10FAE000020180728093000108958F929F92AF92DD
:10FAF000BF92CF92DF92EF92FF920F931F93CF931B
:10FB0000DF93F0E4FF2EE12CAE2DB0E0BD016F0DD0
:10FB1000711D759567956E1511F0F6120BC0E5E035
:10FB2000FDE165917491072E000C880B990B0E94E2
:10FB300074E962C09B0121503109220F331F220F4B
:10FB4000331FF901E95FF34E05911491AB01440FA6
:10FB5000551F440F551FFA01E95FF34EC591D4912B
:10FB60008017910714F4F62ED1CFC817D90714F4D3
:10FB7000E62ECACFF901E75FF34EE590F490FA0163
:10FB8000E75FF34EC590D490BC01601B710B072E4C
:10FB9000000C880B990B0E9474E94B015C01B601C3
:10FBA0006E197F09072E000C880B990B0E9474E9CF
:10FBB0009B01AC01C501B4010E94D3E94B015C017A
:10FBC000C01BD10BBE01DD0F880B990B0E9474E99D
:10FBD0009B01AC01C501B4010E94C7EE4B015C0161
:10FBE000B701FF0C880B990B0E9474E99B01AC01D3
:10FBF000C501B4010E94EBEDDF91CF911F910F91F0
:10FC0000FF90EF90DF90CF90BF90AF909F908F903C
:10FC1000089560E08091C10F9091C20FAEDD6093B6
:10FC20005004709351048093520490935304809134
:10FC3000BF0F9091C00F59DF60934A0470934B043B
:10FC400080934C0490934D04A8951092810F0895D1
:10FC5000DF92EF92FF920F931F93CF93DF93F82ED3
:10FC6000D62EE72E8A0180912702882309F439C015
:10FC7000EEE1FAE18491EF012196882321F00E94C0
:10FC8000188AFE01F7CFED2DFE2D8491EF0121960C
:10FC9000882321F00E94188AFE01F7CFE6EAFBE1F3
:10FCA0008491EF012196882321F00E94188AFE0199
:10FCB000F7CFF7FC0BC06F2DFF0C770B880B990B60
:10FCC0000E94A68D8AE00E94188A0BC0E1EAFBE13F
:10FCD0008491EF012196882321F00E94188AFE0169
:10FCE000F7CF8091870F811108C01092270281E021
:10FCF0008093870FC8010E9414AADF91CF911F91B2
:10FD00000F91FF90EF90DF90D2CE0F931F93CF9380
:10FD1000DF9380912A028F37A0F08F579091840F44
:10FD20009093D20F992311F02C9A01C02C98209116
:10FD3000850F2093D10F90910201222369F09095B5
:10FD40000BC09091D20F891708F02C989091D10F89
:10FD5000891728F0909102019072909300018F5FB3
:10FD600080932A029091D00F81E089278093D00F51
:10FD70008091290285301CF4C1E0C80F01C0C0E0A9
:10FD8000823009F4B8C054F4882301F1813009F0BD
:10FD9000E7C088E080937B0085E4C4C0843009F428
:10FDA000C9C00CF4BBC0853009F0DAC09091CF0F08
:10FDB000911102C08093CF0F8091CF0F815080931B
:10FDC000CF0F882309F4CCC0C5E0CAC080912802B7
:10FDD0008F5F80311CF480932802C2C010922802E9
:10FDE0008091810F811113C08091C50F9091C60F32
:10FDF0009093C20F8093C10F8091C30F9091C40F55
:10FE00009093C00F8093BF0F81E08093810F8AE0B1
:10FE1000E5ECFFE0DF011D928A95E9F71092C40F2F
:10FE20001092C30F0091C10F1091C20F119501954F
:10FE3000110980914E0490914F04D1E018161906D3
:10FE40002CF08091840F811101C0D0E080913605A3
:10FE5000909137059195819591098017910734F418
:10FE60004EE35DE16FE57DE180E0F2DE80911C0212
:10FE700090911D029195819591090817190744F4F5
:10FE8000DD2331F041E75DE162E97DE180E0E0DE24
:10FE9000809148049091490411E0181619062CF03D
:10FEA0008091850F811101C010E02091BF0F30912A
:10FEB000C00F80913405909135058217930734F077
:10FEC0004EE45DE16FE57DE18FEFC2DE20911A0225
:10FED00030911B028091BF0F9091C00F8217930742
:10FEE0000CF43EC01123E1F141E85DE162E97DE1FE
:10FEF0008FEFAEDE35C080917A0086FD2EC08091F6
:10FF00007800909179002091C50F3091C60F820F33
:10FF1000931F9093C60F8093C50F22C088E08093F3
:10FF20007B0086E480937C0080917A0080648093DB
:10FF30007A0016C080917A0086FD11C08091780009
:10FF4000909179002091C30F3091C40F820F931FBD
:10FF50009093C40F8093C30F03C0C2E001C0C4E0FC
:10FF6000C09329020E9482BF8091820F9091830FDB
:10FF7000009799F001979093830F8093820F892BBC
:10FF800061F484EA9DE190932C0780932B07DF9125
:10FF9000CF911F910F910C94448ADF91CF911F91C3
:10FFA0000F9108952F923F924F925F926F927F929E
:10FFB0008F929F92AF92BF92CF92DF92EF92FF9279
:10FFC0000F931F93CF93DF9300D01F92CDB7DEB76F
:10FFD0005C017A8369834A01170107FD07C0802FFE
:10FFE000002E000C990B9C838B8304C0E1E0F0E0B1
:10FFF000FC83EB83F90140805180628073808B81A8
:020000021000EC
:100000009C81880F991F880F991F9C838B8389542B
:10001000904F7C01A3019201FC016081718182817A
:1000200093810E946EE9882391F0F701408251820A
:100030006282738211E020E030E0A901C301B201C5
:100040000E9411F018160CF010E0F5011083F50174
:1000500080818230D1F0833009F45EC0813009F0B4
:100060007CC0EB81FC81E954F04F208131814281D9
:100070005381F40160817181828193810E946EE9D4
:1000800087FD6BC082E0F50180838B819C81895460
:10009000904F9C838B83B60180E090E00E9472E9D0
:1000A0009B01AC01EB81FC81608171818281938134
:1000B0000E94EAED9B01AC01F401608171818281B3
:1000C00093810E9411F087FD14C00E9490586B012B
:1000D0007C019101A8EEB3E00E94DBEDC60ED71EB5
:1000E000E81EF91EE981FA81C082D182E282F382A0
:1000F00034C00E949058E981FA81C080D180E280AA
:10010000F380DC01CB018C199D09AE09BF09B7FD55
:1001100024C083E0F50180830F3F19F047E05DE1E3
:1001200002C04AE15DE16EE27DE1802F0F900F9009
:100130000F900F90DF91CF911F910F91FF90EF9053
:10014000DF90CF90BF90AF909F908F907F906F90F7
:100150005F904F903F902F907BCD0F900F900F901E
:100160000F90DF91CF911F910F91FF90EF90DF9053
:10017000CF90BF90AF909F908F907F906F905F9047
:100180004F903F902F9008957F928F929F92AF92C1
:10019000BF92CF92DF92EF92FF920F931F93CF9374
:1001A000DF9320E030E048E452E460915004709125
:1001B000510480915204909153040E9411F018163A
:1001C0004CF4EBE9FBE1E491C1E001C0CC0FEA950E
:1001D000EAF701C0C0E085E9E82E8BE1F82E0BE9D3
:1001E0001BE196E0A92E912CD0E0CC24C394D12C15
:1001F000F7017490F801849077FC23C0892D90E07A
:10020000082C02C0959587950A94E2F780FD19C0E5
:10021000BE01082C02C0759567950A94E2F76170DB
:10022000B62EB1946B2D872D0E948DC56B2D70E07D
:10023000872D0E94F7C5C60101C0880F8A94EAF78E
:10024000982AAA94FFEFEF1AFF0A0F5F1F4FA11021
:10025000CFCFDF91CF911F910F91FF90EF90DF9063
:10026000CF90BF90AF909F908F907F9008954F92C6
:100270005F926F927F928F929F92AF92BF92CF9236
:10028000DF92EF92FF920F931F93CF93DF93CDB73F
:10029000DEB760970FB6F894DEBF0FBECDBF80917A
:1002A000810F811117C060960FB6F894DEBF0FBEA4
:1002B000CDBFDF91CF911F910F91FF90EF90DF9015
:1002C000CF90BF90AF909F908F907F906F905F90F6
:1002D0004F9008959EDC0E9490584B015C01609104
:1002E0004E0470914F04072E000C880B990B0E944E
:1002F00074E969837A838B839C8344E1C42ED12C77
:100300005CE3E52EF12C00E09E012F5F3F4F40E5BE
:1003100054E067EA7FE086EA9FE044DEC090500444
:10032000D0905104E0905204F0905304609138054D
:1003300070913905072E000C880B990B0E9474E907
:100340009B01AC01C701B6010E9411F018160CF018
:1003500009C160911E0270911F02072E000C880BCC
:10036000990B0E9474E99B01AC01C701B6010E9480
:100370006EE987FFF7C000914E0410914F04B80159
:10038000012E000C880B990B0E9474E9A7019601BD
:100390000E94EAED2B013C0120ED3CEC4CE45DE3D6
:1003A0006091780F7091790F80917A0F90917B0F07
:1003B0000E94D3E96D837E838F83988720919D0F60
:1003C00030919E0F40919F0F5091A00FC701B60131
:1003D0000E94EAED9B01AC016D817E818F81988541
:1003E0000E94D3E96D837E838F83988723E333E371
:1003F00043E75FE36091990F70919A0F80919B0F93
:1004000090919C0F0E94D3E99B01AC016D817E818C
:100410008F8198850E94EBED6D837E838F83988713
:100420006093990F70939A0F80939B0F90939C0FFA
:10043000C0929D0FD0929E0FE0929F0FF092A00F5E
:1004400020E030E040E251E4C301B2010E9411F02B
:1004500018160CF430C220E030E040E251ECC30149
:10046000B2010E946EE987FD2FC2012B09F42CC254
:100470008091980F81112CC22091940F3091950F8B
:100480004091960F5091970F29873A874B875C8749
:100490002091740F3091750F4091760F5091770F26
:1004A000C301B2010E94D3E96B017C01A301920157
:1004B00069857A858B859C850E94EBED69877A87B3
:1004C0008B879C876093940F7093950F8093960F02
:1004D0009093970F2091700F3091710F4091720F90
:1004E0005091730F0E94D3E9A70196010E94EBED92
:1004F0002D813E814F8158850E94EAED6B017C0180
:1005000020E030E04FE753E40E9411F020E030E0BB
:10051000A90118160CF4E3C1C701B6010E946EE9E7
:1005200087FD07C0C701B6010E942FEF759567953B
:100530001AC020E030E0A901C301B2010E946EE9B7
:1005400087FF10C0A301920169857A858B859C8500
:100550000E94EAED6093940F7093950F8093960F2D
:100560009093970F60E06093840F8091AB0F909110
:10057000AC0FA091AD0FB091AE0F0097A105B105E2
:1005800021F1A5019401281B390B4A0B5B0B57FD88
:100590001CC06091AF0F7091B00F80E090E00E949E
:1005A00072E99B01AC0160915004709151048091FB
:1005B0005204909153040E946EE987FF81C146EE78
:1005C0005BE168EF7BE180E043DB80917C0F909101
:1005D0007D0FA0917E0FB0917F0FA5019401281B84
:1005E000390B4A0B5B0B57FD0FC0CEDDD501C401A3
:1005F0008C53964FAF4FBF4F80937C0F90937D0FDE
:10060000A0937E0FB0937F0F8091B10F9091B20FA6
:10061000A091B30FB091B40F0097A105B10511F1EE
:10062000881A990AAA0ABB0AB7FC1CC06091B50FC8
:100630007091B60F80E090E00E9472E99B01AC01DE
:1006400060914A0470914B0480914C0490914D0448
:100650000E946EE987FF20C144EC5BE167ED7BE11E
:100660008FEFF6DA6091480470914904072E000C70
:10067000880B990B0E9474E969837A838B839C832E
:1006800095E0C92ED12C24E1E22EF12C0FEF9E0132
:100690002F5F3F4F4AE454E061EA7FE085EA9FE044
:1006A00081DCC0904A04D0904B04E0904C04F09060
:1006B0004D0420E030E040EA50E4C701B6010E945A
:1006C00011F087FDE5C020E030E040EF52E4C701C3
:1006D000B6010E946EE918160CF4DAC06091480465
:1006E00070914904072E000C880B990B0E9474E945
:1006F000A70196010E94EAED4B015C0120916C0F6D
:1007000030916D0F40916E0F50916F0F0E94D3E9A1
:1007100069877A878B879C872091900F3091910F02
:100720004091920F5091930FC501B4010E94EBEDDF
:100730006D837E838F8398876093900F7093910F62
:100740008093920F9093930F2091680F3091690FCF
:1007500040916A0F50916B0F0E94D3E96D877E879D
:100760008F87988B20ED3CEC4CE45DE36091640F47
:100770007091650F8091660F9091670F0E94D3E989
:100780002B013C0120918C0F30918D0F40918E0FE9
:1007900050918F0FC701B6010E94EAED9B01AC0199
:1007A000C301B2010E94D3E92B013C0123E333E3EF
:1007B00043E75FE36091880F7091890F80918A0F02
:1007C00090918B0F0E94D3E99B01AC01C301B20150
:1007D0000E94EBED2B013C016093880F7093890F11
:1007E00080938A0F90938B0FC0928C0FD0928D0FB5
:1007F000E0928E0FF0928F0F2D853E854F855889A0
:1008000069857A858B859C850E94EBEDA301920119
:100810000E94EAED6B017C0120E030E04FE753E4F9
:100820000E9411F020E030E0A9011816BCF5C501C6
:10083000B4010E9411F0181684F4A50194016D8191
:100840007E818F8198850E94EAED6093900F70936E
:10085000910F8093920F9093930F6FE71AC020E04F
:1008600030E0A901C501B4010E946EE987FF10C004
:10087000A50194016D817E818F8198850E94EAEDAA
:100880006093900F7093910F8093920F9093930FBA
:1008900060E06093850F07CDBED8E4CEC701B601F6
:1008A0000E946EE987FDDBCFC701B6010E942FEFE2
:1008B00075956795EECF81E08093980F6FE753CEE3
:1008C00080E00E946B7B81CE81E08093980F4ACEBE
:1008D0001092980F19861A861B861C86D9CDC301E3
:1008E000B2010E9411F018164CF7A301920169851C
:1008F0007A858B859C850E94EAED6093940F7093B6
:10090000950F8093960F9093970F6FE72CCE0F93D0
:100910001F938091630F813019F40E94905808C092
:1009200060915F0F7091600F8091610F9091620FE5
:1009300000915B0F10915C0F20915D0F30915E0F65
:10094000601B710B820B930B28EE33E040E050E00C
:100950000E948DED8091570F9091580FA091590FE3
:10096000B0915A0FBC01CD01620F731F841F951FF8
:100970001F910F9108951092630F10925B0F1092C8
:100980005C0F10925D0F10925E0F10925F0F10922D
:10099000600F1092610F1092620F1092570F109219
:1009A000580F1092590F10925A0F089590916F009E
:1009B000292F227091FF05C090916F009D7F909329
:1009C0006F0034E0839FC0011124FC01EF51F84E09
:1009D0004081518162817381FC01E55BF04F40836E
:1009E00051836283738381E080934A0F222329F02D
:1009F00080916F00826080936F000895BC01209108
:100A0000480F3091490F4091480F5091490F2417DA
:100A1000350711F09A01F7CF81E02617370709F063
:100A200080E0089590911E18E92FF0E0E75AFA4F00
:100A300080839F5F943018F490931E1802C0109228
:100A40001E1880911F188F5F80931F180895CF93F1
:100A5000FC0120812B33A1F020911F18243080F459
:100A6000C62FBC0180911E18F0E68F9FC001112493
:100A7000825A9A4F0E944FF18C2FD4DF81E001C03F
:100A800080E0CF9108952F923F924F925F926F92A4
:100A90007F928F929F92AF92BF92CF92DF92EF920E
:100AA000FF920F931F93CF93DF9300D000D0CDB769
:100AB000DEB79A8389830E949058E981FA81C680C3
:100AC000D780E084F184C114D104E104F10409F079
:100AD000ACC22485222309F469C3328521502487BE
:100AE00021E0230F22874585241301C01286E98166
:100AF000FA8124E0329FE00DF11D1124C684D784D1
:100B0000E088F188E981FA81C282D382E482F582A9
:100B1000DC01CB018C0D9D1DA11DB11D868397832A
:100B2000A087B18784819581892B09F43FC3FFB7E2
:100B3000FD83F894E981FA81228033802101612CC0
:100B4000712C04811581809119028F3121F08F3F22
:100B500009F068C205C0E9E1F8E124912E83DAC00A
:100B60008FE180931902E9E1F8E184918E838F3F50
:100B700009F458C2823009F469C030F5882309F4B9
:100B80004CC0813009F0C6C01092800010928100E4
:100B900080918100886080938100809181008160D4
:100BA00080938100ECEEF7E2E491F0E0EE0FFF1F9E
:100BB000E756F84D85919491E2E3F8E2E491E093F1
:100BC000D60FE1E0EE8330C19E81943009F482C0FB
:100BD00008F460C0953009F09DC010922001109279
:100BE0002101809121018860809321018091210160
:100BF000816080932101ECEEF7E2E491F0E0EE0FEA
:100C0000FF1FE756F84D85919491E2E3F8E2E491F5
:100C1000E093D30F95E09E8307C114BC15BC84B547
:100C2000826084BD85B5816085BDECEEF7E2E4911C
:100C3000F0E0EE0FFF1FE756F84D85919491E2E347
:100C4000F8E2E491E093D70F1E82ABC21092B0009D
:100C50001092B1008091B00082608093B0008091CA
:100C6000B10081608093B100ECEEF7E2E491F0E036
:100C7000EE0FFF1FE756F84D8591949190932D0547
:100C800080932C05E2E3F8E2E491E0932E05F2E094
:100C9000FE8387C210929000109291008091910083
:100CA0008860809391008091910081608093910091
:100CB000ECEEF7E2E491F0E0EE0FFF1FE756F84D9F
:100CC00085919491E2E3F8E2E491E093D50F23E07B
:100CD0002E83AAC01092A0001092A1008091A100C2
:100CE00088608093A1008091A10081608093A10021
:100CF000ECEEF7E2E491F0E0EE0FFF1FE756F84D5F
:100D000085919491E2E3F8E2E491E093D40F84E0DA
:100D10008E838AC0EE81E7FD85C161E08FE10E948C
:100D2000BBC58E818D7F09F083C04801A12CB12CF9
:100D300060E072E18AE790E0A50194010E94AFEDC6
:100D400029833A834B835C8369017A01F1E0CF1AEE
:100D5000D108E108F1082FEFC216D104E104F10433
:100D600009F008F44EC060E472E48FE090E0A50161
:100D700094010E94AFED69017A0181E0C81AD1089F
:100D8000E108F1089E81923009F5EFEFCE16D1040B
:100D9000E104F10409F008F4CBC160E970ED83E0EF
:100DA00090E0A50194010E94AFED69017A01F1E0A4
:100DB000CF1AD108E108F1082FEFC216D104E104DF
:100DC000F10411F008F041C183E027C08FEFC8168D
:100DD000D104E104F104B9F0B0F068E478EE81E008
:100DE00090E0A50194010E94AFED69017A0191E0C4
:100DF000C91AD108E108F108EE81EE2309F49AC17D
:100E000063C181E001C082E09E81911106C095B569
:100E1000987F892B85BD7AC085E09091B100987F3D
:100E2000892B8093B10072C061E08FE10E94BBC545
:100E30004801A12CB12C60E072E18AE790E0A501A5
:100E400094010E94AFED69017A01E1E0CE1AD10868
:100E5000E108F108C114D104F1E0EF06F10488F0D3
:100E600068E478EE81E090E0A50194010E94AFED86
:100E700069017A0181E0C81AD108E108F10883E02C
:100E800001C081E09E81913071F490918100987F42
:100E9000892B80938100452846284728D9F52FEFD4
:100EA0003FEFA90168C0EE81E33071F490919100A9
:100EB000987F892B8093910045284628472851F533
:100EC0002FEF3FEFA90179C0FE81F43071F49091CA
:100ED000A100987F892B8093A100452846284728A8
:100EE000C9F42FEF3FEFA9017AC02E81253071F4AC
:100EF00090912101987F892B8093210145284628D4
:100F0000472841F42FEF3FEFA9017BC04528462831
:100F1000472869F0D801AA0FBB1F91010E94DBEDA1
:100F200028EE33E040E050E00E948DED03C02FEF4B
:100F30003FEFA9018E81823081F12CF4882361F08A
:100F40008130C9F06FC09E81943009F448C0ACF183
:100F5000953009F456C066C0C7BC2093E80F3093A3
:100F6000E90F4093EA0F5093EB0F80916E0082607F
:100F700080936E0057C0D0928900C0928800209361
:100F8000E40F3093E50F4093E60F5093E70F809105
:100F90006F00826080936F0045C0C092B3002093C1
:100FA0002F053093300540933105509332058091E1
:100FB000700082608093700035C0D0929900C0921A
:100FC00098002093E00F3093E10F4093E20F50938D
:100FD000E30F8091710082608093710023C0D092F2
:100FE000A900C092A8002093DC0F3093DD0F40933E
:100FF000DE0F5093DF0F8091720082608093720049
:1010000011C0D0922901C09228012093D80F3093AB
:10101000D90F4093DA0F5093DB0F809173008260F9
:1010200080937300ED81EFBFC1C0DC01CB018C194F
:101030009D09AE09BF09B7FDB9C04698E981FA819B
:101040001682178210861186B1C068E478EE81E0BE
:1010500090E0A50194010E94AFED69017A01F1E0F1
:10106000CF1AD108E108F1082FEFC216D104E1042C
:10107000F10441F138F164E274EF80E090E0A50101
:1010800094010E94AFED69017A01F1E0CF1AD10815
:10109000E108F1082FEFC216D104E104F10409F0D0
:1010A00008F4BACE62E17AE780E090E0A50194010D
:1010B0000E94AFED69017A0181E0C81AD108E10808
:1010C000F10819C084E0A9CE2FEFC216D104E104C3
:1010D000F10409F008F463C062E17AE780E090E08F
:1010E000A50194010E94AFED69017A01F1E0CF1AE8
:1010F000D108E108F1082FEFC216D104E104F10490
:10110000A9F0A0F089819A81AB81BC812AE0B595D4
:10111000A795979587952A95D1F76C017D01F1E008
:10112000CF1AD108E108F10887E077CE86E075CEC6
:1011300082E073CEEFEFCE16D104E104F10469F141
:1011400060F162E17AE780E090E0A50194010E94FD
:10115000AFED69017A0181E0C81AD108E108F10810
:101160009FEFC916D104E104F104A9F0A0F0898130
:101170009A81AB81BC813AE0B595A7959795879503
:101180003A95D1F76C017D01E1E0CE1AD108E10872
:10119000F10885E03CCE84E03ACE83E038CE84E0AE
:1011A00033CE61E08FE10E94BBC5BFCD26960FB65E
:1011B000F894DEBF0FBECDBFDF91CF911F910F918D
:1011C000FF90EF90DF90CF90BF90AF909F908F9067
:1011D0007F906F905F904F903F902F9008950F9366
:1011E0001F93CF93DF93CDB7DEB72C970FB6F8944C
:1011F000DEBF0FBECDBFE6E3F4E080859185A2851A
:10120000B385448155816681778100811181228176
:10121000338109831A832B833C834D835E836F83E1
:10122000788789879A87AB87BC87AE01475F5F4F16
:10123000BE016B5F7F4FCE0101960E9485BE22E406
:1012400034E0AE01475F5F4FBE016B5F7F4FCE0161
:1012500001960E9483B72C960FB6F894DEBF0FBE9E
:10126000CDBFDF91CF911F910F9108952F923F92A3
:101270004F925F926F927F928F929F92AF92BF92A6
:10128000CF92DF92EF92FF920F931F93CF93DF9352
:10129000EB01FC0180809180A280B380C501B40184
:1012A00020E831E541E050E00E948DEDC9016DE696
:1012B00071E00E94C0F06B017C01C501B40120E126
:1012C0003EE040E050E00E948DEDCA01B90128E106
:1012D00030E040E050E00E948DED362E272E062FA4
:1012E000172F8CE3482E512C612C712CC501B401B1
:1012F000A30192010E948DEDB62EA72ECA01B9015D
:10130000A30192010E948DEDCB01C114D104D9F04B
:10131000AF92BF927F936F932F923F92FF92EF9283
:10132000DF92CF9284EE9DE19F938F93DF93CF93D3
:101330000E9440E98DB79EB70E960FB6F8949EBFF7
:101340000FBE8DBF5CC0E114F104C9F0AF92BF9233
:101350007F936F932F923F92FF92EF9284ED9DE1E6
:101360009F938F93DF93CF930E9440E9EDB7FEB731
:101370003C960FB6F894FEBF0FBEEDBF40C0012BE8
:10138000B9F0AF92BF927F936F932F923F9288EC08
:101390009DE19F938F93DF93CF930E9440E98DB798
:1013A0009EB70A960FB6F8949EBF0FBE8DBF27C09A
:1013B000892BA9F0AF92BF927F936F9380EC9DE150
:1013C0009F938F93DF93CF930E9440E9EDB7FEB7D1
:1013D00038960FB6F894FEBF0FBEEDBF10C0AF92A7
:1013E000BF928CEB9DE19F938F93DF93CF930E94ED
:1013F00040E90F900F900F900F900F900F90DF919A
:10140000CF911F910F91FF90EF90DF90CF90BF9001
:10141000AF909F908F907F906F905F904F903F9094
:101420002F900895FC01238121110C9438A2089576
:101430009091C00095FFFCCF8093C6000895EF9275
:10144000FF921F93CF93DF937C0160E000DB182FA6
:10145000882399F0E3E3FAE18491EF012196882350
:1014600019F0E6DFFE01F8CFB70188EF9DE10E9499
:1014700008B482E2DDDF8AE0DBDF812FDF91CF91EC
:101480001F91FF90EF900895DF92EF92FF920F93DC
:101490001F93CF93DF93CDB7DEB76E970FB6F89457
:1014A000DEBF0FBECDBF60912B0770912C07611579
:1014B000710541F14DE150E0CE0101967C010E94A1
:1014C00017E91E8EF7018F010E191F09D190DD203B
:1014D00019F09AE0D912F7CFF701E00FF11F10824F
:1014E000C701ADDF882371F0DD20A9F00F5F1F4F2A
:1014F00080912B0790912C07080F191F10932C0730
:1015000000932B0781E020912B0730912C07232B90
:1015100029F480E003C000E010E0F0CF6E960FB633
:10152000F894DEBF0FBECDBFDF91CF911F910F9119
:10153000FF90EF90DF9008953F924F925F926F92ED
:101540007F928F929F92AF92BF92CF92DF92EF9253
:10155000FF920F931F93CF93DF931F92CDB7DEB708
:1015600093DF811175C280911F18843008F048C044
:101570000E94674BAC0197FF7BC142C08E3409F0DB
:10158000D8C10115110509F4D4C16BE27FE1C8018E
:101590000E9426E97C01892B09F48DC16EE470E07C
:1015A000C80104960E943BF1009709F484C14AE007
:1015B00050E060E070E001960E94C2E66093EC0F9C
:1015C0007093ED0F8093EE0F9093EF0F8090F418CF
:1015D0009090F518A090F618B090F7182FEF821A97
:1015E000920AA20AB20A681579058A059B0509F4D0
:1015F00064C1EF2809F061C188EF9EE10E9443DADF
:101600008091B909882309F423C280911F188111A0
:1016100002C010925210EE24E3944091330C50918A
:10162000340C6091350C7091360C80912F0C909198
:10163000300CA091310CB091320C481759076A0751
:101640007B0708F4E12C00E010E09924939480E6F5
:10165000882E90E3A92E9FE1B92E2DE8322E80919D
:101660001F18843008F0F4C1E110F2C180915210CB
:101670008111EEC180918A0B90918B0BA0918C0B04
:10168000B0918D0B8093330C9093340CA093350C58
:10169000B093360C41E050E0BE016F5F7F4F82E8AF
:1016A0009BE00E94B8A4019719F4898190E002C0E0
:1016B0008FEF9FEFF82E4090330C5090340C6090D9
:1016C000350C7090360C40912F0C5091300C60917D
:1016D000310C7091320CEE24E394441655066606E4
:1016E000770608F4E12C4416550666067706B0F432
:1016F000019609F469C08AE0F81609F488C09DE0F3
:10170000F91609F484C023E2F21619F08AE3F812FC
:1017100095C080915110811191C06EC00E94A9693D
:1017200082E89BE00E9438A280919D0B882359F1AA
:10173000815080939D0B389EC001112441E061E0EF
:101740008E55944F0E94A3D8E0919D0B94E0E99FA1
:10175000F0011124E256F44F40815181628173817E
:101760004093330C5093340C6093350C7093360CCB
:1017700082E89BE00E944EA18091BA098823A1F0E3
:101780009092B90911C01092B9090E9469B90E94DA
:101790006AB4BDD86D3371058105910528F0B0920A
:1017A0002C07A0922B0770DE8091B909811128C007
:1017B000E3E4FFE184916F012FEFC21AD20A88237C
:1017C000D9F036DEF601F6CFEEE1FAE184916F0151
:1017D0009FEFC91AD90A882319F02ADEF601F6CF3D
:1017E000E4E3FFE184916F012FEFC21AD20A88234C
:1017F00019F01EDEF601F6CF83E2F81208C005C02C
:1018000023E2F21222C100E010E0909252101092F6
:1018100051100115110519F40E9437810CC08091F7
:101820001E18889E000D111D1124F801E25AFA4F6E
:10183000108280E0F7D800E010E011CF0F351105DD
:1018400008F00DCF9BE3F91202C0909251108091E5
:101850005110811104CF80911E18F801889EE00D6F
:10186000F11D1124E25AFA4FF0820F5F1F4FF7CE9D
:10187000982F2091F2183091F3188A3019F09D308A
:1018800009F0B1C0109250102115310519F40E94D1
:10189000378169CEF901E051F04F10821092F318B0
:1018A0001092F21800EF1FE0F8018191803209F0E8
:1018B00065CE8F01F9CFC8017ACE6AE270E0C80127
:1018C0000E9473F19C01009701F1982F901BF12C5D
:1018D000992339F09150F801E90FF11D8081F82624
:1018E000F7CF4AE050E060E070E0C90101960E9445
:1018F000C2E6CF2CD12CE12CF12C6C157D058E0588
:101900009F0531F089ED9EE179CE8FEA9EE176CE9A
:101910008091EC0F9091ED0FA091EE0FB091EF0F31
:101920008093F4189093F518A093F618B093F718D5
:101930000EC08091B709882351F065EF73E0C801AC
:101940000E9446F1892B19F085E89EE157CE8091DF
:101950002702811126C067E470E0C8010E943BF1B4
:101960000097F9F04AE050E060E070E001960E94D4
:10197000C2E697FD16C064307105810591052CF013
:10198000653071058105910561F4EEE0FEE1849119
:101990007F019FEFE91AF90A882319F049DDF70161
:1019A000F6CF69EF73E0C8010E9446F1892B11F46C
:1019B000109220026EEF73E0C8010E9446F1892B5D
:1019C00021F485E09EE10E9414AA63E074E0C8015E
:1019D0000E9446F1892B11F40E941D9861E080EF6E
:1019E0009FE035D8C0CD2F3531050CF0BCCD9C35EE
:1019F000C1F40E94674B97FDB6CD20915010211184
:101A0000B2CD2091F2183091F318A9014F5F5F4FCA
:101A10005093F3184093F218F901E051F04F80838E
:101A2000A2CD9B3319F481E0809350108091501027
:101A3000811199CDC90101969093F3188093F21802
:101A4000F901E051F04F40838ECD10925110E4CE59
:101A50000F90DF91CF911F910F91FF90EF90DF904A
:101A6000CF90BF90AF909F908F907F906F905F903E
:101A70004F903F9008958F929F92AF92BF92EF92B6
:101A8000FF920F931F93CF93DF93CDB7DEB7A0974D
:101A90000FB6F894DEBF0FBECDBF6115710581058D
:101AA000910589F100E0842E912CA12CB12C102FEE
:101AB000EE24E394F12CEC0EFD1EE00EF11C07FD6C
:101AC000FA94A50194010E948DEDF7016083B9019C
:101AD000CA010F5F611571058105910541F71F3F2F
:101AE00021F1E1E0F0E0EC0FFD1FE10FF11D17FD2A
:101AF000FA9580818A3010F097E301C090E3890F56
:101B000097DC1150ECCF80E3A0960FB6F894DEBFBF
:101B10000FBECDBFDF91CF911F910F91FF90EF903E
:101B2000BF90AF909F908F9083CCA0960FB6F89403
:101B3000DEBF0FBECDBFDF91CF911F910F91FF9000
:101B4000EF90BF90AF909F908F900895CF92DF92CB
:101B5000EF92FF926B017C0197FF0AC08DE268DC77
:101B6000F094E094D094C094C11CD11CE11CF11CF1
:101B70004AE0C701B601FF90EF90DF90CF907BCF96
:101B80008F929F92AF92BF92CF92DF92EF92FF928D
:101B9000CF936B017C01B42E20E030E0A9010E94BC
:101BA0006EE987FF06C08DE243DCF7FAF094F7F8A0
:101BB000F094C0E060E070E080E09FE3CB1541F07E
:101BC0002DEC3CEC4CEC5DE30E94D3E9CF5FF6CF0B
:101BD0009B01AC01C701B6010E94EBED6B017C01DA
:101BE0000E9434EF4B015C014AE045DFCC2379F1E0
:101BF000C501B4010E9472E99B01AC01C701B601A5
:101C00000E94EAED6B017C018EE212DC20E030E004
